:020000040800F2
:104000000050002011F300087DC4000881C400089E
:1040100085C4000889C400088DC4000800000000A1
:1040200000000000000000000000000095C400082F
:1040300091C400080000000099C40008E99200083B
:104040009DC40008A1C40008A5C40008A9C40008B4
:10405000ADC40008B1C40008B5C40008B9C4000864
:10406000BDC40008C1C40008C5C4000800000000A9
:104070000000000000000000000000000000000040
:104080000000000000000000E5C40008E9C40008CA
:10409000F9C4000809C5000819C5000829C50008A9
:1040A0002DC5000831C5000835C5000839C5000810
:1040B0003DC5000841C5000845C5000849C50008C0
:1040C0004DC5000851C5000855C5000859C5000870
:1040D0005DC5000861C50008ED89000869C50008D4
:1040E0009949000871C5000875C500080000000066
:1040F00000000000000000000000000000000000C0
:0C41000000000000000000005FF800005C
:1041100030BF704720BF704740BF7047BFF36F8FFD
:104120007047BFF34F8F7047BFF35F8F704701DF5A
:104130007047EFF31480704780F31488BFF36F8FDC
:104140007047EFF30980704780F309887047EFF3F9
:104150000880704780F30888704772B6704762B66F
:10416000704771B6704761B6704780F31188704729
:10417000EFF31280704740BA704700BA70470000F2
:1041800010B500F033FC0B4C0B490C4A0C4B48B1FA
:104190004FF0010C0B4884F800C00B4C1860146001
:1041A000086006E020700948086009491160094A62
:1041B0001A6010BD180B0020400B0020240C0020BA
:1041C000B40B0020618C0008619A0008F58C00088F
:1041D000319200087991000837B509F06BFD6A4B00
:1041E00000254FF480301D7009F084FD09F0E8FED1
:1041F0000128044627D1102009F046F8284609F086
:10420000C9FD284609F0DAFD4FF4806009F0CCFDC5
:104210004FF440304FF4E01109F098FD204609F0CA
:10422000A1FD392009F0B6FE0028FAD0022009F0DD
:1042300013F8022009F09CFD09F0A4FD0828FBD129
:10424000514B01221A700420012109F059FE032369
:104250008DF80630153301A94C488DF807304FF41E
:104260008073ADF8043009F043FA062009F08CFEA3
:104270000120014609F044FE454C4FF480414FF0C7
:10428000006009F039FC4FF4407009F097FB00F032
:104290000FFC00F093FDFFF773FF00F0FBF805F053
:1042A0004DF905F0ADF804F0CFFA00F077F820787A
:1042B00004F0FCFBE07804F055FB364B1B7823B987
:1042C00022696079A16804F0AFFD324B1B780BB115
:1042D00005F06EFC06F0E2F900F010FA07F0A0FE1F
:1042E000012000F0B7FB00F04FF901F033FE05F0BC
:1042F00067FC06F019FA284B4FF400425A6105F0AA
:1043000079F8044603F020FC06F01CFA05F092FC54
:1043100005F070F8001B0028B8BF4042B0F57A7F66
:1043200024DD1C4D2B782C4683B100F05FFB68B96F
:10433000287005F0FDFB05F0E3FAFFF721FF144BB1
:104340001A695879996804F06FFD0CE0237853B925
:1043500000F04CFB38B104F02BFD01232370FFF774
:104360000FFF05F025FC05F045F8044600F048F97C
:1043700000F03AF90028C5D006F090F901F0EAFD06
:1043800006F0D2F9BEE700BF140C0020000801407F
:1043900008000020180B002000100140114B82B0D3
:1043A0001B78E3B1104B04225A6102221A610023E8
:1043B00001E0019B01330193019A0C4B9A42F8D919
:1043C000094B04221A6102225A61002301E0019B79
:1043D00001330193019A054B9A42E3D8F7E702B003
:1043E000704700BF540B0020000C01403F0D03003C
:1043F00010B1012809D104E0044B4FF400625A6166
:1044000003E0024B4FF480621A617047000C0140D8
:1044100010B1012809D104E0044B4FF400621A6185
:1044200003E0024B4FF480625A617047000C014078
:1044300038B50546002455FA04F2E3B212F0010F34
:10444000184602D0FFF7E4FF01E0FFF7D1FF013487
:10445000082CF0D138BD00BF18B1012806D00020CB
:104460000AE0064BD868C0F3C02005E0034BD868CB
:1044700080F48060C0F38020704700BF000C0140D2
:1044800008B1002003E0024B9868C0F3C0007047F9
:10449000000C014062B6704772B6704718B9024B03
:1044A0004FF400425A6170470010014018B9024BA6
:1044B0004FF400421A6170470010014008B100201B
:1044C00005E0034BD3E90023100A40EA036070477C
:1044D000580B0020F8B50D460446B8B9FFF7DCFFCD
:1044E0000B492A464FEAE273C1E90023D1E900678C
:1044F0003B0243EA16633202C1E90023054B1C600C
:10450000054B1C60054B9C84FFF7C4FFF8BD00BF42
:10451000580B0020600C0020380B002000080040E1
:1045200010B9024B09011960704700BF600B0020F1
:1045300020BB11F0040F10D011F0100F04D0104B5D
:104540009A6842F400420CE00D4B9A6822F4004253
:104550009A60DA6842F4004207E0094B9A6822F454
:1045600000429A60DA6822F4004211F00801DA6031
:10457000044B02D001221A7000E01970704700BF8E
:104580000004014030020020084B4FF400721A6012
:10459000074B10B50024204610211C60FFF7C0FF18
:1045A00020462146FFF7C4FF10BD00BF480B002086
:1045B000440B002010B9024B09011960704700BF7D
:1045C0000400002008B9014B5970704730020020E8
:1045D000044B98780138C0B201288CBF002001201C
:1045E000704700BF30020020044B9878012801D0AA
:1045F000002001E002229A70704700BF30020020C4
:10460000082008B504F014FF592804D9064B9A78FD
:104610004AB9013206E0082004F00AFF542802D803
:10462000014B00229A7008BD3002002008B5032813
:1046300003D8DFE800F0040D1217002016E0002078
:1046400004F0F6FEB0F5006F94BF002001200DE0ED
:10465000074B9868C0F3C01008E0054B9868C0F39A
:10466000801003E0034B9868C0F3C03008BD00BF62
:10467000000C01400008014038B500242546E0B296
:10468000FFF7D4FF20B10123A34043EA0505EDB2B3
:104690000134082CF3D1284638BD00BF10B5FF21E6
:1046A0000022032000F014FBFF210122032000F070
:1046B0000FFBFF210022032000F00AFBFF2104462C
:1046C0000122032000F004FB034B40EA04205B6856
:1046D00003EA9000181A10BD3002002008B5FFF759
:1046E000DDFF052801D8012007E0FFF7D7FF40F2E2
:1046F000F933984294BF0020012008BD38B51E4C04
:10470000002021694909FFF755FF2169002001F0C8
:104710001F01FFF757FFFE210022032000F0D8FA07
:1047200040210122032000F0D3FA00210A46032091
:1047300000F0CEFA002104460122032000F0C8FA5E
:10474000082C0E4B05D14FF400629A6040F6FF72C0
:1047500004E04FF400729A6040F2FF325A60FFF7B3
:104760009DFF064B040224464FEAE475C3E9064563
:10477000C3E90445D86038BDB80B002030020020E2
:104780002DE9F84304F036FE624C2062FFF786FF05
:10479000E368606298423EDDA268C11A91420BDA7A
:1047A0005D4BA56A1A684D195143D4E90667721822
:1047B00047EBE173A5622BE094F801C0564A1CF068
:1047C000040F12D063681668C31A5E432CF0040C01
:1047D00036464FEAE677A36200220023C4E9066763
:1047E00084F801C0C4E904234EE0656816685A19CC
:1047F0000132121A7243D4E90667A36AED43ED1839
:10480000B6EB020867EBE27942464B466918A162B3
:10481000C4E9062338E037DAA1681A1A8A420EDAA8
:104820003D4DA16A2D68C91A6A43D4E90667B6EB03
:10483000020867EBE27942464B460918E7E76178E0
:10484000354A11F0040F0FD0126821F004014243E1
:1048500012464FEAE273C4E9062300220023617086
:10486000C4E90423A0620FE0616812680131CB1A29
:104870001B185A43D4E90667B61847EBE277A26AD9
:10488000C4E906679B18A362224B9D6ADA6A196B1A
:10489000AA1A82EAE27CACEBE27C8C452CD942F28B
:1048A00010714A431E6A5C6B3C21341B92FBF4F28C
:1048B00051434FF4807C91FBFCF181EAE172A2EB61
:1048C000E172D96340F6B8318A425E63DD629C636F
:1048D00001DDC82219E0B2F57A7F01DD642214E01F
:1048E000322A01DD0A2210E00A2A01DD05220CE04D
:1048F000012A0BDD012208E0196A5A6B8A1AB2F507
:10490000FA6F03D90022DA6301321A63014BD860CF
:10491000BDE8F883300200200400002038B50D46C1
:1049200018BB124CFFF72CFFD4E90601002901DB6C
:10493000626803E06268404261EB41011202124684
:104940004FEAE2730DF004FBC4E9042328464FEA62
:10495000E071064C0B02020243EA1063D4E9040141
:10496000801841EB0301C4E9060138BD3002002084
:1049700008B508B100200CE0FFF702FF054BD3E9B2
:104980000401D3E90623121A63EB0103100A40EA7B
:10499000036008BD3002002008B54FF4004008F065
:1049A00055FC0C4A002313600B4A002013600B4A8D
:1049B0000021C2E900010A4A93840A4B1B7843B9DB
:1049C000094B9A6822F400429A60DA6822F40042A5
:1049D000DA6008BD600C0020380B0020580B002066
:1049E00000080040300200200004014008B5084BD8
:1049F000587E10F0010005D0002006F023FF80F063
:104A0000080001E006F01EFFC0F3C00008BD00BFB3
:104A10000800002037B5044658B1002003240246A0
:104A200034212346009407F083F900202A21084A04
:104A30000AE00325024634212B46009507F078F959
:104A400020462A2140F2FF7207F02CF93EBD00BF3C
:104A500001F8FFFF37B5044658B100200324024691
:104A600054212346009407F063F900204A21084AA4
:104A70000AE00325024654212B46009507F058F919
:104A800020464A2140F2FF7207F00CF93EBD00BFFC
:104A900001F8FFFF08B510B109F038F801E009F09E
:104AA0003DF808BD08B5C90805F062FA08BD00BFA9
:104AB0002DE9F0457F488BB0DFF80482012108F032
:104AC000A7FE09AD0420012109F01AFA03241026DB
:104AD000404642F206032946ADF824308DF82640C0
:104AE0008DF8276008F004FE0623734F4046C8F88F
:104AF00014304FF0040A4CF208632946ADF8243014
:104B00008DF826408DF827A008F0F2FD082001213D
:104B100009F0F6F941F6164338462946ADF8243037
:104B20008DF826408DF8276008F0E2FD41F216432B
:104B30003B614FF40063384629467B614FF0E80340
:104B4000ADF8243008F500688DF827A08DF82640D0
:104B500008F0CEFD3046012109F0D2F94EF20003F3
:104B600029464046ADF824308DF826408DF8276060
:104B700008F0BEFD4FF460430121C8F810304F48E3
:104B800008F046FE00231A4619464D4C4FF40055D6
:104B900065612046A468013314F4804F4FF400543B
:104BA0000461806808BF013110F4804F18BF0132E2
:104BB0000A2BEAD10A2903D10A2A01D1012200E0F5
:104BC0000022404B01211A703A4808F021FE0420CF
:104BD00001213D4C09F094F900214FF4805008F078
:104BE00017FE0121042009F099F903AD20460AF0CF
:104BF00067F9284609F05AFD294620464FF000057E
:104C00004FF0FF33ADF81030ADF80C50ADF8125046
:104C1000ADF80E5009F0F2FB0022134603212046A6
:104C200009F0FAFD684609F055FD4FF008072046E7
:104C30006946ADF808700AF0DFF84FF004036946E2
:104C40002046ADF800300AF0D7F8204641F65F6103
:104C50000AF028F820460121A58409F04FFD002024
:104C60000F2108F003FE012406A84FF40043069329
:104C70008DF81D708DF81C508DF81E4008F080FADC
:104C8000124B08A89A686E4622F480629A60DA682D
:104C90008DF8234022F48062DA6028238DF82030DA
:104CA0008DF822508DF8215008F092FE0BB0BDE82F
:104CB000F08500BF00023000000C0140000430000D
:104CC00000080140540B002000080040000401408F
:104CD00070B504460D461646032864D8DFE800F098
:104CE0000205080D4FF480520FE04FF4804201E0BE
:104CF0004FF400522D4B5A611AE02D4A138823F0CD
:104D000002031B041B0C138010222A4B5A612848F3
:104D1000022109F057FA0028F9D02946244809F061
:104D2000F5F92348012109F04DFA0028F9D00FE0E8
:104D30002148022109F046FA0028F9D029461E48E8
:104D400009F0E4F91C48012109F03CFA0028F9D0E7
:104D5000E6B1032C27D8DFE804F002070A0F154B51
:104D60004FF480521A6119E04FF4804201E04FF491
:104D700000520E4B1A610FE00E4A0D4B10211161CB
:104D80001A8892B242F002021A8007E0032C0AD875
:104D9000DFE804F004020204074800E0044809F0D8
:104DA000B7F9C0B200E0002070BD00BF00100140A4
:104DB00000380040000C0140003001402DE9F04F68
:104DC00001218BB04FF4804009F0A8F8494C012034
:104DD00009AF014609F094F803264FF0180B20465E
:104DE00039464AF20003DFF81491ADF824304FF051
:104DF000040A8DF826608DF827B008F079FC20466B
:104E000039464FF480430DF11008ADF824308DF889
:104E100026608DF827A008F06BFC4FF48273002405
:104E200002224FF4007C012548464146ADF812307D
:104E30004FF00803ADF81620ADF81AC00392CDF874
:104E400008C0ADF81C30ADF81040ADF81440ADF816
:104E50001850ADF81E40ADF8204009F0E3F8484680
:104E6000294609F01BF929464FF4805009F048F80B
:104E700009F550492846214608F0CAFC48463946FB
:104E80004FF0A003ADF824308DF827B08DF82660E0
:104E900008F02EFC484639464FF04003ADF8243068
:104EA0008DF826608DF827A008F022FC039ADDF823
:104EB00008C04FF482734146ADF812300E484FF0EF
:104EC0002803ADF81620ADF81AC0ADF82040ADF8B3
:104ED0001040ADF81440ADF81850ADF81C30ADF8E6
:104EE0001E4009F09FF80448294609F0D7F80BB096
:104EF000BDE8F08F000C0140003001400038004058
:104F0000014B1878704700BF700200202DE9F8456A
:104F1000054614460E4600294BD0002849D0814250
:104F200047D04FEA42185FFA88F848F0060739463A
:104F3000002006F071FD48F00C018246002006F0CA
:104F40006BFD804628460CF0C5FD054630460CF04A
:104F5000C1FD014628460CF0C9FE064650460CF03D
:104F6000B9FD31460CF0C2FE0CF0D2FF05464046BA
:104F70000CF0B0FD31460CF0B9FE0CF0C9FF0E4943
:104F8000002814BF80464FF001083046002D08BFAE
:104F900001250CF095FF18B14146204606F0B6FFFA
:104FA00039462A46002006F0E9FD044BE4180123A7
:104FB0002371BDE8F88500BF0000A0417002002009
:104FC00070B50D4D044645192B799BB1C6B20B4BFC
:104FD000710141F0060153F8202001F0E6010020A4
:104FE00006F060FE064B304653F8241006F08EFFA4
:104FF00000232B7170BD00BF70020020140B002035
:105000001007002013B5A64CA078002840F01F839D
:105010006378A52B00F0448259D8852B00F0E980F5
:1050200027D8072B00F01D810FD8032B00F0E1805B
:1050300005D8012B00F0B58000F2BD80ABE0052B58
:1050400000F0EF8000F20281D9E0812B00F0A9800E
:1050500009D80D2B00F03281802B00F09C800C2BA6
:1050600040F0F3820AE1832B00F0C98000F2A380B4
:1050700036E1952B00F0688115D88C2B00F0558116
:1050800008D8872B00F03681C0F0CB808A2B40F007
:10509000DC8235E1932B00F0118100F2EF808D2B43
:1050A00040F0D3824AE1A12B00F0DB8109D89A2B92
:1050B00000F07A81A02B00F0CE81992B40F0C582C0
:1050C0005DE1A32B00F0D78100F2DB81CDE1B72BAE
:1050D00000F06D8228D8AD2B00F0248210D8A92BC7
:1050E00000F0068205D8A72B00F0F68100F2FA81C5
:1050F000E3E1AB2B00F00582694C00F20882FBE192
:10510000B12B00F02F8206D8AF2B00F01582644C33
:1051100000F218820AE2B52B00F02E8200F23482EF
:10512000B22B40F0928221E2CC2B00F0798115D88D
:10513000C22B00F0578108D8C02B00F0928000F2FB
:105140004C81B82B40F0818235E2C72B7ED0C82B32
:1051500000F05681C32B40F0788249E1D52B00F056
:105160006E8109D8D22B00F03582D42B00F05F81FC
:10517000D12B40F06A8224E2D82B00F0408203D881
:10518000D62B40F062825EE1D92B00F04182DA2B0F
:1051900040F05B8251E2424B00205A680146DB78C6
:1051A00004E03F4B00205A68DB78022143EA0222E8
:1051B00006F0E4FC4EE23A4C0020E37862680821F5
:1051C00043EA022206F06EFDE378A17862684901A5
:1051D00043EA0222002A41F00601B8BF524201F020
:1051E000E601002006F05EFD2E4AA378D3180122C6
:1051F000DFE12B4B00205A680A21DB7875E0284C50
:105200000020E3786268062143EA022206F04AFDA4
:10521000E2786068A37842EA0020224A22499A187C
:105220000FE01F4C0020E378616843EA012106F09B
:105230006DFEE2786068A37842EA0020194A1B49B3
:105240009A1841F823000023137103E2144B184A03
:10525000D978184B01201B781070174A022B517215
:10526000D8E00F4B0122D978124B1878104B1A70E6
:10527000114B9972002840F0ED81CEE014210020FE
:1052800001AA06F01BFC064A9DF805305168D27849
:1052900052EA012114BF43F0020323F0020362E04B
:1052A0008C06002070020020140B00201007002044
:1052B0001C0C0020200C0020B80B00201421002022
:1052C00001AA06F0FBFBA24A9DF805305168D2788E
:1052D00052EA012114BF43F0010323F0010342E02D
:1052E0009B4B00205A68DB78042143EA022206F037
:1052F000D9FCAFE1964B00205A680E21DB78F4E729
:1053000001AC22461421002006F0D8FB904B224627
:105310009978DB78490141F0140101F0F401002093
:105320008DF8063006F066FD94E1E378894AC3F112
:105330000801C9B2D37205F035F98BE1844B002026
:105340005A681A21DB78D0E7142101AA06F0B6FBCF
:105350006168E2789DF8053052EA012114BF43F0FC
:10536000040323F004038DF80530794B002099786D
:1053700001AA490141F0140101F0F401D2E701ACA6
:1053800022461821002006F099FB714A9DF805304D
:105390009178D278490102F00F0223F00F0341F017
:1053A000180142EA030311E001AC22461821002053
:1053B00006F084FB664A9DF805309178D278490161
:1053C00003F00F0341F0180143EA021301F0F80162
:1053D000224600208DF80530A4E75D4BDA785D4B5E
:1053E0001A7237E1E378626843EA0222594B2AE1F4
:1053F000574B5A68DB7843EA0222564B5A6029E140
:10540000534B554AD978554B01201B781070514A9F
:10541000032BD17740F01E810138FFF743FB19E1E0
:10542000E378626843EA02224A4BDA8112E1484B90
:105430005A68DB7843EA0222464B5A610AE1E27875
:10544000444B9A7706E1424B5A68DB7843EA0222E2
:10545000404B9A83FEE03E4B0020D97805F094F84B
:10546000F8E0E17805F086F8F4E0394B0020D978CF
:1054700004F060FFEEE0364B0020D97804F04EFFD8
:10548000E8E0002004F00CFC314C20B9E178A07871
:1054900004F02CFFDEE0E178A07804F0F7FED9E01C
:1054A00004F0FEFBE178A37818B9184604F012FF67
:1054B000D0E0184604F0D2FECCE0002004F0F0FB6F
:1054C000234C20B9E178A07804F0F8FEC2E0E1783E
:1054D000A07804F0CFFEBDE01D4B0020D97804F089
:1054E000E1FEB7E01A4B0020D97804F0E5FDB1E009
:1054F000E17804F0D5FDADE0E178002004F0C4FDD2
:10550000A8E0134B0020D97804F0B2FDA2E0E178C6
:10551000002004F0A1FDA178114BE27803EBC10358
:105520005A7197E0E17804F03BFD93E094F90310A1
:10553000002004F029FD8DE0054B0020D97804F00F
:10554000BDFF87E0E178002004F0ACFF82E000BFFF
:105550008C060020B80B00201C0C0020200C002022
:10556000280B0020E17804F091FF73E03A4B002013
:10557000D97804F07FFF6DE0374B5A68DB7843EA57
:105580000222364B9A6165E0334A354B5068D27837
:1055900042EA0020186010B9597904F05DFD2E4BE5
:1055A000304A9878125C012A54D1D97835E7E278EC
:1055B0002B4B1A714EE0284B0020D97804F0A2FE44
:1055C00048E0254B00205968DB7843EA0121FFF7CA
:1055D000A5F93FE0204C0020E378626803F01F014A
:1055E00043EA02221D4B1A61FEF7ECFFE378616883
:1055F000A07843EA01214911FEF7DCFF2AE0164BAF
:1056000000205968DB7843EA0121FEF763FF21E0BF
:10561000114C0020E378626803F01F0143EA022284
:10562000114B1A60FEF784FFE3786168A07843EAC3
:1056300001214911FEF774FF0CE0074B5A68DB7833
:1056400043EA0222094B1A6004E0032200E004222C
:10565000074B1A701CBD00BF8C060020B80B002041
:10566000280B0020200C0020480B0020440B0020B9
:105670000407002013B5814B9A78002A40F062821B
:105680005B787F4CDA2B00F23E82DFE813F0DB0020
:10569000DE00E400E700EC00EE00F000F3000101A2
:1056A0001E01350123010A0114013C023C023C02A7
:1056B0003C023C023C023C023C023C023C023C02FA
:1056C0003C023C023C023C023C023C023C023C02EA
:1056D0003C023C023C023C023C023C023C023C02DA
:1056E0003C023C023C023C023C023C023C023C02CA
:1056F0003C023C023C023C023C023C023C023C02BA
:105700003C023C023C023C023C023C023C023C02A9
:105710003C023C023C023C023C023C023C023C0299
:105720003C023C023C023C023C023C023C023C0289
:105730003C023C023C023C023C023C023C023C0279
:105740003C023C023C023C023C023C023C023C0269
:105750003C023C023C023C023C023C023C023C0259
:105760003C023C023C023C023C023C023C023C0249
:105770003C023C023C023C023C023C023C023C0239
:105780003C023C023C023C023C023C023C02DB008C
:10579000DE004201EC00E400E700EE0045013C02BF
:1057A0003C0248013C02500156013C023C023C02D2
:1057B0003C023C0214010A0159013C023C023C0239
:1057C00063016D012301350101013C023C02AB0183
:1057D000AF01B301B701BB01C901D701E501E9017F
:1057E000ED01F101F501F901FC01000205020902D8
:1057F0000D021102150219021C021F0221022402CD
:105800003C023C023C023C023C023C023C02F300F3
:10581000760179017B017E0180013C02F00082016A
:105820003C023C023C0285013C0288018A01A00145
:1058300028022C023C02A201A501A8012F0232027B
:10584000360238020020014601E00020022106F065
:10585000E3F8606079E10020082101E000200A21DE
:1058600006F014F9F5E7074B4AE1074B48E1074B0F
:105870005B7A46E1054B9B7A43E100BF8C06002032
:1058800004070020140B002010070020B80B002094
:10589000002005F0D7FF9D4B9B785B0050FA03F387
:1058A00010E00020142101AA06F008F99DF8053047
:1058B000C3F3400325E10020142101AA06F0FEF8FD
:1058C0009DF8053003F001031BE1914B9B68C3F386
:1058D000C03316E17C21002001AA06F0EFF88B4BC3
:1058E00002219A789DF80630520011FA02F21A420B
:1058F0000CBF0023012304E101AA00207C2106F053
:10590000DDF8824B9DF806209B785B0052FA03F38A
:10591000D8E700200421A3E700200E21A0E7002003
:10592000142101AA06F0CAF89DF80630E9E000202B
:1059300004F096F9C0F108008BE700201A218FE7E8
:105940000020142101AA06F0B9F89DF80530C3F330
:105950008003D6E00020182101AA06F0AFF89DF8D8
:10596000053003F00F03CCE00020182101AA06F057
:10597000A5F89DF805301B09C3E0664B1B7AC0E013
:10598000644BBDE0634B5B68BBE0634BB8E0634BCB
:10599000B6E0604BDB7FB4E05E4BDB89B1E0604B8F
:1059A000AEE0604B00221B78626013B15E4B0132A7
:1059B0005A605E4B5B4A1B780021117023B15A4B31
:1059C0005A6842F002025A600022584BBCE0584B21
:1059D00077E0504B5B6994E04E4B9B7F91E04D4BE1
:1059E0009B8B8EE0002004F043F932E7002004F0A6
:1059F00047F92EE7002004F04BF92AE7002004F0D5
:105A00004FF926E7002004F04BF9474C3F4B18B9FB
:105A1000987804F055F91CE7987804F071F918E7C4
:105A2000002004F03DF9404C384B18B9987804F048
:105A30004FF90EE7987804F073F90AE7002004F0B4
:105A40002FF9394C314B18B9987804F049F900E72F
:105A5000987804F05DF9FCE6002004F049F9F8E6D6
:105A6000002004F065F9F4E6002004F069F9F0E69E
:105A7000002004F06DF9ECE6002004F071F9E8E68E
:105A80002C4B5B793DE0002004F07AF9E1E6002040
:105A900004F07EF940B2DCE6002004F08BF9D8E691
:105AA000002004F08FF9D4E6002004F093F9D0E64A
:105AB000002004F097F9CCE6002004F0A3F9C8E632
:105AC0001D4B1B781DE0134B9B691AE0194B17E027
:105AD000184B1B7915E0002004F0EAF8B9E6002025
:105AE000FEF746FFB5E60B4B1B690AE0FEF7D6FD55
:105AF000AFE60020FEF7E2FCABE6104B00E0104BF7
:105B00001B68636021E0032323701EE08C060020E5
:105B100000080140B80B00201C0B0020DC0B00200B
:105B2000500B0020AC0B002004070020340B002099
:105B3000B00B0020280B0020240B0020480B002075
:105B4000440B00200A4B04221A700A4B1B786BB1DD
:105B5000074B09495A68094B0A601AB91A6842F09A
:105B6000080202E01A6822F008021A601CBD00BF99
:105B700004070020FE060020EC060020940600200A
:105B800010B51B4A5378142B2DD8917871B95468ED
:105B9000D078184A1849927E40EA042041F8230040
:105BA00022B31BB303F5C270013013E0FF2918D1F3
:105BB00063B94FF4C364114920460919042204341F
:105BC00002F07AFCB4F5CD6FF5D10FE003F5C270A9
:105BD0000949013001EB83018000042202F06CFCD2
:105BE00004E0042200E00322054B1A7010BD00BF40
:105BF0008C06002008000020980600208400002069
:105C00000407002038B51F4C6578142D36D8A078CD
:105C100010F0800F18D010F0010F06D000200221E4
:105C200005F0FAFE184B43F82500184B9B7E43B352
:105C3000144B5B782BB303F5C2701349013001EBB1
:105C400083018000042214E0B0B9022105F0E4FED3
:105C50000E4A0D4B927E43F8250092B1617881B1D6
:105C6000A0780422091801F5C270013003EB81010C
:105C7000800002F021FC04E0042200E00322044B37
:105C80001A7038BD8C0600209806002008000020FD
:105C90000407002038B5654CA07808B10422C2E0A2
:105CA0006378952B1DD8932B7DD20D2B0AD80C2B06
:105CB00079D2052B4FD001D8042B09E0062B66D0F2
:105CC000072B1EE0862B46D005D8822B6ED0832B67
:105CD00040F0A88028E08C2B6CD08D2B40F0A28067
:105CE00079E0C32B00F087800ED8B52B77D004D88D
:105CF000993B012B00F296806FE0C12B72D077D8D0
:105D0000C02B40F08F8048E0CC2B7AD005D8C72B31
:105D10003DD0C82B40F0868070E0D52B78D0D62BB4
:105D20007AD0D42B7ED16FE0404D0020062106F0C2
:105D3000CBF8AC780020610141F0060101F0E601EA
:105D400005F0A4FE3A4AAB78D3183A4A42F8240048
:105D500000221A7169E0354D00200C2106F0B4F8DC
:105D6000AC780020610141F00C0101F0EC0105F07C
:105D70008DFEAB78304A2E4942F8240018465B1855
:105D800052F8201000221A7106F0C0F84DE04920A8
:105D900002F07AFB294B587247E04A2002F074FB6C
:105DA000264B987241E00020142100E0042106F007
:105DB0008BF83AE04B200122214902F041FBA37805
:105DC0001E4A184602EB4313D97AC1F10801C9B241
:105DD00004F0E8FB29E01A21E9E71821E7E7582059
:105DE000184913E0482002F04FFB144B18721CE0D6
:105DF000402012490AE04420134907E05F2013497C
:105E000008E04E20124909E012495420042206E01D
:105E100011495E20012202E010495C20022202F0BA
:105E20000FFB02E003220E4B1A7038BD8C060020D7
:105E300070020020140B002010070020B80B002077
:105E4000C30B0020D00B0020BC0B0020D70B002080
:105E5000C60B0020CC0B0020D60B0020D40B00205A
:105E60000407002010B51E4A5378142B34D89278BA
:105E7000AAB91C4A1C4952F823201C4B4A601B78C3
:105E8000002B2CD01A491B4B0A601AB91A6842F031
:105E9000080202E01A6822F008021A601FE0FF2AD6
:105EA00018D163B94FF4C364134920460919042279
:105EB000043402F0C5FAB4F5CD6FF5D10FE003F567
:105EC000C2700849013001EB83018000042202F016
:105ED000B7FA04E0042200E00322034B1A7010BD5D
:105EE0008C0600209806002004070020FE060020F3
:105EF000EC060020940600208400002037B5134CE7
:105F0000657815B1012D1DD112E0042240F2FB701D
:105F100001A902F095FAE378626843EA0222019B44
:105F20009A420B4B02D101225A600EE05D600CE0F8
:105F3000A3782A2B06D1E11C40F2FB70042202F068
:105F4000BBFA02E0024B03221A703EBD8C06002011
:105F500004070020364900230B603649364A0B609F
:105F6000364910B50B6093749360D3601374537407
:105F7000334A4FF0FF3142F82310324A0024D45400
:105F800001332F2BF4D10731204605F045FD2E4B70
:105F90000C211860204605F03FFD2C4BD97A2C4B84
:105FA000C1F108011860C9B2204604F0FBFA294B80
:105FB0000022E2500434B4F5806FF8D1264B9B7E6A
:105FC0005BB104F5067425492046091904220434FE
:105FD00002F036FAB4F5CD6FF5D11F4BDB7E5BB91D
:105FE0004FF4A7641E49204609190422043402F024
:105FF00027FAB4F5C36FF5D1174B1B79012B03D0EA
:10600000112B01D0212B01D1012200E000220A4BEB
:1060100083F8D020104B5B7D23B1FEF7D9FA08B18D
:10602000012200E00022044B83F8D12010BD00BF04
:10603000EC0600200C0700207002002094060020CF
:1060400084020020300C0020140B0020B80B00202C
:106050001007002014070020080000208400002002
:10606000DC01002008B50B4B5A7892B9997881B9B8
:106070005A68DB7843EA022240F2D2439A4208D1BE
:1060800040F2FF7002F096FA02F058FB0120FEF792
:1060900001FD08BD8C06002010B59B4B9A78022AA2
:1060A00000F05581032A00F05B81002A40F0EB816B
:1060B0005A784D2A00F0B78023D8452A70D00ED8E0
:1060C000422A56D005D8402A45D0412A40F0D981ED
:1060D00046E0432A53D0442A40F0D38156E0482A70
:1060E0007CD005D8462A61D0472A40F0CA816AE0B0
:1060F0004B2A00F0858000F28F80492A40F0C18150
:1061000072E0542A00F0DE8011D8512A00F0AB80F2
:1061100006D84F2A00F08D80502A40F0B2819BE0D3
:10612000522A00F0B280532A40F0AB81B7E0832AB4
:1061300000F0F08006D8552A00F0D180572A40F0B0
:10614000A081D9E0852A00F0F580C0F0EB80FF2A1D
:1061500040F09781F7E06C4B40F2FF70D97805E092
:10616000694B6A4ADB7800201946137002F022FA64
:106170008CE1DB78654A194601205370F6E7624BE3
:10618000624ADB78042019461371EFE75E4B5F49E2
:106190005A68DB781C2043EA022341F81C3F0EE0DA
:1061A000DB785A4A194605205371DFE7564B5749A9
:1061B0005A68DB780C2043EA022341F80C3F0422A2
:1061C00002F07AF962E1504B504C5A68DB78214674
:1061D00043EA022341F8083F08206AE0DB784B4994
:1061E000262001F8263F78E0474A484BD27812B182
:1061F000474901224A60DA75444B1720D97DB5E73B
:10620000414B424CDB7803201946E37002F0D2F98F
:10621000E07802F0A7FB39E13B4B3C4ADB780220F7
:1062200019469370A2E7DB78384A19461520537552
:106230009CE7354B354CDB7819201946637602F024
:10624000B9F9607E10F0010002D00020012100E0C9
:10625000014605F015FD19E12B4B2C4ADB78162081
:106260001946937582E7294A127D12F0010F05D075
:10627000DB7813F0010F01D102F060FA224B234AC0
:10628000DB7814201946137570E71F4B1F495A68B5
:10629000DB78202043EA022341F8203F8FE71A4BA6
:1062A0001A4C5A68DB78214643EA022341F8103F32
:1062B0001020042202F000F922696079A16802F03E
:1062C000B3FDE3E05A68DB7843EA0222012A00F2D8
:1062D000DA800E491A2001F81A3F012270E70A4BB2
:1062E0005A68DB7843EA0222012A00F2CC8007498F
:1062F0001B2001F81B3FF0E7034B0449DB78272004
:1063000001F8273FE9E700BF8C06002008000020C5
:10631000040700205A68DB7843EA02225C4BC3F88A
:10632000D420B3E05B4B5A68DB7843EA02225A4B35
:106330001A60ABE0574B5A68DB7843EA0222544BB1
:10634000C3F8D820A2E0534BDA78544B9DE058684C
:10635000D9785A78524B41EA002143F8221095E04F
:106360005A78272A59D00ED8022A33D004D8CAB175
:10637000012A40F0868021E01B2A3ED01C2A44D00E
:10638000092A7ED132E02B2A5FD005D8292A50D0A5
:10639000D978444A54D847E02D2A64D05CD32E2AB9
:1063A0006FD167E05A68DB7843EA02223D4B1A60FE
:1063B00003F020F8364BC3F8DC0067E05A68DB785E
:1063C00043EA0222374B5A6003F014F8304BC3F80B
:1063D000E0005BE05A68DB7843EA0222314B9A60C6
:1063E00003F008F82A4BC3F8E4004FE05A68DB7862
:1063F00043EA02222B4BDA6048E05968DB78002040
:1064000043EA012105F036FD40E05968DB780020C1
:1064100043EA012105F002FD38E05A68DB7843EADF
:106420000222204B1A6131E05B6841EA032151618D
:106430002CE05A68DB7843EA02221A4B9A6125E085
:106440005B6841EA0321D16120E05A68DB7843EAC6
:106450000222144B1A6219E05A68DB7843EA0222DE
:10646000104B5A6212E05A68DB7843EA02220D4B65
:106470009A620BE05A68DB7843EA0222094BDA623F
:1064800004E0032200E00422074B1A7010BD00BF95
:10649000700200208C06002000070020FD0600206E
:1064A00014070020E00B00200407002008B5824BF1
:1064B0009A78022A00F0B980032A00F0BB80002AF3
:1064C00040F01E815B78502B6ED022D8462B54D0E2
:1064D0000ED8422B47D005D8402B3DD0412B40F061
:1064E0000D813EE0442B43D0744B754A43D83DE0C8
:1064F0004B2B4DD006D8482B43D040D3492B40F0EE
:10650000FD8042E04D2B49D045D34F2B40F0F68023
:1065100047E0812B5FD010D8542B4ED005D8522B9A
:1065200047D0664B664A46D841E0572B4BD0802B6C
:106530004DD0552B40F0E28042E0852B5DD004D851
:10654000832B53D05D4B55D84DE0FE2B64D066D8DD
:10655000F02B40F0D3805FE040F2FF7001F094FF39
:106560009CE0574B59E0564B5A78C4E01279C3E08F
:10657000534BDA69BFE05279BEE0514B85E0504B96
:1065800080E04F4B93F82620B5E04D4BDA7D48E094
:106590004B4BDA78AFE04A4B9A78ACE0484B5A7DE7
:1065A000A9E0474B5A7EA6E0454B9A7DA3E0127DB9
:1065B000A2E0434B95E012699EE0414B9A7E9AE03F
:1065C0003F4BDA7E97E03E4B93F8272093E03D4B1C
:1065D00093F8D1208FE03B4B93F8D120042A14BFCD
:1065E0000022012287E0374A926885E0354BD3F8D4
:1065F000D42080E0344A12687EE0324A334BD2F82D
:10660000D8104B4303F5405339332C4923F0004055
:106610004860C2F8D83076E02D4B1A786BE02D4BED
:106620001A78003A18BF012265E05A782A4B53F8CD
:10663000222060E05B78272B33D00DD8022B20D0AE
:1066400003D8C3B1012B59D118E01B2B1FD01C2B31
:1066500021D0092B52D117E02B2B41D005D8292B63
:1066600024D0164B1D4A24D81EE02D2B3ED03AD301
:106670002E2B43D13DE0194B1A683CE0174B5A686A
:1066800039E0164B9A6836E0144BDA6833E00020A4
:1066900005F03EFA02E0002005F026FA074B5860AC
:1066A00031E00E4B1A6926E0526925E00B4B9A69DE
:1066B00021E0D26920E000BF8C0600200407002002
:1066C0000800002070020020000700206D4EC64127
:1066D000140C0020FD06002014070020E00B002011
:1066E000124B1A6A07E0114B5A6A04E00F4B9A6A80
:1066F00001E00E4BDA6A0E4B5A6004E0032200E020
:1067000004220B4B1A700B4B1B786BB1084B0A49D8
:106710005A680A4B0A601AB91A6842F0080202E085
:106720001A6822F008021A6008BD00BFE00B0020C2
:1067300004070020FE060020EC060020940600203E
:1067400010B5154CA07818BB6378012B16D003D375
:10675000022B124C19D114E004F00CFDA17839B1D0
:106760000F4A937FBBB102EB4112927F9A4212D142
:106770000C4B01221A71013A0B4B0BE004F002FDA5
:1067800009E004F007FD606005E00323237002E0E8
:10679000024B04221A7010BD8C0600200407002052
:1067A000B80B002070020020340B002037B5504B8E
:1067B0001A7CA2B94F494868CA7842EA0022B2F16D
:1067C000FF3F04BF4C4A12680A214A43C3F8E8203D
:1067D00002F010FE464B01221A74C3F8EC00454B40
:1067E0005B78042B00F28280DFE803F003353F4F33
:1067F000130002F0FFFD3E4BD3F8EC10D3F8E82075
:10680000411A0029B8BF494291426CD900221A743A
:106810006CE0384B364C987804F0BCFC30B9374A01
:106820002074136823F0100313605FE0D4F8E8309D
:10683000002B57D002F0DEFDD4F8EC20D4F8E8307D
:10684000821A002AB8BF52429A424BD92B4B0021E0
:106850001A68217442E0002004F0F4FF254B244C18
:106860009D786D0050FA05F51CE000207C2101AAFE
:1068700005F024F91F4B02229D789DF806306D002B
:1068800012FA05F51A4C1D400EE001AA00207C21E9
:1068900005F014F9174A9DF806309578144C6D00F0
:1068A00053FA05F515F0010506D0144B00211A68BE
:1068B000217422F0100213E0D4F8E83093B102F012
:1068C00099FDD4F8EC20D4F8E830821A002AB8BF39
:1068D00052429A4206D9094B25741A6842F01002B6
:1068E0001A6003E0024B9A68013A9A603EBD00BF0D
:1068F000700200208C060020EC0600209406002088
:1069000008B5184B9A7812B1022A26D106E05868C9
:10691000DB7843EA0020FEF79DF821E0587807284D
:106920000AD85A68DB7853EA022202D1FDF760FDEB
:1069300016E0FDF76DFD13E0FF280CD15868DB78F9
:1069400043EA0020B0F1FF3F0ABF074BC0B21878FE
:10695000FDF76EFD04E0032200E00422034B1A70F1
:1069600008BD00BF8C060020EC06002004070020B4
:1069700010B5224B9A78012A23D003D3022A204C47
:1069800028D122E05878082802D8FDF74FFE15E0FC
:106990000A2801D100220AE00B2802D1FDF79EFE51
:1069A0000CE00C2806D1174B9A68C2F3C032144B86
:1069B0005A6011E0FF280FD1FDF75EFE104B5860C2
:1069C0000AE0587802F034FDF8E75878FDF744FD06
:1069D000606001E0042323700B4B1B786BB1084B04
:1069E0000A495A680A4B0A601AB91A6842F0080242
:1069F00002E01A6822F008021A6010BD8C0600201E
:106A00000407002000080140FE060020EC060020DC
:106A10009406002010B5204B5A78812A3AD19A78F2
:106A2000922A37D19A79A32A34D15A79B42A31D10A
:106A30001A79C52A2ED1DB78D62B2BD1174B4FF4E0
:106A400000421A6103F074F802F0D4FC044602F02C
:106A5000D1FC001B0028B8BF4042B0F57A7FF6DBBE
:106A6000FDF71AFD06F078FF002007F0A5FC0021D5
:106A70000B4806F027FB0A4806F084FA094805F09F
:106A80003FFF06F06FFB4FF0804008F019FA00203E
:106A9000FEF700F810BD00BF8C060020001001407A
:106AA00008000240002401402DE9F3479D4A9E4D15
:106AB000D0785168137840EA01204FF0640C222B03
:106AC00085F800C06B70686000F0798554D80F2B92
:106AD00000F0358324D8072B00F00A8210D8032B4E
:106AE00000F0F88006D8012B00F0A680022B40F0C1
:106AF000A787C8E0052B00F0F38100F2F58101E1E2
:106B00000B2B00F0DF8205D8092B00F0D38200F2B6
:106B1000D582CBE20D2B00F00A8300F20C83EAE26F
:106B2000192B00F0B38412D8152B00F0BF8306D8C0
:106B3000132B00F00883142B40F082876BE3172B94
:106B400000F08484794B00F2948400F078BC1E2B12
:106B500000F0C68409D81B2B00F0BA84C0F0A684CC
:106B60001C2B40F06D8700F0B6BC202B00F0BE84DB
:106B700000F2BF8400F0B7BC812B00F0CE852ED888
:106B8000412B00F0B08515D8252B00F05E8507D885
:106B9000232B00F02085242B40F0528700F027BDE6
:106BA000272B00F08985C0F05B85402B40F048879B
:106BB00000F096BD452B00F0A28506D8432B00F0CF
:106BC000988500F2998500F091BD472B00F09D85D6
:106BD000C0F09885802B40F0338700F099BD882B5A
:106BE00000F03D8612D8842B00F0E28507D8822B76
:106BF00000F0AB85832B40F0238700F0ABBD862BE4
:106C000000F0F08500F24A8600F0E7BD8C2B00F022
:106C10008F8606D88A2B00F0728600F2848600F0F8
:106C20006BBEF22B00F0DC86FF2B00F0FB868D2B79
:106C300040F0068700F07FBE9378FBB93B4B4FF0E6
:106C4000010C83F804C03A4B00241C70394B2146D8
:106C50001C702046022204F0B9FE2046062140F2B4
:106C6000FF7205F01FF82F4B20465A68DB78082189
:106C700043EA022205F016F800F0E5BE2A4B042292
:106C80001A7000F0E0BE274DAC78F4B9274B4FF0F6
:106C9000010C83F804C0264B21461C70254B20466E
:106CA0001C70022204F092FE2046062140F2FF7280
:106CB00004F0F8FF6A68EB78204643EA0222524269
:106CC000082104F0EFFF00F0BEBE174B04221A703B
:106CD00000F0B9BE94788CB9154B20461C70154B4A
:106CE0001C7004F04FFA20462146022204F06EFE8A
:106CF0002046082104F0EAFF00F0A5BE04232B7013
:106D000000F0A1BE074B9A78002A40F0E4805B783F
:106D1000032B00F2DB80DFE813F00F004900940042
:106D2000BA0000BF8C06002004070020700200207B
:106D3000AC0B0020340B0020A54D0020FEF740F9DD
:106D4000A44EAB7800246868EA78F454A24E590146
:106D500042EA0022F45401F0E001204604F00EFF64
:106D6000A9782246204604F031FEA9789B4A02EB1E
:106D700041139B7F002B00F06686002900F063869C
:106D8000927F9A4240F05F862046FEF719F96A68C2
:106D9000EB78204643EA0222214604F0EFFE20462B
:106DA0002146224604F012FE00F04DBE884D002020
:106DB000FEF706F9AB78874A00245901D454864A75
:106DC00041F00201D45401F0E201204604F024FE17
:106DD000EB786E68A97843EA06268619490101F026
:106DE000E0013246204604F0C9FE2046A97822463A
:106DF00004F0ECFDA878794A794902EB40139B7FB7
:106E00004E60002B00F01F86002800F01C86927F49
:106E10009A4240F01886FEF7D3F80221204604F08B
:106E2000FBFD6A68EB78214643EA0222821820467D
:106E300004F0A4FE20462146224604F0C7FD00F0DF
:106E400002BE634CE378626843EA0223142B19DC28
:106E5000644A002052F82360FEF7B2F8A378324665
:106E60005C4E0025F5545C4E5901284601F0E001C6
:106E7000F55404F083FE2846A1782A4604F0A6FDC6
:106E800000F0E1BD564B04221A7000F0DCBD504CFE
:106E90000020E3786268002543EA0222514B53F850
:106EA0002260FEF78DF8A37832464A4E5901F55418
:106EB000494E284601F0E001F55404F05FFE2846F3
:106EC000A1782A4604F082FD00F0BDBD444B0322A8
:106ED0001A7000F0B8BD424B04221A7000F0B3BD26
:106EE000FEF790F800F0AFBDFEF7C4FB00F0ABBDBD
:106EF000907818B104232B7000F0A5BD53789A2B1D
:106F000021D8992B80F08280822B6DD00BD8062B54
:106F10004AD003D8042B3BD0052B0AE0072B4AD0DC
:106F20000C3B012B0CE08C2B63D005D8832B2FD08E
:106F3000862B40F0B68031E08D2B61D0933B022B45
:106F400000F2AF803EE0C72B2ED00ED8C12B69D007
:106F500005D8B52B5FD0C02B40F0A3802BE0C22B0F
:106F600067D0C32B40F09D806AE0D22B7DD005D83E
:106F7000C82B6CD0CC2B40F094806FE0D52B00F068
:106F80008280D62B00F08680D42B40F08A8073E07C
:106F90000020062104F0D0FD00F055BD00200C219A
:106FA00004F0CAFD00F04FBD0C4B4920597A01F0A6
:106FB00001FB00F048BD094B4A20997A01F0FAFA2A
:106FC00000F041BD0020142104F0B6FD00F03BBDEF
:106FD0008C060020340B0020AC0B0020B80B0020E6
:106FE0000407002098060020042104F0A5FD00F00D
:106FF0002ABD4B209E49012201F05EFA00F023BD1C
:1070000000201A2104F098FD00F01DBD182104F0A5
:1070100093FD00F018BD58209649042201F04CFA67
:1070200000F011BD944B4820197A01F0C3FA00F02A
:107030000ABD40209049042201F03EFA00F003BD51
:1070400044208E49042201F037FA00F0FCBC5F2096
:107050008B49012201F030FA00F0F5BC4E2089493D
:10706000022201F029FA00F0EEBC502086490422E9
:1070700001F022FA00F0E7BC54208449042201F018
:107080001BFA00F0E0BC5E208149012201F014FAF5
:1070900000F0D9BC5C207F49022201F00DFA00F01B
:1070A000D2BC7D4B03221A7000F0CDBCFEF7F2FD7E
:1070B00000F0C9BCFEF7F0FF00F0C5BCFFF7F6F921
:1070C00000F0C1BC9378022B11D15378372B0AD82A
:1070D000724903F5A77001EB83018000042201F0DF
:1070E000EBF900F0B0BC03232B7000F0ACBC042320
:1070F0002B7000F0A8BC6A4B9A78022A12D15B78F8
:10710000372B0AD8654903F5A77001EB830180008E
:10711000023201F095F900F096BC5F4B03221A7021
:1071200000F091BC5C4B04221A7000F08CBCFFF79D
:1071300007FB00F088BCFFF7E3FB00F084BCFFF71F
:1071400017FC00F080BC5278564B092A53D8DFE870
:1071500002F0050D151D26313941494C504A196878
:107160005068D27842EA0022521843E04C4A19682B
:107170005068D27842EA00228A1A3BE0484A1968ED
:107180005068D27842EA00224A4333E0444A196800
:107190005068D27842EA002291FBF2F22AE040489D
:1071A00019684468C27842EA042291FBF2F002FBBB
:1071B00010121FE03A4A19685068D27842EA002259
:1071C0000A4017E0364A19685068D27842EA00222D
:1071D0000A430FE0324A19685068D27842EA002226
:1071E0004A4007E01A68D24304E02D4A5168D27839
:1071F00042EA01221A602B4A2B4B12682AB91A68FC
:1072000042F008021A6000F01EBC1A6822F0080260
:107210001A6000F018BC224B224A5968DB781268C9
:1072200043EA01239A4206DD1F4B1A6842F004022A
:1072300022F003020CE01C4B05D11A6822F0060272
:1072400042F0010204E01A6822F0070242F0020252
:107250001A60144A144B126822B91A6842F00802E4
:107260001A60F0E31A6822F008021A60EBE300BF2C
:10727000C30B0020D00B0020B80B0020BC0B00205B
:10728000D70B0020C60B0020C80B0020CC0B002021
:10729000D60B0020D40B0020040700201407002088
:1072A0008C060020EC0600209406002053780C2B5E
:1072B00000F2C983DFE813F00D001B00290037003E
:1072C0004500530061006F007D008B009900A7000E
:1072D000B500944B1B6813F0080F00F0B483924B79
:1072E0005A68DB7843EA0222904B9A60ABE38D4BFD
:1072F0001B6813F0080F40F0A6838B4B5A68DB78AD
:1073000043EA0222894B9A609DE3864B1B6813F087
:10731000010F00F09883844B5A68DB7843EA02221D
:10732000824B9A608FE37F4B1B6813F0010F40F094
:107330008A837D4B5A68DB7843EA02227B4B9A6052
:1073400081E3784B1B6813F0040F00F07C83764BCD
:107350005A68DB7843EA0222744B9A6073E3714BFC
:107360001B6813F0050F00F06E836F4B5A68DB78D3
:1073700043EA02226D4B9A6065E36A4B1B6813F087
:10738000020F00F06083684B5A68DB7843EA022200
:10739000664B9A6057E3634B1B6813F0030F00F0D2
:1073A0005283614B5A68DB7843EA02225F4B9A6052
:1073B00049E35C4B1B6813F0100F00F044835A4BF9
:1073C0005A68DB7843EA0222584B9A603BE3554BFC
:1073D0001B6813F0200F00F03683534B5A68DB789C
:1073E00043EA0222514B9A602DE34E4B1B6813F087
:1073F000400F00F028834C4B5A68DB7843EA0222A6
:107400004A4B9A601FE3474B1B6813F0800F00F054
:107410001A83454B5A68DB7843EA0222434B9A6051
:1074200011E3404B1B6813F4807F00F00C833E4B4C
:107430005A68DB7843EA02223C4B9A6003E33A4AFB
:107440005168D27842EA01229A60FCE2374BDA684E
:10745000072A00F2F88234499C684868C97841EAF2
:107460000020511C03EB8202C2F8F0409860D96002
:10747000E9E2DA682D4B002A00F0E582013A03EBDD
:107480008201D1F8F010DA609960DCE253782E2B9B
:1074900003D8274A0121D154D5E2FF2B03D1234B36
:1074A00001225A74CFE203232B70CCE21E4B5B788F
:1074B0002E2B03D81E4A0021D154C4E2FF2B03D146
:1074C0001A4B00225A74BEE21A4B03221A70BAE217
:1074D000FFF76CF9B7E2154B002283F8D120B2E236
:1074E000FEF74EFBAFE2FEF7BDFCACE2FEF78AFB17
:1074F000A9E20D4A104B52780A2A52D8DFE802F06E
:10750000060B20252B33393F45494C000B491A689F
:1075100009688A1803E0094A196812688A1A1A6009
:107520003FE000BF940600208C060020700200207F
:10753000300C002004070020EC0600200C0700207F
:10754000934A196812684A43E9E7914A1968126830
:1075500091FBF2F2E3E78E4A1968126891FBF2F0B0
:1075600002FB1012DBE78A491A68096801EA020285
:10757000D5E787491A68096841EA0202CFE78449DA
:107580001A68096881EA0202C9E7814B1A68D24386
:10759000C5E71A687E4BC2E77D4A1868116810601B
:1075A00019607C4A7C4B126822B91A6842F00802C2
:1075B0001A6048E21A6822F008021A6043E2754B2A
:1075C00001F07F4118681B7841EA10215160D370A7
:1075D000FDF718FD37E26F4B01F07F4118681B780B
:1075E00041EA10215160D370FEF756FD2BE26B4B40
:1075F0005B78052B00F22782DFE803F003090F1503
:107600001B21654B1A6802F00F021A601BE2624BE5
:107610001A6822F010021A6015E25F4B1A6822F015
:1076200020021A600FE25C4B1A6822F040021A60D6
:1076300009E2594B1A6822F080021A6003E2564BA5
:107640001A6822F480721A60FDE153782E2B04D858
:10765000534A02EB83035861F5E103232B70F2E1F7
:107660004F4BDFF830C1D3F810914E4993F82C21DD
:10767000D3F814A1CCF80090DFF814C1D3F8187136
:10768000D3F81C81D3F82061D3F82451D3F82841D2
:10769000CCF800A0885CDFF800C19F60CCF80080C7
:1076A0001E74C3F8EC50C3F8E84008B101238B54B2
:1076B0003B4B00229A74C6E193786BB9374B5B78E9
:1076C000142B05D8334A1168374A42F82310BAE11F
:1076D000364B03221A70B6E1344B04221A70B2E121
:1076E00002F070FAAFE102F06FFAACE102F06EFA6C
:1076F000A9E102F06DFAA6E102F06CFAA3E102F052
:107700006BFAA0E102F06AFA9DE102F069FA9AE1EF
:10771000234B002283F8D12095E1537813B1012B3C
:1077200010D104E01E4B012283F8D1208BE1B0F58B
:10773000006F04D21A4A906082F8D13083E10423AA
:107740002B7080E103232B707DE1154B022283F81F
:10775000D12078E1124B002199745974104A4FF0EE
:10776000FF3402F1140040F821400E480023435436
:1077700001312F29F2D1084913740B60054982F8B1
:10778000D1300B60024993600B60D3605BE100BFB6
:107790000C070020EC060020940600208C06002038
:1077A00070020020300C0020980600200407002002
:1077B0008D4B1B7D13F0020F0CD1B0F5006F06D27C
:1077C0008A4B0422C3F8300183F8D1203BE1042323
:1077D0002B7038E108232B7035E1844B002283F8AD
:1077E000D12030E1804B01219A78814BB0F5006FB8
:1077F0001970804B1A7028D27B4B1C7D0C4024D111
:10780000694600F0DFFF7B4B9DF800709DF801603A
:107810009DF802509DF806C09DF805009DF80410E3
:107820009DF803201C725F709E70DD7083F804C0A9
:1078300058719971DA7101236E4A985C117A01339B
:107840004118082B1172F7D1FDE00123694A00218C
:1078500099540133082BF9D113781372F3E053785C
:107860008BB9614A01209178634A1468604A1070AC
:10787000604A11700133E21812F8011C5D4A082BAE
:107880009954F7D1DFE0012B40F0DD8018222A71F6
:107890000422EA717032AA716B71D4E0574B5B78A5
:1078A000032B00F2D080DFE803F002101D224F4AC4
:1078B000534BD2F8301192F8D1C0107C0A0A1971DA
:1078C00083F807C098715A71BDE0484A4C4B9168E3
:1078D00092F8D1C0107C0A0A197183F807C0987118
:1078E0005A71B0E0474B1A68454B5A60ABE0464BC3
:1078F0001A68434B5A60A6E0FEF7B4FBA3E0527847
:10790000424B02B101221A703C4B414AD878374BA6
:10791000107093F834113F4A002311703E4A1370DF
:107920003E4A13708FE0314B012283F835218AE003
:10793000FEF7E4FA87E0314B5B78032B4CD8DFE8A5
:1079400003F00C023C472D4B28495A68DB78D1F8EC
:10795000381143EA022C00232BE0244BD3F83821C2
:10796000092A0CD82549501C4C68C97803EB8202BF
:1079700041EA0421C2F83C11C3F8380163E0204B0E
:1079800009221A705FE052F82340581C64450FD159
:1079900002EB8002013904E052F8040C013342F892
:1079A000080C04328B42F7D3104BC3F838114AE06D
:1079B00003468B421A4AE6D345E00C4A0023C2F83C
:1079C0003831174A0021D1500433282BF9D13AE03D
:1079D0000B4B0A225A6036E0094B03221A7032E040
:1079E000FFF718F82FE000BF080000207002002009
:1079F000F0060020F4060020000000208C06002085
:107A000004070020EC0600200C070020200B0020BB
:107A10004C0B00201E0C0020640C00203C0B0020AE
:107A2000AC030020094B5A68DB7843EA022240F29B
:107A3000D2439A4207D1064B012283F8642102E027
:107A4000044B02221A70BDE8FC8700BF8C060020A0
:107A5000700200200407002073B5204B02464078D6
:107A60001F4D1870907800265870D078EC469870AA
:107A700010790C4698715079587192F806E095E8A3
:107A8000030083F804E0D2798CE80300DA70154B28
:107A90001E70FFF709F8144B1B7873B963702370DD
:107AA0002B78A3706B78E370EB792371AB796371FA
:107AB0006B79A3712B79E37108E0012B06D10B4B95
:107AC0009B195B78A3550136082EF8D1044B6A4602
:107AD00092E8030083E803007CBD00BF8C06002011
:107AE00004070020FE060020F0060020F406002017
:107AF000F7B5114D114C6F684FF0000C07F07F4740
:107B000047EA13276F600E4F6E4687F800C0287053
:107B10006970AA7094E80300EB7086E80300FEF732
:107B2000C3FF96E803006368227884E803000549F0
:107B300018460A70FEBD00BF8C0600200407002016
:107B4000FE060020700200202DE9F04F984B9BB0FC
:107B50001B781BB9974B93F865316BB1964B1B782B
:107B6000062B09D00A2B07D00F2B05D01F2B03D0D3
:107B7000904B002283F834218E4A92F83431591EFA
:107B8000C9B2012946D892F866018C498C4ACC6862
:107B90001278012B0CBF4FF0070C4FF0080C00239C
:107BA0000E948DF834C08DF835008DF83630CAB992
:107BB000844B8E681D7819795C7893F807C09879A2
:107BC0005B798DF83C608DF83D508DF83E408DF826
:107BD0003FC08DF840008DF841308DF842108DF88F
:107BE00043200AE0012A08D1774A0133995C1AA898
:107BF000C218082B02F82D1CF6D1744B1B78002BF1
:107C000040F0C2800DA801F02DF8002840F0BC80A3
:107C100000F00FBC032B25D192F8D040002C40F08F
:107C20008680674B1B7893B9644D664CA8786E7854
:107C3000227863788619B618E279F618A379B6180F
:107C40006279F6182379B618F618F6B219E0012B06
:107C500040F09A805C4BE05C013400F09FFE092C00
:107C6000F8D191E0042B27D1544D564CAB786E7867
:107C700018469E1901360023012222706360F6B275
:107C8000637000F08BFE687800F088FE207800F0CA
:107C900085FE607800F082FEE07900F07FFEA0793A
:107CA00000F07CFE607900F079FE207900F076FE2D
:107CB000304600F073FE67E0072B3CD192F8D030DD
:107CC000002B34D13E4A127822BB3C4A3D4B5578BA
:107CD00096781C7893F801C0AF19D879E71999798B
:107CE00067445A79C7191B79CF19D719DF198DF84D
:107CF00058708DF850608DF851508DF852408DF8C5
:107D000053C08DF854008DF855108DF856208DF81D
:107D1000573008E0012A06D12B4A995C14AAD154A5
:107D20000133092BF8D1294B1B786BB328E0254888
:107D300004F006FA28E0082B26D1204B00225978BF
:107D40009878224B45181C781E4B4FF0010C0135DA
:107D50005A608DF852C08DF8532016468DF8542085
:107D60008DF855208DF856208DF857208DF85850F5
:107D70005A7083F800C08DF850008DF851101CB176
:107D800014A8092101F0AAFD114B1B78002B00F06B
:107D90009980104A0D4B12780F4C013A062A00F2D6
:107DA0008C80DFE802F01B1B418A8A8A650000BFD5
:107DB000FD060020700200208C0600200800002034
:107DC000F006002004070020F4060020180B002015
:107DD000640C00201E0C00203C0B0020AB4A94F8E1
:107DE00000C0D068926819788DF82C206FF07F025F
:107DF0008DF82D200A3200238DF82E207D328DF84B
:107E000032C08DF824208DF826300A908DF82F305E
:107E10008DF830308DF831308DF8253000294CD177
:107E200009A800F01FFF48E0984D2278AB786E78E3
:107E300018469E190A36B61800F0B0FD687800F0B2
:107E4000ADFD802000F0AAFD8A2000F0A7FD0020F3
:107E500000F0A4FD002000F0A1FD002000F09EFD38
:107E6000F6B2207800F09AFD304600F097FD24E04D
:107E700086482278417880786FF07F0500EB010C0E
:107E80001C780CF10A0C002394448DF846500A35F6
:107E90008DF847508DF84A308DF84CC08DF844006D
:107EA0008DF845108DF848308DF849308DF84B200D
:107EB0001CB111A8092101F011FD754A00231370AE
:107EC000744A1370744B754893F864110022027061
:107ED00083F8652183F8342111B10120FCF7DAFD24
:107EE0006D4B93F8352152B193F8D0200021D2F197
:107EF000010238BF002283F8351183F8D020684B87
:107F00001B78002B46D10DA800F08AFE002841D036
:107F10009DF83430062B3DD9624B5C4A9DF83C708D
:107F20009DF83D609DF83E509DF83F409DF840E033
:107F30009DF841C09DF84280116983F803801F704D
:107F40005E709D709C7183F805E083F804C00E9B01
:107F5000514A9DF835008B4282F8660102D1012317
:107F600082F8653101F046FA9DF834304FF0000296
:107F7000072B4D4B484C18604C4B1A7001D1012314
:107F800000E0022384F83431434B93F8D1305A1E79
:107F9000D2B2E8E0404C94F8D050002D40F08C80F4
:107FA0000DF1670000F0C8FC002800F0858000F0AB
:107FB000DFFC08B184F86751374B9DF8670093F8F0
:107FC00067114A1CD2B2C918092A81F8680183F8DE
:107FD000672140F0F1802D4993F8682148784FF0EF
:107FE000000C904283F867C107D091F82730002B2E
:107FF00000F0E2809A4240F0DF80244B93F8273073
:10800000934203D1244B012283F8652100231A46B1
:10801000214C04F5B471C95C01335218082BD2B25B
:10802000F6D194F8703193422DD11E4B94F86D1116
:1080300094F86E2194F86F5194F8696194F86AE1AC
:1080400094F86BC194F86C01DD7059711A711E704F
:1080500083F801E083F802C0987101F0CBF9144D68
:1080600094F8D1302860591E12480022C9B202701B
:108070000320012984F8340184F8672177D9052B7E
:1080800075D0013291E0042373E000BF08000020A6
:10809000640C00203C0B002070020020F006002041
:1080A000180B00208C060020100C0020190B00205B
:1080B000180C00201D0C00209B4C94F8D03083B18C
:1080C0009A4804F083F860B101F094F9984994F863
:1080D000D130086097495A1E00200870D2B203219F
:1080E0003FE0914B93F8D040002C45D1924B1B7848
:1080F000002B41D017A801F0DBFB00283CD0234621
:10810000224617A9C95C01335218082BD2B2F8D104
:108110009DF86410844C91422BD1844B9DF86110E2
:108120009DF862209DF85D609DF85EE09DF85FC05F
:108130009DF860009DF8635059711A711E70DD70D2
:1081400083F801E083F802C0987101F053F978498F
:1081500094F8D130086077495A1E00200870D2B2D6
:10816000072184F83411012A01D9052B1CD10022E2
:108170001BE084F834311FE06B4C94F8D130013BA4
:10818000DBB2012B18D8A368B3F5006F10D2FCF74F
:108190001FFA68B1A368654918460133A36000F06F
:1081A00011FB092384F834310122644B1A7003E077
:1081B0005D4B002283F8D1205B4C94F8D130042B26
:1081C00005D15A4E327812F0800F00F00581564BDF
:1081D00093F834313BB1042B05D0082B03D0062B88
:1081E00001D0FEF761FC504C94F83431092B40F07B
:1081F000CA8001F0FFF8D4F8DC30514AC31A002BD2
:108200001268B8BF5B4293420AD94E4B1A78012AD2
:1082100001D101321A7001F0EDF8434BC3F8DC00D4
:1082200001F0E8F8404BD3F8E020454B821A002AD1
:108230005B68B8BF52429A420AD9424B5A78012A27
:1082400001D101325A7001F0D5F8374BC3F8E00084
:1082500001F0D0F8344BD3F8E420394B821A002ACD
:108260009B68B8BF52429A420AD9364B9A78012A83
:1082700001D101329A7001F0BDF82B4BC3F8E40034
:10828000294A537C002B7ED0937C002B7BD19C46CB
:108290002D4BD2F8EC001B68D2F8E81007932B4B5B
:1082A00004901B68D2F810810693294BD2F8147100
:1082B0001B68D2F81841059392F82C31D2F81C6152
:1082C0000293107C9368D2F82051D2F824B1D2F8EE
:1082D0002821039101926246DFF86890194619F847
:1082E00002A0BAF1020F18D11A4951F82210B1F1C7
:1082F000FF3F0ED00546D0B202900398DDF810B0D3
:108300000190059E069FDDF81C804FF0010C0020B7
:1083100004E0002109F802101946234601322F2AF1
:108320001AD01C460B46D7E7700200208C060020AE
:10833000180C00201D0C0020180B0020FE06002049
:10834000E00B0020300C0020EC0600200C07002081
:108350009406002084020020374A9160C2F8183148
:108360000199029B82F812C0C2F81081C2F8147100
:10837000C2F81C611074C2F82051C2F824B1C2F8CE
:10838000281182F82C312C4B93F83421092A06D17C
:1083900093F8D110022902D1033183F8D110264B72
:1083A000D3F83811002944D0092A42D193F8D120BA
:1083B000012A3ED19868002308E054F82340013395
:1083C000A04203D1052382F8D13032E01A4A8B4211
:1083D00002F59E74F1D32CE094F834314BB3042BA6
:1083E00027D0082B25D0062B23D0F3787168D4F83A
:1083F0003001124D43EA0123B0F5006F6A706B60E3
:1084000012D2314600F00EF93146D4F8300100F0B6
:1084100031F930B1D4F830310133C4F8303165234B
:1084200000E007232B7004E007232B70002384F85F
:10843000D1301BB0BDE8F08F70020020040700208F
:1084400070B5044600200E46154603210246FCF78F
:108450003FFC0020C4F307210246FCF739FC002052
:10846000E1B20246FCF734FC002407E0944214BF5A
:1084700000220122FCF72CFC3055013400206A1E3A
:10848000AC420146F2D370BD10B504460020032172
:108490000246FCF71DFC0020C4F307210246FCF74E
:1084A00017FC0020E1B20246FCF712FC0020014656
:1084B0000122FCF70DFC10BD2DE9F04104460F46EA
:1084C0001646002006210122FCF702FC00200521AF
:1084D0000246FCF7FDFB002001220146FCF7F8FBF9
:1084E00010F0020FF2D0002002210246FCF7F0FB50
:1084F0000020C4F307210246FCF7EAFB0020E1B2AA
:108500000246FCF7E5FB002543E0013414F03F0888
:10851000795D01D1012204E0721E954214BF002250
:1085200001220020FCF7D4FBB8F1000F30D1731EFC
:108530009D422DD2002005210246FCF7C9FB0020F8
:1085400001220146FCF7C4FB10F00100F2D1062124
:108550000122FCF7BDFB002005210246FCF7B8FB19
:10856000002001220146FCF7B3FB10F0020FF2D00D
:10857000002002210246FCF7ABFB0020C4F30721D8
:108580000246FCF7A5FB0020E1B20246FCF7A0FB87
:108590000135B542B9D3002005210246FCF798FB0E
:1085A000002001220146FCF793FB10F0010FF2D1ED
:1085B000BDE8F08138B5012204460D4600200621B1
:1085C000FCF786FB002005210246FCF781FB00201A
:1085D00001220146FCF77CFB10F0020FF2D00020D4
:1085E00002210246FCF774FB0020C4F30721024677
:1085F000FCF76EFB0020E1B20246FCF769FB29465E
:1086000000200122FCF764FB002005210246FCF754
:108610005FFB002001220146FCF75AFB10F0010F1E
:10862000F2D138BD38B50725454305F500650C4640
:10863000284609780135FFF7BDFF284661780135E6
:10864000FFF7B8FF2846A1780135FFF7B3FF2846AA
:10865000E1780135FFF7AEFF284621790135FFF7B4
:10866000A9FF28466179FFF7A5FF681CA179FFF7EC
:10867000A1FF38BD2DE9F3470725454300200C46EF
:1086800002460321FCF724FB05F500650020C5F335
:1086900007210246FCF71CFB0020E9B20246FCF76A
:1086A00017FB002001460246FCF712FB8246002021
:1086B00001460246FCF70CFB8046002001460246BC
:1086C000FCF706FB0746002001460246FCF700FBCC
:1086D0008146002001460246FCF7FAFA06460020D1
:1086E00001460246FCF7F4FA054600200122014645
:1086F000FCF7EEFA237853451DD1637843451AD130
:10870000A378BB4217D1E37821798DF804608DF806
:1087100005508DF80600627943EA012343EA0243DB
:10872000A079019A43EA006049EA0229814514BF11
:108730000020012000E00020BDE8FC8738B54FF4A0
:108740000064002006210122FCF7C2FA0020052166
:108750000246FCF7BDFA002001220146FCF7B8FAF8
:1087600010F0020FF2D0002002210246FCF7B0FA0E
:108770000020C4F307210246FCF7AAFA0020E1B268
:108780000246FCF7A5FA002500203F2D14BF002269
:10879000012201460135FCF79BFA402DF4D100205F
:1087A00005210246FCF794FA002001220146FCF75D
:1087B0008FFA10F0010FF2D14034B4F5804FC0D1E0
:1087C00038BD00BF38B50725454300200C4602469A
:1087D0000321FCF77DFA05F500650020C5F30721AC
:1087E0000246FCF775FA0020E9B20246FCF770FA7F
:1087F000002001460246FCF76BFA2070002001467B
:108800000246FCF765FA6070002001460246FCF75C
:108810005FFAA070002001460246FCF759FAE070AA
:10882000002001460246FCF753FA20710020014661
:108830000246FCF74DFA6071002001460122FCF768
:1088400047FAA07138BD00BF37B5002005210246A8
:10885000FCF73EFA002001220146FCF739FA10F03D
:108860007104F2D100F0C6FD054605E0FFF70CFEED
:10887000422814BF0024012400F0BCFD431B002B40
:10888000B8BF5B42B3F5FA6F40F2FF7002DA002C1A
:10889000ECD000E01CB1234B1B78002B36D040F20B
:1088A000FF700021FFF786FEFFF748FF00201E49FA
:1088B0004022FFF701FE4FF480701C49B422FFF7FD
:1088C000FBFD40201A492022FFF7F6FD002301930B
:1088D0004FF4C36401AD2046042204342946FFF757
:1088E000EBFDB4F5FF6FF5D100230193A4F53074CF
:1088F0002046042204342946FFF7DEFDB4F5C36F99
:10890000F6D140F2FF704221FFF754FE00204022D2
:108910000549FFF795FD402006492022FFF790FD0D
:108920003EBD00BF540B0020080000204026010877
:1089300070260108B80B0020094B19685A6891424B
:1089400001D100200BE01A68D118097A01320170B8
:108950001A601A68202A01D100221A60012070478B
:10896000E4030020014B9862704700BFE40300203D
:10897000034B1A78104612B100221A70012070477A
:10898000700C002008B5FBF787FD034B00221A602E
:108990005A60FBF77FFD08BDE403002038B50B4BA0
:1089A0008446DC6A1A6B0134202C08BF00249442F0
:1089B0000AD0DD6A0648ED1885F834C040F2277108
:1089C0000122DC6206F014FB38BD00BFE403002086
:1089D0000044004038B50546002401E0FFF7DEFF03
:1089E0002B5D01341846002BF8D138BD2A4910B54B
:1089F0000B8813F0200F1CD0284BDB6813F0020FFC
:108A000001D08B8815E0264B5A6818680132202A5D
:108A100008BF0022824205D05C688888E118C0B295
:108A200008725A601F4B0A221A601D4B9A6A1E4B2D
:108A30001A601948038813F0800F1BD01A4B1A686C
:108A4000C2B9174BDC6A196B8C420FD01349022450
:108A50000C61196BCC1894F834C00131A0F804C033
:108A60001963196B202905D11A6303E040F22771BD
:108A700006F0BEFA0848038813F0400F0BD040F20E
:108A8000266106F0ADFB064B1A6BDB6A9A4202D1F7
:108A9000024B02225A6110BD004400400008014010
:108AA000E40300206C0C0020680C002030B5054663
:108AB00087B0564806F0E4FB4FF40030012105F082
:108AC0002DFA0420012105F01BFA0420002105F0F5
:108AD00033FA0820002104F09BFE06AC4FF004039B
:108AE00024F8083D03234A4821468DF812301533F7
:108AF0008DF8133004F0FCFD482345488DF8133001
:108B000021464FF00803ADF8103004F0F1FD68463F
:108B100006F038FA0B2D25D8DFE805F02406090CFD
:108B20000F1215181B1E20224FF461531CE04FF446
:108B3000964319E04FF4E14316E04FF4164313E077
:108B40004FF4614310E04FF496330DE04FF4E133FE
:108B50000AE04FF4613307E02E4B05E02E4B03E0B3
:108B60002E4B01E04FF416530093009B06A95B08BF
:108B700041F8183D2548694606F03AFB26230024B3
:108B8000012505A88DF8143007238DF815308DF8D0
:108B900016408DF8175004F01BFF1C4840F2FF31BF
:108BA00006F0FAFA28212246184806F021FA2A4649
:108BB000164840F2277106F01BFA2A46134840F285
:108BC000266106F015FA2A46104840F2255106F0B3
:108BD0000FFA22460D4840F2244106F009FA2246D7
:108BE0000A4840F6460106F003FA2246074840F6D6
:108BF0006A1106F0FDF960212246044806F0F8F9F2
:108C00002946024806F0E6F907B030BD00440040AE
:108C10000008014090D0030020A1070040420F004F
:108C200030B50C4B0C4C844622681B689A4201D12B
:108C300000200EE02368094A5D1C02EB03130FCBF2
:108C40008CE80F0025602368082B01D100232360E6
:108C5000012030BD000D0020740C0020800C00208D
:108C6000704700BFF0B5437887B00646426833B11D
:108C700004238DF80C3000230292019303E001924B
:108C800002938DF80C30B37803B102238DF80D30C8
:108C9000327800238DF80E20F21801A8117AC2183C
:108CA0000133082BD172F7D103F064FF042818D1E7
:108CB0000D4D0E4B2C681B680134082C08BF002496
:108CC0009C4201D100200DE096E80F002F68084E6D
:108CD00006EB071C8CE80F00012001462C6003F016
:108CE0003BFF012007B0F0BD780C00207C0C002079
:108CF000040D00207FB52B4B2B4A19681268914256
:108D000004D10120002103F027FF48E01968274A19
:108D100002EB0111487850B11B6802EB0312536853
:108D200004228DF80C2000220192029307E01B68B8
:108D3000029002EB031253688DF80C000193194B5B
:108D40001A681A4B03EB02139B781BB102238DF8B0
:108D50000D3001E08DF80D30124B00221968134BD5
:108D60000901CB5C8DF80E300E4B0DF1180C186814
:108D70000CEB020102EB001C0C4801326044007A4B
:108D8000082A01F8090CEFD11A6801321A601A6832
:108D9000082A01D100221A6001A803F0EBFE07B0F7
:108DA00000BD00BF7C0C0020780C0020040D0020CA
:108DB00073B50220002103F0CFFE1020002103F044
:108DC000CBFE01AC0021012003F0C6FE00250726E2
:108DD000142320468DF804308DF805608DF8065078
:108DE0008DF8075004F0F4FD152320468DF804306B
:108DF0008DF805608DF806508DF8075004F0E8FDF9
:108E0000204613238DF804308DF805608DF8065048
:108E10008DF8075004F0DCFD04F0A8F829464FF067
:108E2000007005F07BF87CBD2DE9F04101388AB077
:108E30000C46154607285BD8DFE800F04C40342884
:108E40001C5A10040C238DF81C3003238DF81D30A0
:108E500000238DF81B304FF0020354E00C238DF8F3
:108E60001C3003238DF81D3000238DF81B304FF08C
:108E700004023AE00C238DF81C3003238DF81D30DA
:108E800000238DF81B304FF010022EE00C238DF8DC
:108E90001C3003238DF81D3000238DF81B304FF05C
:108EA000140330E00C238DF81C3003238DF81D30A3
:108EB00000238DF81B304FF0280216E00C238DF8AC
:108EC0001C3003238DF81D3000238DF81B304FF02C
:108ED000640318E00C238DF81C3003238DF81D303B
:108EE00000238DF81B304FF0C802ADF81E200CE0B7
:108EF0000C238DF81C3003238DF81D3000238DF8D2
:108F00001B304FF00803ADF81E3004F02FF801219C
:108F10004FF0007005F002F80120014604F0F0FF68
:108F20000820012104F0ECFF0820002105F004F8DE
:108F300001214FF4EA1004F06BFC0AAE4FF400720A
:108F400026F8042D032331468A488DF82630153340
:108F50008DF8273004F0CCFB0423314685488DF88A
:108F600027304FF4807300260127ADF8243004F039
:108F7000BFFB05A88DF81A608DF814608DF8157088
:108F80008DF816608DF817608DF818708DF81970CF
:108F900003F0E0FCB4F5006F01A815DA4FF0FF32E2
:108FA0006301ADF80830ADF810608DF812708DF8DF
:108FB00004608DF805608DF80670ADF80A60ADF8B4
:108FC0000C20ADF80E2013E04FF0FF338DF8067043
:108FD000ADF810608DF812608DF804608DF80560B2
:108FE000ADF80860ADF80A60ADF80C30ADF80E30A1
:108FF00003F022FDDDB1B5F5006F18DA0022012380
:109000006901ADF80A208DF805204FF0FF3201A864
:10901000ADF808108DF812308DF804308DF8063058
:10902000ADF80C20ADF80E20ADF8103016E000239E
:109030000122ADF80A308DF812308DF80530ADF808
:1090400008304FF0FF3301A8ADF810208DF8042050
:109050008DF80620ADF80C30ADF80E3003F0ECFCC6
:10906000E30043F004030DF1040800270126022267
:109070006413ADF80A3040464FF0FF338DF80420FA
:10908000ADF808408DF805708DF80660ADF80C302D
:10909000ADF80E30ADF810708DF8126003F0CCFC16
:1090A000BD421ADDEB0043F004036D130322ADF85B
:1090B0000A304FF0FF3340468DF804208DF80570DC
:1090C000ADF808508DF812608DF80660ADF80C30E0
:1090D000ADF80E30ADF8106017E003238DF80430C2
:1090E0004FF004024FF0FF334046ADF80870ADF882
:1090F00010608DF812708DF805708DF80660ADF86F
:109100000A20ADF80C30ADF80E3008AF03F094FC37
:10911000012407260025142338468DF820308DF8C9
:1091200021608DF822508DF8234004F051FC152366
:1091300038468DF820308DF821608DF822508DF85A
:10914000234004F045FC132338468DF820308DF879
:1091500021608DF822508DF8234004F039FC022064
:10916000214603F0F9FC2146102003F0F5FC0AB07B
:10917000BDE8F081000C014030B52A4D2A4B2C6827
:109180001B680134082C08BF00249C4287B044D0DF
:10919000012001A903F0CAFD9DF80C20234B042AED
:1091A00009D12A68012103EB021251702A6803EBEE
:1091B0000213029A08E02A68002103EB02125170A0
:1091C0002A6803EB0213019A5A609DF80D30154A84
:1091D000022B164B04D1126803EB0213012203E0A9
:1091E000126803EB021300229A700E4B9DF80E10CA
:1091F0001A680E4B1201D15400230A4A06A9C81856
:1092000011680A4D03EB011110F8090C01334919DB
:10921000082B0872F1D1146002E0012003F06AFD0E
:1092200007B030BD000D0020740C0020800C002021
:1092300030B52A4D2A4B2C681B680134082C08BF16
:1092400000249C4287B044D0002001A903F06EFDA9
:109250009DF80C20234B042A09D12A68012103EB35
:10926000021251702A6803EB0213029A08E02A687E
:10927000002103EB021251702A6803EB0213019ADA
:109280005A609DF80D30154A022B164B04D1126816
:1092900003EB0213012203E0126803EB0213002226
:1092A0009A700E4B9DF80E101A680E4B1201D15495
:1092B00000230A4A06A9C81811680A4D03EB0111D8
:1092C00010F8090C01334919082B0872F1D1146008
:1092D00002E0002003F00EFD07B030BD000D0020BD
:1092E000740C0020800C0020F0B5384B1A787AB14D
:1092F0005968374A013159601168364B01311160A4
:109300001A6812B11A68013A1A6000222F4B00E065
:1093100001221A70304B1A683AB11A68013A1A6081
:109320001B6813B92D4B01221A702D4B2D4A9B8CB3
:109330002D499BB2136010680B68984218DD1468C1
:1093400008682A4B201AB0F5004F294806DAD3E9FD
:109350000045166809680268701A29E0D3E90045DB
:109360000E68116806F5803C0268C1EB0C0011E044
:1093700010680B68984223DA0C6810681B4B201A9F
:10938000B0F5004F1A480ADAD3E900450E681168B3
:109390000268701A5043261A65EBE0770CE0D3E9B7
:1093A00000451268096802F5803C0268C1EB0C00B8
:1093B0005043261845EBE07730463946C3E90001B3
:1093C000084B1A68084B1A60F0BD00BF3804002033
:1093D00000070020680C00206C0C0020700C00209E
:1093E00000080040600C0020380B0020580B0020C3
:1093F000600B0020014B5868704700BF3804002004
:1094000008B5042004F0ACFF48F6A04004F0B8FF13
:10941000012004F0BBFF04480321002204F0A6FB56
:10942000012004F0C9FF08BD9AC30200000000003B
:109430000828F8B508D009280ED008B100205AE055
:109440003B4B188880B256E0394B588840F21323C2
:1094500080B2584300134EE0354B988880B208F034
:1094600039FB07F01BFF0022324B07F06BFF22A3F2
:10947000D3E9002306460F4607F064FF20A3D3E993
:10948000002307F0ADFD1EA3D3E9002304460D46DB
:109490003046394607F056FF1BA3D3E9002308F0F6
:1094A0007BF802460B462046294608F075F808F07E
:1094B0000BFA07F0F3FE00221F4B08F06DF807F0DF
:1094C00095F913A3D3E9002307F03CFF12A3D3E9D6
:1094D000002307F085FD02460B4611A1D1E90001EA
:1094E00008F05AF810A3D3E9002307F077FD08F03D
:1094F000EBF908F00DFDF8BD6666666666660AC0A3
:109500006666666666660A409A99999999990140D5
:10951000C3F5285C8FA272400000000000FEAA4044
:109520009A999999FD6F2F41C3F5285C8F1271406C
:10953000400400200000303F00002440F0B593B00C
:1095400011AF01240025032641483946ADF84440B7
:109550008DF846608DF8475004F0CAF84FF01103BB
:1095600039463C48ADF844308DF846608DF8475098
:1095700004F0BEF82046214604F0B4FC21464FF426
:10958000007004F0BDFC344803F0FCFC334B32485F
:109590000193334B01A9029380230693DB180793B1
:1095A00003F540730893A3F57873099303F5FF530C
:1095B0000A930395049605950B9503F053FD2648F1
:1095C000214603F07FFD4FF4602326480CA90E933B
:1095D0008DF834400C958DF835400F958DF840602E
:1095E00002F0ECFF1F4808212246334603F068F8DA
:1095F0001C4804210222334603F062F83346324607
:109600001848294603F05CF82A4616484FF4FC61D6
:1096100003F018F81348214603F00AF811482146D0
:1096200002F0FCFF0F4803F017F80E4803F01AF899
:109630000028FAD10B4803F019F80A4803F01CF887
:109640000028FAD10748012103F01AF813B0F0BD41
:10965000000C014000080140080002404C24014079
:109660004004002000240140014B03221A6070478F
:1096700048040020044A054B927A0AB1052200E012
:1096800001221A60704700BF900D0020480400209E
:10969000704700BF014B00225A6070474804002009
:1096A00008B5074B1A6892B242F008021A601A68AD
:1096B00092B242F004021A60FFF7D6FF08BD00BF65
:1096C000405C004010B5064C4FF6FB73226802EA7E
:1096D00003032360FFF7CEFF4FF40643236010BD62
:1096E000405C0040072818BF1F4B10B51E4C18BF28
:1096F00018702378052B33D8DFE803F003060A0E31
:109700001621FFF7DFFF2BE0FFF7DCFF042328E043
:1097100002236370013324E06378013BDBB26370A2
:109720006378FBB9042218E0104B1A6892B242F039
:1097300010021A6005232370DB18637012E063784F
:10974000013BDBB26370637863B9084A4FF6EF738D
:10975000116801EA030313600622034B1A7001E04B
:109760000623237010BD00BFF40D0020405C0040B4
:10977000034B9B7A13B1034B05221A60704700BF5D
:10978000900D002048040020014B04221A6070470D
:1097900048040020034B1A7A202A01D100221A72B1
:1097A000704700BF48040020704700BF212808B55B
:1097B00008D1124B1B681B7803F07F03212B1AD1B1
:1097C0000F4B0EE0202816D10C4B0E4A1B681B785D
:1097D00010720D4A03F07F03212B0CBF13460023A8
:1097E0004BB1064A4FF0000112680020518293618C
:1097F0009847002000E0022008BD00BFF00D0020C7
:1098000041980008480400205D980008074B1B6839
:109810001B7803F07F03212B05D1022801D02228D9
:1098200001D1002000E00220704700BFF00D0020B1
:1098300019B9012801D8084600E00220704700BF8E
:1098400028B9044B4FF008021B681A8200E0024856
:10985000704700BFF00D00204800002028B9044BDD
:109860004FF008021B681A8200E00248704700BFF0
:10987000F00D0020480000200B4B10B5DA6882B1D3
:109880001B68052B01D000220BE0002303E00749F1
:10989000595CC15401330449CC68A342F7D3002377
:1098A000CB60104610BD00BF48040020F80D00201A
:1098B000084BDB68082B01D800200AE00023064A89
:1098C0009A5CC2540133092BF9D1024B0022DA60B1
:1098D0000120704748040020F80D002010B5074C07
:1098E0000B468AB2C021636006F0A6FA0120A18867
:1098F00006F0B0FC012006F07BFB10BD4804002000
:1099000007B5142200238DF8042001A801228DF848
:1099100006308DF807208DF8053004F059F80EBD9B
:1099200007B5142200238DF8042001A801228DF828
:1099300006308DF807208DF8053004F049F80EBD8B
:1099400008B5064B1B68DB78042B01D9002004E026
:10995000034901EBC30105F017FE08BDF00D00201F
:109960005000002008B5024905F00EFE08BD00BFFA
:109970007000002008B5024905F006FE08BD00BFD2
:1099800078000020334B10B51B686FF03F020024B5
:109990005A72DC729C72204606F0A2FA20464FF4FE
:1099A000007106F0BBFA1021204606F0CDFA4021E6
:1099B000204606F023FC8021204606F00FFC2046BE
:1099C00006F04CFB244B204693F8641006F064FC30
:1099D000204606F01BFB0120214606F09FFA0120DD
:1099E000C02106F0FBFB0120202106F0ADFA01208A
:1099F000214606F0C1FA02204FF4C06106F08EFA4B
:109A000002204FF4807106F0E9FB0220214606F0A7
:109A1000B3FA0220202106F097FA0320214606F02F
:109A20007DFA03204FF4887106F0E8FB0320402103
:109A300006F032FC03204FF4405106F09DFA214617
:109A4000032006F081FA204605F0ACFD034B01220D
:109A50001A6010BDF00D00204800002048040020CE
:109A600008B5174B174A196889B211801649128830
:109A7000098801EA020212F4806F05D04FF6FF3226
:109A80001A60124BDB6B98470E4B1A880E4B1B88E3
:109A900003EA020212F4007F08D009490C4A4FF68B
:109AA000FF500860117C0131C9B21174054A128857
:109AB000134013F4004F01D006F0FAF808BD00BFC0
:109AC000445C0040860D0020380E00204800002035
:109AD0004804002010B5032006F00EFC064C034697
:109AE00002464FF488710548E36006F0BDF9032093
:109AF00006F08CFA10BD00BF48040020F80D0020CD
:109B000008B500B10120FAF785FF08BD38B5064D4C
:109B100001232B60054B002420461C60FFF7F0FF5B
:109B200003232B60204638BD405C0040445C00406D
:109B300008B5FFF7EBFF08BD08B50120FFF7E0FF10
:109B4000064B0121196006494FF4E0520A8005498D
:109B50000020186008601A6008BD00BF405C00402B
:109B6000380E0020445C0040084B10B51B680024F0
:109B70009C72FFF7E1FF064A4FF406431460043A73
:109B80001360044A1460044A138010BDF00D0020D5
:109B9000445C004048040020380E0020002008B536
:109BA00004F024F94FF40000012104F0B7F908BDD6
:109BB00008B5FFF7F3FFFFF7B3FE06F01BF808BD8B
:109BC000704700BF704700BF704700BF704700BFBD
:109BD000704700BF704700BF704700BF704700BFAD
:109BE00008B5FAF75BFD052805D9FAF757FD40F2ED
:109BF000F933984201D9012200E00022094B5A6052
:109C0000094B1B786BB1074B08495A68084B0A602F
:109C10001AB91A6842F0080202E01A6822F0080233
:109C20001A6008BD04070020FE060020EC06002094
:109C30009406002010B5FFF7DDFB074C2368C31A1C
:109C4000B3F5FA7F07D9054BDA6882F00402DA60CF
:109C5000FFF7D0FB206010BD3C0E0020000C01403F
:109C6000024B03EBC003D879704700BF5C040020AF
:109C7000024B03EBC0035879704700BF5C0400201F
:109C8000024B03EBC0039879704700BF5C040020CF
:109C9000024B0B2202FB0033187A70475C04002051
:109CA000024B0B2202FB0033587A70475C04002001
:109CB000024B0B2202FB0033D87A70475C04002071
:109CC000024B0B2202FB0033987A70475C040020A1
:109CD000024B0B2202FB0033187B70475C04002010
:109CE000024B0B2202FB0033587B70475C040020C0
:109CF000024B0B2202FB0033987B70475C04002070
:109D0000024B0B2202FB0033187C70475C040020DE
:109D1000024B0B2202FB0033587C70475C0400208E
:109D2000024B0B2202FB0033987C70475C0400203E
:109D3000024B052202FB0033187D70475C040020B3
:109D4000024B052202FB0033587D70475C04002063
:109D5000024B052202FB0033987D70475C04002013
:109D6000024B052202FB0033D87D70475C040020C3
:109D7000024B052202FB0033187E70475C04002072
:109D8000024B032202FB0033187F70475C04002063
:109D9000034B032202FB003393F91D00704700BF01
:109DA0005C040020024B032202FB0033987F7047C3
:109DB0005C040020024B03EBC00393F820007047C3
:109DC0005C040020024B03EBC00393F821007047B2
:109DD0005C040020024B03EBC00393F822007047A1
:109DE0005C040020024B03EBC00393F82300704790
:109DF0005C040020024B03EBC00393F8240070477F
:109E00005C040020024B03EBC00393F8250070476D
:109E10005C040020024B03EBC00393F8260070475C
:109E20005C040020024B03EBC00393F8270070474B
:109E30005C04002006281AD8DFE800F004070A0DA9
:109E4000101316000A4B9B6A10E0094BDB6A0DE009
:109E5000074B1B6B0AE0064B5B6B07E0044B9B6BED
:109E600004E0034BDB6B01E0014BDB7B0B607047D5
:109E70005C04002070B5C0F30741054600220120B4
:109E8000FAF726FF0A4C0602C5F30721002201203B
:109E9000A662FAF71DFF064301203602E9B2024628
:109EA000A662FAF715FF06433609A66270BD00BF29
:109EB0005C0400202D4B032202FB003310B51C3341
:109EC00093F901203F2A01DD3F225A70274B0322DC
:109ED00002FB00331C3393F9012012F13F0FBCBF8A
:109EE0006FF03E025A70214B032202FB00331C33F9
:109EF0009A781F2A01D91F229A701C4B032202FB59
:109F000000324FF440211964127F012A04BF4FF43C
:109F100050221A64154B03EBC00292F827203AB97D
:109F2000033202FB0032527F196C02F07F020BE019
:109F3000032101FB003191F81DC002F003020CF077
:109F40007C0C196C4CEA0202084C41EA02221A64A9
:109F5000032303FB0040236C827F42EA030318467D
:109F60002364FFF787FF236CA36310BD5C0400200C
:109F700008B5044B032202FB00339977FFF79AFFE1
:109F800008BD00BF5C04002008B5044B032202FB9F
:109F900000335977FFF78EFF08BD00BF5C04002037
:109FA00008B5044B032202FB00331977FFF782FF49
:109FB00008BD00BF5C040020264B052210B502FB43
:109FC00000331A7D012A01D901221A75214B05227D
:109FD00002FB003314335A78032A01D903225A7042
:109FE0001C4B052202FB003314339A780F2A01D947
:109FF0000F229A70174B052202FB00331433DA78D4
:10A00000032A01D90322DA70124B052202FB003326
:10A0100014331A790F2A01D90F221A710D4C052316
:10A0200003FB004000F114021379017D43F4202367
:10A03000507843EAC133917843EA4033D27843EA17
:10A04000012343EA421318462364FFF713FF236CEE
:10A05000636310BD5C04002008B5044B052202FBBD
:10A0600000331976FFF7A8FF08BD00BF5C0400208D
:10A0700008B5044B052202FB0033D975FFF79CFF9E
:10A0800008BD00BF5C04002008B5044B052202FB9C
:10A0900000339975FFF790FF08BD00BF5C040020F6
:10A0A00008B5044B052202FB00335975FFF784FF06
:10A0B00008BD00BF5C04002008B5044B052202FB6C
:10A0C00000331975FFF778FF08BD00BF5C0400205E
:10A0D000514B0B2210B502FB00331A7A032A01D927
:10A0E00003221A724C4B0B2202FB003308339A787E
:10A0F000032A01D903229A70474B0B2202FB00333B
:10A1000008331A790F2A01D90F221A71424B0B22F8
:10A1100002FB003308335A79072A01D907225A7102
:10A120003D4B0B2202FB003308339A790F2A01D9E9
:10A130000F229A71384B0B2202FB003310335A78EE
:10A140000F2A01D90F225A70334B0B2202FB003326
:10A1500010339A780F2A01D90F229A702E4B0B22B6
:10A1600002FB0032117AC90341F400241C64527AC4
:10A1700012B141F404211964274B0B2101FB00317A
:10A18000C97A19B1196C41F400511964224B8AB98A
:10A190000B3202FB0032083292F804C091784FEA89
:10A1A000CC1C1C6C4CEAC12C51794CEA040242EAEA
:10A1B00001121DE00B2202FB0032127C1AB11A6C54
:10A1C00042F480521A64144B0B2101FB0031103110
:10A1D00091F801E01A6C897842EACE1201F0070C7E
:10A1E00042EA0C1211F0080F1A6402D042F4006225
:10A1F0001A64094B0B2202FB00300830C27922B9E5
:10A2000081791A6C41EA02021A64034C206CFFF750
:10A2100031FE236C236310BD5C04002008B5064B9F
:10A220000B2202FB00330833DA791AB10022DA710B
:10A23000FFF74EFF08BD00BF5C04002008B5064BC9
:10A240000B2202FB00330833DA791AB90132DA71D2
:10A25000FFF73EFF08BD00BF5C04002008B5044BBB
:10A260000B2202FB00339974FFF732FF08BD00BFD9
:10A270005C04002008B5044B0B2202FB0033597428
:10A28000FFF726FF08BD00BF5C04002008B5044BA3
:10A290000B2202FB00331974FFF71AFF08BD00BF41
:10A2A0005C04002008B5044B0B2202FB00339973B9
:10A2B000FFF70EFF08BD00BF5C04002008B5044B8B
:10A2C0000B2202FB00335973FFF702FF08BD00BFEA
:10A2D0005C04002008B5044B0B2202FB0033197309
:10A2E000FFF7F6FE08BD00BF5C04002008B5044B74
:10A2F0000B2202FB00339972FFF7EAFE08BD00BF94
:10A300005C04002008B5044B0B2202FB0033D97219
:10A31000FFF7DEFE08BD00BF5C04002008B5044B5B
:10A320000B2202FB00335972FFF7D2FE08BD00BFBB
:10A330005C04002008B5044B0B2202FB00331972A9
:10A34000FFF7C6FE08BD00BF5C04002010B5254B1A
:10A350004FF460221A6403EBC00292F8272012B176
:10A360004FF470221A641F4B03EBC00292F82110C5
:10A3700092F820C01C6C090341EA8C312143196416
:10A3800092F82220012A04BF41F480611964154B20
:10A3900003EBC00191F823C01A6C42EA0C221A6444
:10A3A00091F82410012904BF42F080021A640D4B79
:10A3B00003EBC00292F82520012A03D11A6C42F067
:10A3C00040021A64074C04EBC00090F82620236C6E
:10A3D00043EA021318462364FFF74CFD236CE36342
:10A3E00010BD00BF5C04002008B5044B03EBC003A4
:10A3F00083F82610FFF7AAFF08BD00BF5C04002009
:10A4000070B50F4B064603EBC00393F82650032D9F
:10A4100002D00321FFF7E8FF3046FFF797FF084B14
:10A420009C6A14F4002F1CBF6FEA04346FEA1434E2
:10A43000032D03D030462946FFF7D6FF204670BDD6
:10A440005C04002008B5044B03EBC00383F825101F
:10A45000FFF77CFF08BD00BF5C04002008B5044B7B
:10A4600003EBC00383F82410FFF770FF08BD00BFA3
:10A470005C04002008B5044B03EBC00383F82310F1
:10A48000FFF764FF08BD00BF5C04002008B5044B63
:10A4900003EBC00383F82210FFF758FF08BD00BF8D
:10A4A0005C04002008B5044B03EBC00383F82110C3
:10A4B000FFF74CFF08BD00BF5C04002008B5044B4B
:10A4C00003EBC00383F82010FFF740FF08BD00BF77
:10A4D0005C040020064B10B503EBC003044683F870
:10A4E0002710FFF733FF2046FFF7E4FC10BD00BF45
:10A4F0005C04002010B5144B00221A6403EBC00268
:10A50000527912B14FF400721A640F4B03EBC00280
:10A5100092791AB11A6C42F480721A640A4B03EBF6
:10A52000C003DA790F2A01D90F22DA71064C04EB45
:10A53000C000C279236C42EA030318462364FFF784
:10A5400099FC236CE36210BD5C04002070B5084DDB
:10A550009DF810E09DF8146005EBC0042671627050
:10A56000A37084F803E005F83010FFF7C3FF70BD57
:10A570005C04002008B5034B03EBC0039971FFF79F
:10A58000B9FF08BD5C04002008B5054B03EBC00310
:10A59000597109B10422DA71FFF7ACFF08BD00BFA1
:10A5A0005C04002008B5054B042903EBC003D971F6
:10A5B00001D000225A71FFF79DFF08BD5C04002006
:10A5C0002DE9F047344D0446401990F844000E46FA
:10A5D00017469846DDF82090DDF824A004281FD8FF
:10A5E000DFE800F003090F151B002046FFF770FDA0
:10A5F0006519012316E02046FFF7A8FE651902231E
:10A6000010E02046FFF7D8FC651903230AE0204636
:10A61000FFF750FC6519042304E02046FFF76AFFAA
:10A620006519002385F844301B4B03EBC40494F8F0
:10A630002620012A0DD002D3022A23D111E016B11F
:10A640009B6A9B0C3370EFB1134B9B6A9B0A3B7068
:10A6500018E0B8F1000F15D09B6A9B0AC8F80030CB
:10A6600010E0B8F1000F04D09B6ADB0B5B01C8F867
:10A670000030B9F1000F05D0074B9B6AC3F3842368
:10A6800089F80030BAF1000F03D0034B9B6A8AF8B7
:10A690000030BDE8F08700BF5C040020214B10B5FE
:10A6A000032200244FF0050C02214FF0010E83F825
:10A6B00025E0197383F80EC09A745C7483F81CE06B
:10A6C00083F81DC083F81EC083F8202083F8212062
:10A6D00083F8224083F8234083F8244083F826102F
:10A6E00083F827401C755C759C75DC751C765C7165
:10A6F0009C71DC7119725C72DC729C725A73DC732F
:10A700001C742046FFF758FC2046FFF7D3FB204679
:10A71000FFF71CFE2046FFF7EDFE2046FFF7D8FCB2
:10A7200010BD00BF5C04002008B5044A0023917AE4
:10A73000034A18461370FAF7B5F908BDB80B0020A4
:10A74000200C00202DE9FF417F4B1A7822B90132FD
:10A750001A706FF000425A607B4B1C7A5CB9E0B211
:10A76000F9F764FF784B03F10C0210550134082C03
:10A77000F5D101221A7227240025E8B2F9F756FF15
:10A78000724A535D834219D0714B291D53F8213011
:10A790005055022B05D0032B0AD0012B0ED168B1E6
:10A7A00006E058B96B4A115D012907D1135505E040
:10A7B000684B1A5D012A01D101321A550135013465
:10A7C000082DDAD1644EF36993B1644C25787DB9D4
:10A7D000FEF710FE624AF3691268821A002AB8BFB7
:10A7E00052429A4204D9284601F08EFA012323707E
:10A7F000594E336A93B15B4C25787DB9FEF7FAFD6B
:10A80000594A336A1268821A002AB8BF52429A42E1
:10A8100004D9284601F078FA012323704A4D534C9D
:10A820002A7D930004EBC3010E7B002E00F02B81E8
:10A830004F48504F504E0021C318BF18B61810464D
:10A840000A4600970196FFF7BBFE2B7D04EB4314ED
:10A85000227B013A042A00F20581DFE812F00500AC
:10A860004E00D3004E00D300444A374D926812F494
:10A87000004F1BD05D192A7E022A04D1404AD25CC7
:10A88000002A00F0EF80394A2F4C02EB43121846A1
:10A89000517AFAF707F9207DFFF7C0FC237D384A8B
:10A8A0000021E418D15402232376DBE05D192A7ECF
:10A8B000012A04D1324AD25C002A00F0D3802B4C0A
:10A8C000184604EB4313997AFAF7ECF81E4B187DFF
:10A8D00004EB4014A37A13B9FFF7B0FC04E0284B53
:10A8E0001B5C0BB1FFF79AFC174A2549137D00202A
:10A8F000D218C85401231376B4E01F4A124DD25621
:10A90000002A3FDB5D192A7E022A02D11C4AD25C52
:10A910008AB1164A0C4C02EB43121846517AFAF7E8
:10A92000C1F8207DFFF77AFC237D154A0021E41849
:10A93000D15402232376044C257DFEF75BFD04EB06
:10A940008504606056E000BFA4040020B00400202D
:10A95000E00B0020300C0020080000201D0C00201F
:10A96000180C0020190B0020100C0020B80B002040
:10A97000500B0020240B0020B00B002000080140E9
:10A980001C0C00205B191B7E012B11D0FEF732FD41
:10A990002B7D8B4A05EB830502EB43139B8B0A222D
:10A9A00053436A68821A002AB8BF52429A4204DCB2
:10A9B000844B854A1B7DD35CE3B1824D804C287D5E
:10A9C00004EB4013997AFAF76DF8287D04EB4014F4
:10A9D000A37A13B9FFF732FC04E07B4B1B5C0BB18D
:10A9E000FFF71CFC774A7849137D0020D218C85421
:10A9F00001231376734B1A7D714B03EB42131B7BC0
:10AA0000042B20E06F4A9A18127E022A02D16E4A65
:10AA1000D25C8AB16A4A6B4C02EB43121846517AF7
:10AA2000FAF740F8207DFFF7F9FB237D664A002105
:10AA3000E418D15402232376624B1A7D604B03EB5A
:10AA400042131B7B052B0DD1604B9B6813F4004F09
:10AA500004D05F4B4FF400425A6103E05C4B4FF46B
:10AA600000421A61FEF7C6FC564CE369C31A002B7C
:10AA7000B8BF5B420A2B40F36A83F9F781FEFEF709
:10AA8000B9FCE06163E3F9F77BFEFEF7B3FCEB6929
:10AA9000C31A002BB8BF5B420A2B40F35883297DB1
:10AAA0003046490141F00A0101F0EA0100F0EEFFF1
:10AAB0000446287D01F04CF92B7D0C205843454974
:10AAC0004218157A0DB1455800E05568424AD25CEB
:10AAD000032A00F2E780DFE802F002831C4B002C1F
:10AAE00000F0E080364A374D02EB4311C97F3A4E01
:10AAF00029B11846F9F7D6FF2B7D032207E002EBB8
:10AB000043121846517AF9F7CDFF2B7D0222F254F9
:10AB1000C8E04CB95B0143F0080101F0E8012046B0
:10AB200000F0B4FF002865D0264E254B307D03EBA6
:10AB30004013D97F002900F0AE80002D84EAE47232
:10AB4000B8BF6D42A2EBE472AA4202D0002C40F0E2
:10AB50009C80224B53F830108A4280F09C8003EB9B
:10AB6000C0031979F9F79EFF164B01211B7D90E078
:10AB7000002D84EAE471B8BF6D42A1EBE471A942F3
:10AB800002D0002C40F08780144A0E4D52F833005A
:10AB9000114E814208D202EBC30218461179F9F72F
:10ABA00081FF2B7D012208E0054A184602EB431382
:10ABB000597AF9F777FF2B7D0222F2546BE000BF40
:10ABC000B80B0020A40400201C0C00200008014049
:10ABD00000100140640B0020200C0020280B0020F6
:10ABE00044BB5B0143F0080101F0E801204600F09E
:10ABF0004DFFF8B9FEF7FEFB1F4D204A2B7D4FF0AD
:10AC00000A0E02EB4311B1F81CC099004E19766888
:10AC10000EFB0CFC861B002EB8BF7642664541DD5C
:10AC200002EBC1021846917AF9F73CFF2B7D144ADA
:10AC3000D45437E0104E114A337D02EB4312D17FDA
:10AC400049B3002D84EAE472B8BF6D42A2EBE4720E
:10AC5000AA4200D0C4B90B4951F833108A421AD322
:10AC6000064A184602EB4313597AF9F71BFF024BC9
:10AC700002211B7D0DE000BFA4040020B80B0020C2
:10AC8000200C0020280B00201846F9F70BFF337D1D
:10AC90000321A34AD154A34D2E7DFEF7ABFB05EB58
:10ACA000860568609F4DA04F2B7DA04E1846F61874
:10ACB000FF189F4B002103EB80030A460196009783
:10ACC0009C4EFFF77DFC287D06EB40139B6943B348
:10ACD000F9F7D6FB28B3287D84EAE47206EB40132B
:10ACE0009B69A2EBE4729A421BD901F00DF82A7D10
:10ACF000914906EB42139B7F0120885443B1B27FF8
:10AD00009A4205D1013800F0FFFF002000F03AFA26
:10AD1000844B8A4A1B7D0F33D15C012901D101315B
:10AD2000D154804D2B7D022B25D8002000F08AFDC8
:10AD300095F8203010F0010F03F0F80385F820306B
:10AD40001CBF43F0010385F8203010F0040F8DF88C
:10AD50000C0006D0734B93F8202042F0020283F8D7
:10AD6000202010F0100F06D06E4B93F8202042F0F8
:10AD7000040283F82020724A137853B1694991F88C
:10AD800020100B4205D16F496F480978037001B953
:10AD900011706D4B1B784BB1624A92F8202003EA88
:10ADA00002029A4202D1694B01221A705D4B93F85C
:10ADB000202012F0010F0AD093F8213013F0010F78
:10ADC00005D15E4BDA78012A01D10132DA70554B98
:10ADD00093F8202012F0020F0AD093F8213013F0DC
:10ADE000020F05D1554B1A79012A01D101321A718E
:10ADF0004C4B93F8202012F0040F0AD093F8213026
:10AE000013F0040F05D14D4B5A79012A01D10132BB
:10AE10005A71444D03222B7D04A8B3FBF2F2821831
:10AE200012F9042C95F82010002A85F821104ADA2E
:10AE30005B0143F01601002001F0F60102AA00F0C8
:10AE40003DFE9DF80A3013F0400F08D02A7D3B49A3
:10AE500052001B32885C012801D10130885413F064
:10AE6000800F0AD02F49354A097D0E3112F81100A2
:10AE7000012802D1013002F8110013F0100F09D09F
:10AE8000284A2E49127D52001B32885C012801D1CC
:10AE90000130885413F0200F0AD0224A274B127D2C
:10AEA0000E3213F81210012902D1013103F81210E9
:10AEB0001C4B0020197D02AA490141F0160101F046
:10AEC000F60100F097FF174F1A4E3B7D06EB431239
:10AED0005269002A00F081801D4AD55C002D7CD18A
:10AEE000002C7AD05B0143F0020101F0E201284618
:10AEF00000F092FD8046387DF9F73AFD397DC0EBD0
:10AF0000080806EB41135B69B8F1000F83EAE372AE
:10AF1000B8BFC8F10008A2EBE37290455DDD19E00F
:10AF2000200C0020A4040020240B0020B00B0020E3
:10AF3000500B0020B80B0020AC0B0020300C002080
:10AF40004C0B0020200B00203C0B0020640C002048
:10AF5000340B0020002B0EDD084600F0D5FE3B7DB3
:10AF600006EB43139B7F3BB3B27F9A4224D1284622
:10AF700000F0CAFE1DE02846022200F027FD397DC0
:10AF80002846490141F0080101F0E80100F09EFE69
:10AF90003B7D06EB43139B7F73B1B27F9A420BD18B
:10AFA00029462846022200F011FD2846082100F01B
:10AFB0008DFE284600F0E6F8664B674A1B7D153388
:10AFC000D15C012901D10131D154624B634A1B7D0F
:10AFD00001211846D15400F0D5F8614F3B68002B91
:10AFE00047D05C4E5D4A337DD55C002D41D1002CAD
:10AFF00040D05B0143F0020101F0E201284600F07D
:10B000000BFD8046307DF9F759FA3B68C0EB080824
:10B01000B8F1000F83EAE372B8BFC8F10008A2EBF1
:10B02000E372904531DD002B317D03DD084600F0F1
:10B030006BFE0CE02846022200F0C8FC317D284659
:10B04000490141F0080101F0E80100F03FFE414BE9
:10B05000414A1B7D1533D15C012901D10131D15405
:10B060003C4B3E4A1B7D01211846D15400F08AF822
:10B070000BE054B9374B0020197D490141F008011C
:10B0800001F0E80100F002FD20B1324D354B2E7D7C
:10B090009B5D43B32F4B344A1B7D02EB4312D28995
:10B0A00012B9304AD35C1BB3FEF7A4F9294D2E49DF
:10B0B0002B7D4FF00A0C9A0001EBC201C98952198D
:10B0C000526A0CFB01F1821A002AB8BF52428A422E
:10B0D0000EDD264EF25C5AB91846FFF7AFF82B7D0D
:10B0E0000122F25404E0FEF785F905EB860568625B
:10B0F000184E1F4D307D002C55F83030B8BF6442DB
:10B100009C420AD2FEF734FE337D05EBC3056A7913
:10B1100082420DD11846002108E0FEF729FE337D5A
:10B1200005EBC3056979884202D01846FEF794FF03
:10B13000084C207D00F034F8237D0133DBB2237509
:10B140000BB100232375FEF755F9024BD861BDE81A
:10B15000FF8100BFA4040020300C0020340B00202D
:10B16000440B0020280C0020B80B00202C0C0020E1
:10B17000280B0020024B1A5C0AB901321A5470479E
:10B18000CC040020024B1A5C0AB10F221A547047FB
:10B19000CC040020014B185C704700BFCC04002099
:10B1A0002DE9F3474601F5B2044645F07C01002045
:10B1B00001AA00F083FCB74A610002EB4413187A3D
:10B1C00006EB020710F0400F9DF8063012D04FF04A
:10B1D00001084FF0020C08FA01F80CFA01FCB15812
:10B1E0007E680CEA030208EA0307C1F10009C6F110
:10B1F000000A0FE04FF0010C4FF002080CFA01FCBE
:10B2000008FA01F156F80290D7F804A00CEA0302FC
:10B2100001EA030710F0800F00F03F0606D09E4BB6
:10B220009B6883F40048C8F3C03803E09A4B9B68DE
:10B23000C3F3C038731E072B00F2D182DFE813F08E
:10B2400008000800080008006E016E016E016E0122
:10B25000924B1B5D013B0E2B00F2C182DFE813F025
:10B260000F003D00530062007A0082008E00A000B3
:10B27000D10014012401BF0243014E01A60201AA1C
:10B2800045F014010020854F00F018FC9DF80530B2
:10B2900045F0060507EB8408C8F80430294600206D
:10B2A00000F0F4FB0222C8F808002146002000F05C
:10B2B0008DFB023E0020294640F2FF7200F0F2FCB6
:10B2C000F6B200200322214600F05AFB012E01D8DD
:10B2D000022300E004233B5581E2704E002006EB80
:10B2E00084035A68214602F00402824214BF0522F8
:10B2F000012200F045FB45F008014A46002000F01D
:10B30000D1FC032324E0002A00F0698245F0020109
:10B31000002000F081FB614B04221A55604B43F87A
:10B3200024005CE25D4E002006EB84035A6821464F
:10B3300002F00402824214BF0622022200F020FB27
:10B3400045F00801C9F10002002000F0ABFC052324
:10B35000335544E2002F00F04282204600F0D4FC36
:10B3600006222FE200202146032200F009FB45F0CF
:10B3700008015246002000F095FC68E1002F40F0E3
:10B380002E8245F008053A463846294600F08AFCE8
:10B39000CAF100023846294600F084FC082211E276
:10B3A000002F00F01C8245F00201002000F034FB69
:10B3B00006460020024645F0080100F073FC384BB9
:10B3C000002053F824702146BF1B43F82470032249
:10B3D00000F0D6FA8AEAEA7245F00601A2EBEA72B8
:10B3E000002000F05FFC610101F0E0013246002026
:10B3F00000F0C4FB00200246214600F0E7FA0922D3
:10B40000E0E1002000F01EFA630050FA03F313F0AD
:10B41000010F00F0E48145F002073946002000F0FA
:10B42000FBFA204B45F0080543F8240000200246B3
:10B43000294600F037FC00200222214600F0C6FA1F
:10B4400000200246394600F099FB002061010246C7
:10B4500001F0E001033E00F091FBF6B2002120462E
:10B46000F9F75CFA012E0D4E0CD80020214602227D
:10B4700000F0ACFA2946CAF10002002000F012FCEC
:10B480000A2365E70E2363E7002F00F0A8810B2253
:10B4900098E100BFB80B002000080140CC04002058
:10B4A0001C0B0020DC0B0020002F40F0988145F0A1
:10B4B0000201384600F0B0FA45F0080106463A4667
:10B4C000384600F0EFFB6101022296FBF2F201F038
:10B4D000E001384600F052FB3A463846214600F07B
:10B4E00075FA0D226EE1002000F0ACF9630050FA0D
:10B4F00003F313F0010F00F0728162E1A84E45F0F2
:10B50000060106EB84050020AA6800F0CBFB2A792F
:10B510000020214600F034FA002319E7A04B1B5D00
:10B52000013B0E2B00F25B81DFE813F00F003400CB
:10B530005200620081005901930059015901CC0069
:10B54000DC00AD0008014F01400145F0140101AAE3
:10B550000020934F00F0B2FA9DF805C007EB84037A
:10B5600000200222C3F804C0214600F02FFA002078
:10B5700045F0060140F2FF7200F094FB0020032228
:10B58000214600F0FDF9062E02D0082E7FF4A2AE6F
:10B59000022217E1062E0CD1814B002003EB84031D
:10B5A0005A68214602F00402824214BF0522012299
:10B5B00004E0082E04D100202146032200F0E0F927
:10B5C0004A4645F00801002000F06CFB0322F9E038
:10B5D000731FDBB2012B05D822B1062E704E30D17D
:10B5E0000423B5E6B8F1000F00F0F9800C22E9E081
:10B5F000052E0CD16A4B002003EB84035A682146C8
:10B6000002F00402824214BF0622022204E0072E46
:10B6100004D100202146032200F0B2F9C9F1000252
:10B6200045F00801002000F03DFB0522CAE0731F31
:10B63000DBB2012B07D837B1052E594E01D10223B9
:10B6400086E60F2384E6B8F1000F00F0C8800722D9
:10B65000B8E0B8F1000F40F0C280073EF6B2012E0C
:10B660000DD94F4B404603EB84035A68214602F044
:10B670000402002A14BF0522012200F081F945F0DE
:10B680000801524619E0B8F1000F40F0A880073ECB
:10B69000F6B2012E0DD9424B404603EB84035A68A3
:10B6A000214602F00402002A14BF0622022200F002
:10B6B00067F945F00801CAF10002002000F0F2FA33
:10B6C0000A227FE0B8F1000F00F0898045F0020106
:10B6D000002000F0A1F9324B0B2103EB8402195535
:10B6E000D0607CE0B8F1000F79D145F0020140460E
:10B6F00000F092F92B4BA700294E03EBC7038AEA0F
:10B70000EA72814645F00601A2EBEA72404683F8F0
:10B710000D80BF1900F032FAFB68610199440223E1
:10B7200099FBF3F201F0E001404600F027FA4046B1
:10B730002146424600F04AF90D2309E6002000F0B8
:10B7400081F8630050FA03F313F0010F47D0144B54
:10B750000E2245F002061A553146002000F05CF931
:10B76000114B45F0080143F824000020024600F088
:10B7700099FA21460020022200F028F900203146E3
:10B78000024600F0FBF900206101024601F0E001F1
:10B7900000F0F4F920460021F9F7C0F81FE000BFDF
:10B7A000CC040020B80B0020DC0B00200020214638
:10B7B000022200F00BF9002045F00801024600F0DB
:10B7C00071FA0E22074B1A5509E0064D002005EBD1
:10B7D00084031A79214600F0D3F800232B55BDE8E5
:10B7E000FC8700BFCC040020154B10B503EB001202
:10B7F000926891420EDD8A1AC2F18074A2424FEA29
:10B80000001C03DC63445C6812190EE063445A6850
:10B81000141B0FE00FDA521AC2F18074A2424FEAF1
:10B82000001C04DC63445C68A21A5A6003E06344B1
:10B830005A68A4185C60024B03EB0010816010BDD5
:10B84000400E0020012108B502200A46F9F740FA0F
:10B8500008BD00BFF8B51378144613F0600F064614
:10B860000D4627D1414A127B22BB13F0010F21D193
:10B870005F2B1FD83E4A1278E2B913F09F0301D024
:10B88000082B17D13B4F387860B9384BD97F19B1A5
:10B89000F9F708F9032304E00846597AF9F702F9A1
:10B8A00002233B70344F3B7823B10020FEF7B6FCF7
:10B8B00000233B70002221780220F9F709FA287052
:10B8C000002261780220F9F703FA68700022A1785B
:10B8D0000220F9F7FDF9A87001220220E178F9F7BA
:10B8E000F7F9E870237813F0010F3ED15F2B3CD8B5
:10B8F00003F01E02082A04D0142A2CD0062A34D1C0
:10B900001BE0242171435B090C2000FB0313A57885
:10B9100094F803C0194A4CEA05259D50A37813F00A
:10B92000080F22D02678760900FB0616B3586FEA76
:10B9300003536FEA1353B35017E0242256435B09B5
:10B940000C22A17802FB0363E27842EA01220B4950
:10B950005B185A6009E0242256435B090C2202FB63
:10B9600003630649E2785B181A72F8BDB80B002031
:10B97000280C0020200C00202C0C0020640B002040
:10B980002DE9F3414901CEB201AC46F0150317464B
:10B99000694622468DF804308046FFF75BFF9DF82C
:10B9A00001C09DF8033046F0140640466946224621
:10B9B0006D468DF804608DF805C08DF806708DF821
:10B9C0000730FFF747FFBDE8FC8100BF2DE9F341D9
:10B9D0004901CEB201AC46F015031746694622462E
:10B9E0008DF804308046FFF735FF9DF801C09DF8C3
:10B9F000023046F014064046694622466D468DF8F0
:10BA000004608DF805C08DF806308DF80770FFF7DB
:10BA100021FFBDE8FC8100BF37B541F001030C46B2
:10BA20006A4601A98DF800300546FFF713FF9DF81F
:10BA300006009DF8052000029DF8073040EA02400C
:10BA4000184310F4000F18BF40F07F405F2C1AD845
:10BA5000C4F3411314F01E0402D0022C13D106E0EB
:10BA6000032202FB0535084A2D01A8580BE00322EA
:10BA700002FB053520F07F41E8B2FFF7B5FE024B2F
:10BA800003EB051568683EBD400E002007B541F088
:10BA900001036A4601A98DF80030FFF7DBFE9DF82F
:10BAA00006009DF8073043EA002010F4006F1CBF29
:10BAB0006FEA00506FEA10500EBD00BF13B541F0A1
:10BAC0000103144601A96A468DF80030FFF7C2FE53
:10BAD0009DF805109DF806309DF807202170A27092
:10BAE00063709DF804001CBD07B5410141F01601CB
:10BAF00001F0F601002001AAFFF7E0FF9DF80530F4
:10BB0000D80913F0200F18BF40F002000EBD00BF8F
:10BB100007B5410141F0160101F0F601002001AA2C
:10BB2000FFF7CCFF9DF80530C3F3801013F0100F22
:10BB300018BF40F002000EBD37B50C4641EA401177
:10BB400001AA0546C9B20020FFF7B8FFB4235D4340
:10BB50006408032305F5807503FB04549DF8041065
:10BB60002046FCF727FD601C9DF80510FCF722FD20
:10BB7000A01C9DF80610FCF71DFD3EBD5F292DE9B8
:10BB8000F3410D460646144662D8C1F3411811F040
:10BB90001E0102D002295BD11EE0032202FB0088B5
:10BBA000344A4FEA081083185B688450E01A002872
:10BBB000B8BF4042B0F5000F0ADB9C42CCBF2E4C10
:10BBC0002E4C2C4A1C1902EB0812012313733FE080
:10BBD00002EB081211733BE0032707FB0087254B9C
:10BBE0003801C1587A00C4EB010C0132BCF1000FDE
:10BBF000B8BFCCF1000C00EB030EBCF5000F24F035
:10BC00007F40CEF8044043F832001DDBA142CCBF98
:10BC1000194B1A4B4FEA4818E3184FEA234E4FEAE4
:10BC2000232C3046694601AA8DF807308DF8048030
:10BC30008DF805E08DF806C0FFF70CFE0D4B03EB09
:10BC4000071701233B7303E003EBC20300221A71C1
:10BC50004FEA244C23123046694601AA8DF804505D
:10BC60008DF805C08DF806308DF80740FFF7F2FD1E
:10BC7000BDE8FC81400E0020FFFF7F00010080FF37
:10BC800038B50D4668210446FFF7C6FE15B140F0F1
:10BC9000010201E020F0010220466821FFF76EFF5B
:10BCA00038BD00BF07B513464FEA222C8DF80410AB
:10BCB0004FF0000E694601AA8DF805E08DF806C028
:10BCC0008DF80730FFF7C6FD0EBD00BF07B50B4668
:10BCD00011F01E01024601D0022905D11046194675
:10BCE0000022FFF74BFF0DE04FF0000C694601AA60
:10BCF0008DF804308DF807C08DF805C08DF806C0AA
:10BD0000FFF7A8FD0EBD00BF10B5C4B22146640107
:10BD100000200222E4B2FFF759FE002044F008019F
:10BD2000FFF7D4FF44F00A010020FFF7CFFF10BD5A
:10BD300007B59DF810C08DF804108DF805206946F0
:10BD400001AA8DF806308DF807C0FFF783FD0EBD00
:10BD500030B5430185B0044643F00303002003A936
:10BD600002AA8DF80830FFF775FD9DF80E109DF8BA
:10BD70000D209DF80F30090241EA02411943204687
:10BD8000FFF732FD174B03EB041108310A7932B388
:10BD9000154A0C2000FB0422107A00BB2201D518A2
:10BDA000D2586B68C3EB020CBCF1000FB8BFCCF1EA
:10BDB000000CBCF5000F05DB9A42CCBF0B4A0C4AC5
:10BDC0009A1800E008716101C2F30723D4B201F0B0
:10BDD000E0010020C2F307420094FFF7A9FF05B07D
:10BDE00030BD00BF400E0020640B0020FFFF7F002D
:10BDF000010080FF07B5937892F800E092F801C047
:10BE00008DF8041001AA69468DF805E08DF806C08A
:10BE10008DF80730FFF71EFD0EBD00BF37B544019A
:10BE200044F01604E4B20D4601AA21460020FFF7B3
:10BE300045FE9DF8053015F0010F1ABF6FEA436308
:10BE40006FEA536303F07F038DF805309DF80530EA
:10BE500015F0020F14BF43F0200323F020038DF8E8
:10BE6000053000231846214601AA8DF80630FFF759
:10BE7000C1FF3EBD37B5440144F01604E4B20D469F
:10BE800001AA21460020FFF719FE9DF8053015F0A4
:10BE9000010F14BF43F0400323F040038DF8053039
:10BEA0009DF8053015F0020F14BF43F0100323F086
:10BEB00010038DF8053000231846214601AA8DF89D
:10BEC0000630FFF797FF3EBD73B5B42545434B08D9
:10BED000032205F5807502FB0355044628460E46ED
:10BEE000FCF7D2FA8DF80400681CFCF7CDFA8DF847
:10BEF0000500A81CFCF7C8FA46EA44148DF80600B1
:10BF0000E1B2002001AAFFF775FF7CBD2DE9F74FD4
:10BF10004001C7B24C05002047F0180101AAFFF705
:10BF2000CDFD9DF80560640D06F00F053609B5429C
:10BF30000EDB204605F090F9AD1B80460120A8409D
:10BF4000894605F099F90022334B05F0FBF90FE023
:10BF5000204605F081F9751B80460120A8408946DE
:10BF600005F08AF902460B4600202B4905F014FB28
:10BF700002460B464046494605F00EFB05F0A4FC80
:10BF800005F08CF922A3D3E9002305F0DBF905F0D5
:10BF90009BFC05F083F90022204B05F0D3F94FF00C
:10BFA000FF36B046002582468B460120A84005F0AA
:10BFB00063F902460B465046594605F0C3F905F0B1
:10BFC0005BFCA0F180027F2A98BF2E46034605F154
:10BFD000010588BF43460E2D01D09846E5E70025B0
:10BFE00047F0120101AA28468DF805308DF8066049
:10BFF0008DF80450FFF7FEFE284647F00C0122465C
:10C00000FFF750FE2846BDE8FE8F00BFAFF300806B
:10C0100004560E2DB29DEF3F00006040000020400E
:10C0200013B5154B587E10F0010003D00020682195
:10C03000212201E0682120220024FFF79FFD2046F5
:10C040007E21202223460094FFF772FEE1B20020F9
:10C050000134FFF739FF1D2CF8D10C210020FFF728
:10C06000DBFC01460020FFF751FF0020162143F2C0
:10C07000FF12FFF717FE1CBD08000020AFF3008081
:10C08000084B1868034605E02C2A02D100221A70DA
:10C0900003E001331A78002AF6D1024A0133136013
:10C0A000704700BFDC04002010B50E4B02461B7821
:10C0B000ABB10D4B1C7994B19C68601CE4180D2A3F
:10C0C0002273986002D03F2800D851B9064C01462F
:10C0D00004F10C00FDF702FC0023A36001E0FCF773
:10C0E0005DFC10BD180B0020DC04002030B50121E0
:10C0F000044687B02020FFF7D7FF002C04DA2D205C
:10C100000121FFF7D1FF644200230A2194FBF1F2E1
:10C1100001FB124101AD3031E954591C141E01DDFF
:10C120000B46F2E7ED181C460121013C15F8010908
:10C13000FFF7BAFFB4F1FF3FF6D107B030BD00BF43
:10C1400038B50C4D0446A87801214030C0B2FFF745
:10C15000ABFF687801214030C0B2FFF7A5FF20781F
:10C16000FFF7C4FF6068FFF7C1FF0D200121FFF753
:10C170009BFF38BD0800002070B5124B06461B78A7
:10C18000EBB1FCF7D9FB104C054618B10023237125
:10C19000012016E0E36C226D934208D21A1992F83E
:10C1A0005420013301203270E364207109E004F16E
:10C1B0005400FDF761FBE5642065284601E0FCF7CB
:10C1C000BBFB70BD180B0020DC0400202DE9F341FF
:10C1D00004460DF10700FFF7CFFF002800F0CB80E9
:10C1E0008B4B8C4A93F8941019BB51789DF807003B
:10C1F000403188420DD1D3F89810002940F0BB801F
:10C200001179012231F0010183F8942040F0B380CC
:10C21000AFE00D2801D01B2802D100227C4B05E0A5
:10C22000D3F898207E2A00F2A6800132C3F8982025
:10C23000A1E0117931F0010103D19DF80700FFF76A
:10C2400033FF9DF807301F2B0BD9714AD2F8981095
:10C250007E297FD8481C891881F89C30C2F8980044
:10C2600078E0082B08D16A4BD3F89820002A71D0C7
:10C27000013AC3F898206DE00D2B6BD1644BD3F8D5
:10C280009830002B66D0634B1A79112A15D1587853
:10C2900001214030C0B2FFF707FF002503E0585DE1
:10C2A000FFF702FF01355A4B0121D3F898209C3348
:10C2B0009542F4D30D20FFF7F7FE554A0023156889
:10C2C000D2F8987019461A4633E001290FD002D3EC
:10C2D00002292DD122E04E4E06F19C00805C2028E0
:10C2E00026D09E1986F81C010133012120E0484820
:10C2F00000F19C0C1CF802C0BCF1200F0AD1012BEC
:10C3000004D91818002180F81C110133424D022174
:10C31000ED180DE0181880F81CC108E03C4E06F13D
:10C320009C00805C202803D09E1986F81C010133F4
:10C330000132BA42C9D3364A0021981880F81C113C
:10C340000120C2F89810156082F8A001C2F89C3153
:10C3500082F894109DF807301B2B0CD12D4A2C4BE2
:10C3600012790021012A83F89410C3F8981002D1A1
:10C370000D20FFF799FE264B93F8A001002878D0F6
:10C380000022164683F8A0211546DFF8A88007276B
:10C3900007FB058720483946013504F03BF930B9E1
:10C3A000BE797B7916F0010F237049D007E018F8A9
:10C3B00006300736002B5ED0FF2DE6D15BE0FFF79D
:10C3C0005FFE23780546042B0CD1144904F022F9B2
:10C3D0000346D8B12846124904F01CF970B128462A
:10C3E00010490FE00D2B28D10F4904F013F9034633
:10C3F00060B128460D4904F00DF908B9012305E0A4
:10C400000B49284604F006F9B0B90223637017E01F
:10C41000DC04002008000020F80500205129010854
:10C4200055290108592901085F29010865290108D2
:10C430006A29010848270108284604F0E5F86070D9
:10C4400016F0020F04D0FFF71BFE04F0DDF8A07019
:10C4500016F0040F0CD0FFF713FE04F0D5F8010E10
:10C46000C0F30722C0F30743A17122716371E0702A
:10C470000120BDE8FC8100232370F9E7704700BF6D
:10C48000FEE700BFFEE700BFFEE700BFFEE700BF1C
:10C49000704700BF704700BF704700BF704700BFC4
:10C4A000704700BF704700BF704700BF704700BFB4
:10C4B000704700BF704700BF704700BF704700BFA4
:10C4C000704700BF704700BF704700BF704700BF94
:10C4D000704700BF704700BF704700BF704700BF84
:10C4E000704700BF704700BF08B5024B1B689847F4
:10C4F00008BD00BF400B002008B5024B1B689847E1
:10C5000008BD00BF240C002008B5024B1B689847EB
:10C5100008BD00BFB40B002008B5024B1B6898474C
:10C5200008BD00BFD80B0020704700BF704700BF98
:10C53000704700BF704700BF704700BF704700BF23
:10C54000704700BF704700BF704700BF704700BF13
:10C55000704700BF704700BF704700BF704700BF03
:10C56000704700BF704700BF704700BF704700BFF3
:10C57000704700BF704700BF704700BF704700BFE3
:10C58000704700BF704700BF704700BF704700BFD3
:10C59000704700BF704700BF704700BF704700BFC3
:10C5A000704700BF704700BF704700BF704700BFB3
:10C5B000704700BF704700BF704700BF436830B589
:10C5C00023F470230C680A7923F48073234343EA2D
:10C5D0000223436082688D68CC680A4B45EA040CEC
:10C5E00002EA03034A794CEA030343EA4203836005
:10C5F0000B7CC26A013B22F47002DBB242EA0353B5
:10C60000C36230BDFDF7F1FF002301220274C36055
:10C610000360037143718360704700BF19B1836881
:10C6200043F0010302E0836823F001038360704755
:10C6300019B1836843F4807302E0836823F4807344
:10C6400083607047C9B212B14368194302E043687E
:10C6500023EA010141607047836843F00803836067
:10C66000704700BF8068C0F3C0007047836843F024
:10C6700004038360704700BF8068C0F38000704788
:10C6800019B1836843F4A00302E0836823F4A00394
:10C69000836070478068C0F38050704743680139F9
:10C6A00023F4604343EA41334360704719B1436860
:10C6B00043F4006302E0436823F40063436070477F
:10C6C000092930B511D94FF0030C0CFB01FC0725EB
:10C6D000ACF11E0C05FA0CF503FA0CFCC46824EA54
:10C6E000050343EA0C03C3600EE04FF0030C0CFBA0
:10C6F00001FC072505FA0CF503FA0CFC046924EA91
:10C70000050343EA0C030361062A0DD80523013A09
:10C710005A434FF01F0C0CFA02FC9140436B23EA82
:10C720000C020A4342631CE00C2A0DD805235A432D
:10C730004FF01F0C233A0CFA02FC9140036B23EAE2
:10C740000C020A4302630CE005235A434FF01F0C0E
:10C75000413A0CFA02FC9140C36A23EA0C020A43F4
:10C76000C26230BD19B1836843F4801302E083686C
:10C7700023F4801383607047C06C80B2704700BFA1
:10C78000014B1868704700BF4C24014019B1436841
:10C7900043F4806302E0436823F48063436070479E
:10C7A00019B1436843F4805302E0436823F4805393
:10C7B00043607047836823F4E04341EA03038360E6
:10C7C000704700BF19B1836843F4004302E08368F7
:10C7D00023F400438360704719B1836843F4021364
:10C7E00002E0836823F40213836070478068C0F31B
:10C7F00040507047092930B511D94FF0030C0CFB9C
:10C8000001FC0725ACF11E0C05FA0CF503FA0CFC33
:10C81000C46824EA050343EA0C03C3600EE04FF04A
:10C82000030C0CFB01FC072505FA0CF503FA0CFCC4
:10C83000046924EA050343EA0C030361836BC3F331
:10C84000015CCCEB020202324FF0050CD2B20CFBC1
:10C8500002F20CF11A0C0CFA02FC914023EA0C03D0
:10C860000B43836330BD00BF836B013923F4401356
:10C8700043EA0153836370470A5070472830405899
:10C8800080B27047436823F4400323F4007341EA05
:10C8900003034360704700BF41628262704700BF7C
:10C8A000436823F01F0341EA03034360704700BF5E
:10C8B00020B1054B9A6842F4000203E0024B9A68EB
:10C8C00022F400029A607047002401400368194274
:10C8D0000CBF002001207047C9430160704700BFB2
:10C8E0004368006810EA112004D0C9B219420CBF95
:10C8F00000200120704700BF6FEA112101607047DE
:10C9000008B5134B98420FD003F5A053984213D0AB
:10C91000A3F5C053984219D14FF40070012101F0E2
:10C920000BFB4FF400700EE04FF48060012101F02A
:10C9300003FB4FF4806006E04FF40040012101F05A
:10C94000FBFA4FF40040002101F0F6FA08BD00BFE9
:10C9500000280140374B01221A605A6812F0010288
:10C9600001D1104664E00278012A0BBF1A681A68E8
:10C9700042F0800222F080021A604378012B04D139
:10C980002C4B1A6842F0400203E02A4B1A6822F04E
:10C9900040021A608378012B04D1264B1A6842F0BA
:10C9A000200203E0234B1A6822F020021A60C378A9
:10C9B000012B04D11F4B1A6842F0100203E01D4BFB
:10C9C0001A6822F010021A600379012B04D1194B66
:10C9D0001A6842F0080203E0164B1A6822F00802B7
:10C9E0001A604379012B04D1124B1A6842F00402F9
:10C9F00003E0104B1A6822F004021A608279C379AE
:10CA000090F808C0920742EA03624189437A42EAF9
:10CA10000C4242EA03520139064B0A43DA611A68B2
:10CA200022F001021A60586880F0010000F0010055
:10CA3000704700BF0064004090F800C0012202FA75
:10CA40000CF23B4B2DE9F045D3F8004292B244F092
:10CA50000104C3F80042D3F81C42D14301EA0404A4
:10CA6000C3F81C428478A4B90CF1480CD3F80C72BA
:10CA7000B0F80AA0C688B0F8088085884FEACC04D0
:10CA800004F1804446EA0A4645EA084501EA0707F8
:10CA900015E0012C1AD10CF1480CD3F80C72B0F847
:10CAA00004A0C688B0F8088045894FEACC0404F198
:10CAB000804446EA0A4645EA084542EA070704F583
:10CAC000C844C3F80C7243F83C60656043782BB9E6
:10CAD000174BD3F8044201EA040404E0144BD3F8E2
:10CAE000044242EA0404C3F80442838923B9104B88
:10CAF000D3F81442214006E0012B06D10C4BD3F8A9
:10CB0000141242EA0101C3F81412837B012B05D1F0
:10CB1000074BD3F81C120A43C3F81C22044BD3F86A
:10CB2000002222F00102C3F80022BDE8F08500BF18
:10CB30000064004003220272013A002342724FF067
:10CB40000102C3714281037043708370C37003712B
:10CB500043718371704700BF19B1054B5A69104387
:10CB600003E0034B5A6922EA00005861704700BF96
:10CB700000640040364B70B59968024611F0806F32
:10CB800001D000200CE0996811F0006F01D0012065
:10CB900006E09B6813F0805F01D1042056E002207C
:10CBA0002B4B00F118010901CC5804F00104CC50C2
:10CBB000157A92F809C035B9146864051460CD5827
:10CBC0004CEA050C07E0546845EA0C0CE40054609C
:10CBD000CE584CEA060C4CEA0404CC50947A00F18E
:10CBE000180C4FEA0C1C04F00F040CF180439472F3
:10CBF00003F5C8435D68010125F00F055D605D68C0
:10CC000001F180412C435C60537B947BD57A1B04FB
:10CC100043EA0463147B2B4343EA042301F5C84130
:10CC2000C1F88831557C937CD47B2D0445EA03659B
:10CC3000137C45EA040242EA0322054BC1F88C2129
:10CC40005CF8032042F001024CF8032070BD00BFE5
:10CC500000640040012810D002D302282CD11AE031
:10CC6000164A91689368926801F0010103F002038B
:10CC700043EA8103C2F380621AE0104A9368916824
:10CC800003F48073926801F400719B0943EA112355
:10CC9000C2F3C0620CE0094A9368916803F48033E0
:10CCA000926801F400319B0B43EA1143C2F3007216
:10CCB0001343034AD05C70470023FAE70064004046
:10CCC00028280108012808D002D302280FD109E042
:10CCD000074B9A6842F0800208E0054B9A6842F4DC
:10CCE000004203E0024B9A6842F400029A607047E7
:10CCF0000064004018B9044B2022DA6002E0024BC5
:10CD000020221A61704700BF0064004010B9064B32
:10CD1000D86805E0012801D0002003E0024B186923
:10CD200000F00300704700BF00640040254B00F195
:10CD30001B02120110B5D45804F004040C721CB983
:10CD4000D3585B0D0B6002E0D358DB084B6000F159
:10CD50001B021C4B1201D35802F1804203F0020364
:10CD60004B7202F5C8425468030104F00F0C81F8BD
:10CD70000AC0526803F18043120ACA7403F5C8431B
:10CD8000D3F8B821CA72D3F8B821120A0A73D3F8BB
:10CD9000B821120C4A73D3F8B821120E8A73D3F853
:10CDA000BC21CA73D3F8BC21120A0A74D3F8BC217F
:10CDB000120C4A74D3F8BC311B0E8B74FFF79AFF28
:10CDC00010BD00BF00640040044B1A6842F002022C
:10CDD0001A601868C0F34000704700BF006400404C
:10CDE000054B1A6822F002021A60186880F00200EF
:10CDF000C0F34000704700BF00640040034B9B69D4
:10CE000018420CBF00200120704700BF00640040A2
:10CE1000024B9A6922EA00029A617047006400405E
:10CE2000202831D00CD8062820D004D8042825D0BA
:10CE3000052844D118E007281DD008283FD11FE05D
:10CE4000B0F5007F2BD005D840281FD0B0F5807FEB
:10CE500035D11FE0B0F5803F2CD0B0F5003F2BD08E
:10CE6000B0F5806F2BD11FE0012201E04FF48072FA
:10CE7000134B9A6023E04FF48032F9E7082200E078
:10CE800010220F4BDA601AE0082200E010220C4B4F
:10CE90001A6114E00A4B9A6922F0010208E0084B7B
:10CEA0009A6922F0020203E0054B9A6922F004021B
:10CEB0009A6104E0082200E01022014B5A6070479A
:10CEC0000064004001420CBF00200120704700BFF9
:10CED000202808B532D00CD8062821D004D8042840
:10CEE00026D0052818D119E007281ED0082813D10C
:10CEF00020E0B0F5007F29D005D8402820D0B0F53B
:10CF0000807F09D120E0B0F5803F27D0B0F5003F09
:10CF100022D0B0F5806F1BD0002024E0012101E079
:10CF20004FF48071104B98681BE04FF48031F9E7A3
:10CF3000082100E010210C4BD86812E0082100E025
:10CF40001021094B18690CE0012102E0022100E0E8
:10CF50000421054B986904E0102100E00821024BF0
:10CF60005868FFF7AFFF08BD00640040012108B515
:10CF70004FF0007000F0EEFF4FF00070002100F065
:10CF8000E9FF08BD0268002322F00102026003608D
:10CF900043608360C3602D4B984233D011D83C3B33
:10CFA000984229D006D8283B984221D01433984281
:10CFB0004BD11FE0264B984220D01433984244D1E5
:10CFC0001EE0244B98422CD008D8A3F567739842F2
:10CFD0001DD003F56273984237D11DE01E4B984275
:10CFE00029D0143398422BD0283B98422DD11DE0F4
:10CFF0001A4B12E0194B15E0184B18E0174B1BE0C9
:10D00000164B1EE0154B5A6842F470021CE0134B9D
:10D010005A6842F0706217E0114B5A6842F00F02F2
:10D0200012E00F4B5A6842F0F0020DE00C4B5A68C8
:10D0300042F4706208E00A4B5A6842F4704203E01E
:10D04000074B5A6842F470225A6070476C000240E5
:10D05000440002401C04024044040240000002401C
:10D06000000402408A6870B50C6A0B6944EA020247
:10D070004C691A438B692243CC6905684E6A42EABF
:10D08000030323438C6A334325F4FE4C23432CF0E3
:10D09000F00C43EA0C030360CB6843600B688360C9
:10D0A0004B68C36070BD00BF0023836203604360B0
:10D0B0008360C360036143618361C3610362436250
:10D0C000704700BF19B1036843F0010302E0036831
:10D0D00023F001030360704712B10368194302E0B3
:10D0E000036823EA01010160704700BF406880B215
:10D0F000704700BF10F0805F14BF044B044B1B68E7
:10D1000003420CBF00200120704700BF0004024012
:10D110000000024010F0805F14BF024B024B5860C9
:10D12000704700BF000402400000024010F0805F22
:10D1300014BF044B044B1B6803420CBF00200120AA
:10D14000704700BF000402400000024010F0805F02
:10D1500014BF024B024B5860704700BF00040240EE
:10D1600000000240044B00221A605A609A60DA60A4
:10D17000024A5A61704700BF00040140FFFF0700E8
:10D18000837930B5016802794BB3184BCC431D68E5
:10D1900090F805C004EA05051D605D682C405C60E0
:10D1A000D45844EA0101D15002689868D14301EA99
:10D1B00000009860D8680140BCF1100FD96007D119
:10D1C000996811439960D96841EA0202DA600BE07C
:10D1D0005CF8031041EA02024CF8032004E0034B20
:10D1E000D05820EA0101D15030BD00BF00040140F9
:10D1F00000230C228371427103600371704700BFEA
:10D20000024B1A6940EA02021A61704700040140A9
:10D21000034B5B6918420CBF00200120704700BF20
:10D2200000040140014B5861704700BF00040140F9
:10D23000054B1A685B69034001D1184603E01042B0
:10D240000CBF00200120704700040140014B5861D1
:10D25000704700BF00040140044B1A6802F0380216
:10D260001A601A6840EA02021A6070470020024001
:10D27000044B1A6822F008021A601A6840EA020297
:10D280001A60704700200240044B1A6822F0100216
:10D290001A601A6840EA02021A60704700200240D1
:10D2A000034B044A5A6002F188325A60704700BF4B
:10D2B0000020024023016745024B1A6942F08002B8
:10D2C0001A61704700200240014BD86980087047FE
:10D2D00000200240014B186A704700BF0020024046
:10D2E000024BD869C0F34000704700BF00200240E5
:10D2F000024B1868C0F34010704700BF0020024086
:10D3000019B1054B1A69104303E0034B1A6922EA6D
:10D3100000001861704700BF00200240012804D1BE
:10D32000054BD86900F0010005E0034BDB681842AB
:10D330000CBF00200120704700200240014BD86044
:10D34000704700BF00200240094BDA6812F0010F5D
:10D3500001D001200BE0DA6812F0040F01D00220A6
:10D3600005E0DB6813F0100F14BF032004207047A2
:10D370000020024013B504460AE000230193FF3366
:10D3800001E0019B013B0193019B002BF9D1013C82
:10D39000FFF7DAFF012802D1002CEED100E004B93A
:10D3A00005201CBDF8B5124C124B0546A36003F1D5
:10D3B00088330F20A3600E461746FFF7DBFF0428D3
:10D3C00014D1236945F0F80543F0100323612E437F
:10D3D000094B37430B305F80FFF7CCFF012805D0A6
:10D3E000226941F6EF7302EA03032361F8BD00BF2F
:10D3F000002002402301674500F8FF1F38B50546AD
:10D4000040F6FF70FFF7B6FF04283CD11E4C1F4BBF
:10D4100040F6FF70A36003F18833A360236943F0F3
:10D4200020032361236943F040032361FFF7A2FF38
:10D43000042820D1226941F6DF7302EA0303236145
:10D44000236943F0100323611DB1114B4FF000021B
:10D4500002E00F4B4FF0A5021A8040F6FF70FFF775
:10D4600089FF01280FD0084A41F6EF73116901EADC
:10D470000303136107E0012805D0226941F6DF7339
:10D4800002EA0303236138BD0020024023016745FF
:10D4900000F8FF1F10B504460F20FFF76BFF0428AC
:10D4A0003DD11F4A1F4BE443936003F188339360DF
:10D4B0001169E3B241F01001FF2B116106D01A4A45
:10D4C0000B301381FFF756FF04281FD1C4F3072345
:10D4D000FF2B06D0144A0F205381FFF74BFF04287F
:10D4E00014D1C4F30743FF2B06D00F4A0F209381BA
:10D4F000FFF740FF042809D1240EFF2C01D104209E
:10D5000006E0094B0F20DC81FFF734FF012806D02D
:10D51000034A41F6EF73116901EA0303136110BD79
:10D52000002002402301674500F8FF1F70B5044644
:10D530000F200E46FFF71EFF042815D10B4D0C4B94
:10D540000B30AB6003F18833AB602B6943F0100301
:10D550002B612680FFF70EFF012805D02A6941F6CE
:10D56000EF7302EA03032B6170BD00BF002002408D
:10D570002301674570B504460F200E46FFF7FAFEFB
:10D58000042810D1084D0B302B6943F001032B61A7
:10D590002680FFF7EFFE012805D02A6941F6FE73C9
:10D5A00002EA03032B6170BD0020024070B50446FF
:10D5B0000F200E46FFF7DEFE042818D10C4DB3B243
:10D5C0002A690B3042F001022A612380FFF7D2FE64
:10D5D000042804D1360C66800B30FFF7CBFE0128FF
:10D5E00005D02A6941F6FE7302EA03032B6170BD80
:10D5F0000020024010B540F6FF70FFF7BBFE042884
:10D600002CD1174C174B40F6FF70A36003F1883301
:10D61000A360236943F020032361236943F040039F
:10D620002361FFF7A7FE042810D1226941F6DF73BA
:10D6300002EA0303236123694FF0A50243F01003BC
:10D640002361094B0B301A80FFF794FE012805D0A7
:10D65000226941F6EF7302EA0303236110BD00BFA4
:10D66000002002402301674500F8FF1F10B540F677
:10D67000FF70FFF77FFE042814D10B4C40F6FF70BB
:10D68000236943F004032361236943F040032361CA
:10D69000FFF770FE012805D0226941F6FB7302EA0C
:10D6A0000303236110BD00BF0020024038B50546CA
:10D6B00040F6FF70FFF75EFE042815D10B4C40F6D4
:10D6C000FF70236943F0020323616561236943F01E
:10D6D00040032361FFF74EFE012805D0226941F681
:10D6E000FD7302EA0303236138BD00BF002002403E
:10D6F000CB78F0B513F0100F18BF8A78098803F0C3
:10D700000F0C18BF4CEA020C11F0FF0F1AD004687E
:10D7100000220126964006EA0105B5420ED1960088
:10D720000F27B7400CFA06F624EA07043443282BE7
:10D7300001D1456102E0482B08BF05610132082A8A
:10D74000E7D10460FF291CD94468002202F10805D2
:10D750000126AE4006EA0105B5420ED196000F271C
:10D76000B7400CFA06F624EA07043443282B01D10B
:10D77000456102E0482B08BF05610132082AE5D166
:10D780004460F0BD0423C370022383704FF0FF3365
:10D7900003807047836819420CBF00200120704746
:10D7A000806880B2704700BFC36819420CBF002078
:10D7B00001207047C06880B2704700BF01617047A8
:10D7C000416170470AB1016100E04161704700BFEB
:10D7D000C160704741F480338361816183618369F3
:10D7E00083697047064A10B514684FF6807341EAA2
:10D7F000001104EA030341EA0303136010BD00BFF4
:10D8000000000140014B1860704700BF1C0020421F
:10D810000304154A00F4401C1B0CBCF5401F30B536
:10D82000546806D1556824F0706425F07065556021
:10D8300011E010F4801F06D0C0F303424FF0030C38
:10D840000CFA02F203E0420D120113FA02F224EA8A
:10D85000020444F0706419B1400D000183401C4380
:10D86000014B5C6030BD00BF0000014001F00303CC
:10D870009B000F229A4010FA03F310B58908074C59
:10D88000023154F8210020EA020244F8212054F821
:10D890002120134344F8213010BD00BF0000014097
:10D8A0000120014608B500F047FB0120002100F0EF
:10D8B00043FB08BD08B5264B98422BD00CD8A3F5E6
:10D8C000006398421AD003F5806398421CD0A3F5F8
:10D8D000006398423AD10BE01E4B984226D003F5E4
:10D8E0008063984228D0A3F5006398422ED117E0B8
:10D8F0000420012100F020FB042024E00820012165
:10D9000000F01AFB08201EE01020012100F014FB9B
:10D91000102018E02020012100F00EFB202012E052
:10D920004020012100F008FB40200CE08020012174
:10D9300000F002FB802006E04FF48070012100F02F
:10D94000FBFA4FF48070002100F0F6FA08BD00BF2A
:10D9500000140140001C01400B4B4FF0FF316FF0F1
:10D960007042C3F88010C3F88420C3F88011C3F854
:10D970008421002303F1C001034A013300200F2B4F
:10D9800042F82100F6D1704700E100E0094B4FF06A
:10D9900020605860084800224FF0FF319A60D8603C
:10D9A0001A615A619A61DA611A625A629962D9629D
:10D9B0001963704700ED00E00000FA0540F0BE601A
:10D9C000024B40F42020D860704700BF00ED00E01B
:10D9D00030B5C27803787AB31C4A4178D2684FF0E8
:10D9E0000F0CD243C2F302222CFA02FCC2F1040251
:10D9F0009140807803F003020CEA000C4CEA010C21
:10DA0000D2004FEA0C1CFF2090400CFA02FC0124CB
:10DA100003F01F02944099080D4AC03152F821507A
:10DA20000CEA000C25EA00004CEA00005B0942F811
:10DA3000210042F8234008E003F01F020121914039
:10DA40005B09034A203342F8231030BD00ED00E0AB
:10DA500000E100E00023C3700370437083707047DF
:10DA6000024B5868C0F30930704700BF00ED00E07A
:10DA7000012200F01F0312FA03F34009044A403068
:10DA800052F820001840984214BF0020012070472F
:10DA900000E100E0014B1860704700BF00EF00E0BC
:10DAA00000F01F0301229A404009024B603043F806
:10DAB0002020704700E100E0024B58688005800D8F
:10DAC000704700BF00ED00E0012200F01F0312FAD2
:10DAD00003F34009044A803052F82000184098426D
:10DAE00014BF00200120704700E100E0014B1868DE
:10DAF000704700BF00ED00E021F0604121F07F01A0
:10DB0000014B01439960704700ED00E0014A024B70
:10DB1000DA6070470400FA0500ED00E0014A024BAC
:10DB2000DA6070470100FA0500ED00E019B1054B1D
:10DB30001A69104303E0034B1A6922EA00001861D6
:10DB4000704700BF00ED00E000F01F00012313FA52
:10DB500000F019B1044B5A6A104303E0024B5A6AB1
:10DB600022EA00005862704700ED00E0144B70B5E7
:10DB7000DC684FF0FF0CE443C4F302242CFA04F5F4
:10DB8000C4F1040411FA04F4C0F30126F6000CFAFF
:10DB900006FC02EA050545EA0404240114FA06F627
:10DBA000C0F38110063053F8202022EA0C0243F81B
:10DBB000202053F82020164343F8206070BD00BF9A
:10DBC00000ED00E0C0F3832001238340044A506A43
:10DBD00003EA0000984214BF00200120704700BFF4
:10DBE00000ED00E000F01F0001228240024B596866
:10DBF0000A435A60704700BF00ED00E000F01F02CA
:10DC00000123013A13FA02F2024B59680A435A609F
:10DC1000704700BF00ED00E0C0F383300123834074
:10DC2000044A506A03EA0000984214BF0020012011
:10DC3000704700BF00ED00E0C0F3814313B90A4B09
:10DC4000D86A10E0012B0CD1074AC0F30153906A47
:10DC5000DA00D040022B14BF00F00F0000F0FF00EC
:10DC600001E0014B186B704700ED00E010F4800FED
:10DC70000BBF024B014B586B986B704700ED00E0F7
:10DC800008B5F6F775FA08BD08B50001F6F76DFAA4
:10DC900008BD00BF08B5F6F766FA08BD08B5F6F787
:10DCA00060FA08BD08B5F6F75AFA08BD08B5F6F7E8
:10DCB00054FA08BD0D4B0E4A196841F00101196074
:10DCC000596801EA02025A601A6822F0847222F44A
:10DCD00080321A601A6822F480221A605A6822F48C
:10DCE000FE025A6000229A60704700BF0010024096
:10DCF0000000FFF80C4BB0F5803F1A6822F4803228
:10DD00001A601A6822F480221A6003D0B0F5802FBE
:10DD100008D103E01A6842F4803202E01A6842F443
:10DD2000A0221A60704700BF00100240034B1A681F
:10DD300022F0F80242EAC0021A6070470010024066
:10DD4000014B1860704700BF00004242044B5A6804
:10DD500022F47C1240EA02020A435A60704700BF74
:10DD600000100240014B1860704700BF6000424243
:10DD7000034B5A6822F0030240EA02025A607047DD
:10DD800000100240024B586800F00C00704700BFC2
:10DD900000100240034B5A6822F0F00240EA0202EF
:10DDA0005A60704700100240034B5A6822F4E06248
:10DDB00040EA02025A60704700100240034B5A6862
:10DDC00022F4605242EAC0025A60704700100240DA
:10DDD00019B1054B1A78104303E0034B1A7822EA75
:10DDE00000001870704700BF09100240014B186016
:10DDF000704700BFD8004242034B5A6822F44042A9
:10DE000040EA02025A60704700100240064B0022AE
:10DE100001281A701A7002D0042804D101E0187089
:10DE200001E005221A70704720100240014B186073
:10DE3000704700BF80044242024B1A6A40EA020265
:10DE40001A62704700100240014B1860704700BF13
:10DE50003C0442421F4B10B55A6802F00C02042ADF
:10DE600013D0082A11D15A685968C2F3834202328A
:10DE700011F4803F03D05B6813F4003F01D0164BD0
:10DE800000E0164B5A43026001E0144B0360114A54
:10DE9000134B51680468C1F30311595C34FA01F162
:10DEA00041605468C4F3022C13F80C4031FA04F4B6
:10DEB00084605468C4F3C22C13F80CC021FA0CF12E
:10DEC000C1605268C2F381329B181B7CB1FBF3F135
:10DED000016110BD0010024000093D0000127A00EF
:10DEE0003028010819B1054B5A69104303E0034B70
:10DEF0005A6922EA00005861704700BF00100240D2
:10DF000019B1054B9A69104303E0034B9A6922EA61
:10DF100000009861704700BF0010024019B1054B26
:10DF2000DA69104303E0034BDA6922EA0000D861A2
:10DF3000704700BF0010024019B1054BDA6810436A
:10DF400003E0034BDA6822EA0000D860704700BFA4
:10DF50000010024019B1054B1A69104303E0034B4E
:10DF60001A6922EA00001861704700BF00100240E1
:10DF7000014B1860704700BF40044242014B1860DB
:10DF8000704700BF4C004242014B1870704700BF01
:10DF9000071002404309012B02D1084B1B6805E022
:10DFA000022B0BBF054B054B1B6A5B6A00F01F0081
:10DFB00033FA00F000F00100704700BF001002408B
:10DFC00008B53120FFF7E6FF094B18705A68013297
:10DFD0005A601A7822B95A6840F2FF139A42F0D177
:10DFE0003120FFF7D7FF003818BF012008BD00BF60
:10DFF00080060020024B5A6A42F080725A627047D3
:10E0000000100240034B9B6818420CBF0020012007
:10E01000704700BF00100240014B1870704700BFEE
:10E020000A1002400B884A88B1F804C01A43CB8812
:10E0300042EA0C02B1F808C01A434B8930B542EAF3
:10E040000C028D89B0F800C0CC891A432A432243C0
:10E050000CF4415313439BB20380838B23F400637E
:10E060001B041B0C83830B8A038230BD00234FF0FB
:10E070000702C3810282038043808380C3800381BF
:10E0800043818381704700BF002343810380438025
:10E090008380C3804FF002030381704721B103885E
:10E0A0009BB243F0400304E0038823F040031B04C9
:10E0B0001B0C0380704700BF21B1838B9BB243F4DC
:10E0C000806304E0838B23F480631B041B0C838335
:10E0D000704700BF0909012313FA01F189B21AB18F
:10E0E00083889BB2194303E083889BB223EA010132
:10E0F000818070471AB183889BB2194303E08388FB
:10E100009BB223EA01018180704700BF8181704783
:10E11000808980B2704700BF4FF6FF63994205D0F7
:10E1200003889BB243F48073038002E003881940A4
:10E130000180704721B183889BB243F0040304E05F
:10E14000838823F004031B041B0C8380704700BFEB
:10E15000038823F400631B041B0C038003889BB219
:10E1600041EA03030380704703889BB243F4805362
:10E170000380704721B103889BB243F4005304E04D
:10E18000038823F400531B041B0C0380704700BF5B
:10E19000012914BF008B808A80B27047008A80B248
:10E1A000704700BFB1F5804F04D103889BB243F4A0
:10E1B000804304E0038823F480431B041B0C03808A
:10E1C000704700BF038919420CBF0020012070472F
:10E1D000202906D1038903889BB243F040030380C2
:10E1E00008E0402901D0082901D1038902E0C94390
:10E1F00089B20181704700BF012301F00F0213FAB9
:10E2000002F2B0F804C000891FFA8CFC80B2104002
:10E2100006D009098B401CEA030F0CBF0020012027
:10E22000704700BF552906D1038903889BB243F08C
:10E23000400303800DE0562901D0532901D1038901
:10E2400007E001F00F01012313FA01F1C94389B27C
:10E2500001817047838BF0B523F47A6323F01F03A9
:10E260001B041B0C83834FF0020303840B89868BF2
:10E27000022B87B004460D46B6B201D1002225E03C
:10E2800001A88F88FFF7E6FDEB88002F0CBF012760
:10E290000227B3F5007F2989019A06D1A3F5FB7304
:10E2A00053430902B3FBF1F305E00A2349015A4342
:10E2B0004F43B2FBF7F305330A229BB2B3FBF2F3F1
:10E2C00003F001021202C3F34F0392B2991E89B206
:10E2D000FE2928BF002228BF0223E98842EA03035F
:10E2E0000B439BB223842B886A8846EA0303A988E0
:10E2F00043F4006313436A890B4313439BB2A38324
:10E3000007B0F0BD08B5154B98421BD003F5744318
:10E31000984204D0A3F5784398421DD10AE0012128
:10E320004FF48050FFF708FE4FF480500021FFF7B4
:10E3300003FE11E04FF480400121FFF70BFE4FF484
:10E34000804006E04FF400400121FFF703FE4FF448
:10E3500000400021FFF7FEFD08BD00BF003C00406B
:10E36000042804D1054B1A6842F0040203E0034B71
:10E370001A6822F004021A60704700BF10E000E043
:10E38000014B5860704700BF10E000E0012804D145
:10E39000084B1A6842F0010206E010F1020F05D1A5
:10E3A000044B1A6822F001021A6002E0014B0022BD
:10E3B0009A60704710E000E020B1054B1A6842F007
:10E3C000020203E0024B1A6822F002021A60704750
:10E3D00010E000E0014B9868704700BF10E000E0DB
:10E3E000C308022B0BBF044B034B1B68DB6833FADB
:10E3F00000F000F00100704710E000E0038803F037
:10E400008F0303800388B1F806C04A889BB243EAB1
:10E410000C0313439BB203808B8883850B88038591
:10E42000064B984203D003F50063984201D10B7A62
:10E4300003864FF001038382704700BF002C014028
:10E44000038C2DE9F04123F001031B041B0C038412
:10E45000038C0A894C8823F002031C4E14431B04CE
:10E460008288B1F806C0058B1B0CA4B2B04244EA06
:10E47000030392B20C88ADB2A0F834C003D006F505
:10E480000066B04218D18E894F89B1F80E804FF6E0
:10E49000F77C03EA0C0C4CEA070748EA06064FF63D
:10E4A000FB73898847F6FF4C02EA0C0C07EA03036A
:10E4B000B2B20B4342EA0C024FF68F7105EA01013A
:10E4C0002143828001830384BDE8F081002C014058
:10E4D000038C2DE9F04123F010031B041B0C038473
:10E4E000028CB1F808C022F0200212048488120CB9
:10E4F0004B8842EA0C1242EA0313A2B21B4C068B71
:10E50000B1F806C0A0420D88B6B29BB2A0F838C0E0
:10E5100003D004F50064A0421BD1B1F80A804FF685
:10E520007F748F8903EA040447F2FF3C02EA0C0C73
:10E5300044EA0814CA894FF6BF73898804EA0303C2
:10E540004CEA870C43EA01134CEA82023C469BB238
:10E5500092B248F6FF7106EA010141EA052189B24B
:10E56000828001830384BDE8F08100BF002C01405C
:10E57000038C2DE9F04123F480731B041B0C0384EE
:10E58000028CB1F808C022F4007212048488120CC4
:10E590004B8842EA0C2242EA0323A2B21A4C868B31
:10E5A000B1F806C0A0420D88B6B29BB2A0F83CC03C
:10E5B00003D004F50064A0421BD1B1F80A804FF2E9
:10E5C000FF748F8903EA040444F6FF7C02EA0C0C12
:10E5D00044EA0824CA894FF6FF33898804EA030312
:10E5E0004CEA071C43EA01234CEA02123C469BB268
:10E5F00092B24FF68F7106EA01012943828081832E
:10E600000384BDE8F08100BF002C0140038CF0B50D
:10E6100023F480531B041B0C0384B1F806C0078C41
:10E620000C8882880D89868B4B88A0F840C0DFF863
:10E6300048C0BFB2604592B2B6B203D00CF5006CD0
:10E64000604505D192048989920C42EA811292B206
:10E650004DF6FF7C07EA0C0C48F6FF7106EA010153
:10E660004CEA053C41EA04214CEA033389B29BB2EF
:10E67000828081830384F0BD002C0140B1F802C088
:10E680000B888A884CEA0303B1F806C013430A8951
:10E6900043EA0C03B1F80AC013438A8943EA0C0326
:10E6A00013439BB2A0F84430704700BF00234FF0E3
:10E6B000FF320372438082800380C380704700BFB3
:10E6C0000023C381038043808380C380038143810F
:10E6D0008381704700234FF0010203810380438050
:10E6E0008280C380704700BF002383810380438002
:10E6F0008380C38003814381704700BF21B10388B9
:10E700009BB243F0010304E0038823F001039B055F
:10E710009B0D0380704700BF39B1B0F844306FEAF9
:10E7200043436FEA53439BB203E0B0F844305B04C9
:10E730005B0CA0F8443070471AB183899BB219432F
:10E7400003E083899BB223EA01018181704700BF06
:10E75000818270470A43A0F8482070471AB1838924
:10E760009BB2194303E083899BB223EA01018181B3
:10E77000704700BF038923F007031B041B0C0381B0
:10E78000704700BFB0F808C05FFA8CFC41EA0C0C7F
:10E7900042EA0C0C4CEA032C1FFA8CFCA0F808C0CF
:10E7A000704700BF10B50446FFF7ECFF23899BB20A
:10E7B00043F48043238110BD10B50446FFF7E2FF08
:10E7C000238923F077031B041B0C43F07703238179
:10E7D00010BD00BF01858282704700BF038823F00F
:10E7E00070039B059B0D41EA03030380704700BF44
:10E7F000038923F070031B041B0C41EA030303810C
:10E80000704700BF10B50446FFF7F2FF23899BB2A3
:10E8100043F00703238110BD30B50489B0F818C058
:10E82000058C2CF4407CADB22CF0030C24F00704D2
:10E830004FEA0C4C25F0220542EA050524044FEA74
:10E840001C4C45EA0315240C4CF4807C21434CF00D
:10E85000010CADB20181A0F818C0058430BD00BF25
:10E86000038B23F070031B041B0C41EA0303038397
:10E87000704700BF038B23F4E0431B041B0C43EAE7
:10E8800001239BB203837047838B23F070031B0427
:10E890001B0C41EA03038383704700BF838B23F47F
:10E8A000E0431B041B0C43EA01239BB283837047A4
:10E8B00021B103889BB243F0800304E0038823F076
:10E8C00080039B059B0D0380704700BF21B18388A7
:10E8D0009BB243F0040304E0838823F004031B0489
:10E8E0001B0C8380704700BF21B183889BB243F02B
:10E8F000080304E0838823F008031B041B0C8380B7
:10E90000704700BF21B183889BB243F0010304E04C
:10E91000838823F001031B041B0C8380704700BF16
:10E92000038B23F008031B041B0C41EA030303833E
:10E93000704700BF038B23F400631B041B0C43EAE6
:10E9400001239BB203837047838B23F008031B04CE
:10E950001B0C41EA03038383704700BF838B23F4BE
:10E9600000631B041B0C43EA01239BB283837047A3
:10E97000038B23F004031B041B0C41EA03030383F2
:10E98000704700BF038B23F480631B041B0C43EA16
:10E9900001239BB203837047838B23F004031B0482
:10E9A0001B0C41EA03038383704700BF838B23F46E
:10E9B00080631B041B0C43EA01239BB283837047D3
:10E9C000038B23F080031B041B0C41EA0303038326
:10E9D000704700BF038B5B045B0C43EA01239BB2CF
:10E9E00003837047838B23F080031B041B0C41EAD5
:10E9F00003038383704700BF838B5B045B0C43EA94
:10EA000001239BB283837047038C23F002031B0412
:10EA10001B0C41EA03030384704700BF038C23F0FF
:10EA200008031B041B0C41EA03030384704700BF67
:10EA3000038C23F020031B041B0C43EA01139BB23D
:10EA400003847047038C23F080031B041B0C43EAF0
:10EA500001139BB203847047038C23F400731B04DF
:10EA60001B0C43EA01239BB203847047038C23F4FD
:10EA700000631B041B0C43EA01239BB20384704711
:10EA8000038C23F400531B041B0C43EA01339BB299
:10EA90000384704701238B408A40018C89B221EAAC
:10EAA00003030384018C0A4392B20284704700BFBF
:10EAB00004238B408A40018C89B221EA030303843A
:10EAC000018C0A4392B20284704700BF01238B403D
:10EAD000B0F820C010B51FFA8CFC2CEA03030384A5
:10EAE00009B1082909D11830490844584FF68F73E5
:10EAF00004EA0303435043580CE004391830C1F3CF
:10EB00004E01445848F6FF7304EA030343501202CF
:10EB1000435892B243EA0202425010BD21B1038829
:10EB20009BB243F0020304E0038823F002039B0539
:10EB30009B0D0380704700BF21B103889BB243F057
:10EB4000040304E0038823F004039B059B0D03806A
:10EB5000704700BF21B183889BB243F0800304E07B
:10EB6000838823F080031B041B0C8380704700BF45
:10EB7000038823F008039B059B0D038003889BB249
:10EB800041EA030303807047838823F070031B046A
:10EB90001B0C838083889BB241EA03038380704708
:10EBA000038923F007031B041B0C038103899BB219
:10EBB00041EA030303817047038923F080031B04A8
:10EBC0001B0C038103899BB241EA03030381704755
:10EBD00081847047818570478186704701877047BF
:10EBE00081877047A0F84010704700BF038B23F067
:10EBF0000C031B041B0C0383038B9BB241EA03032E
:10EC000003837047038B23F440631B041B0C0383B3
:10EC1000038B9BB243EA01239BB20383704700BF7F
:10EC2000838B23F00C031B041B0C8383838B9BB20D
:10EC300041EA030383837047838B23F440631B04FF
:10EC40001B0C8383838B9BB243EA01239BB2838398
:10EC5000704700BF0388DBB2038003889BB241EAA0
:10EC600003030380704700BF808E80B2704700BFEF
:10EC7000008F80B2704700BF808F80B2704700BFA6
:10EC8000B0F8400080B27047808C80B2704700BFFF
:10EC9000008D80B2704700BF038A19420CBF00206C
:10ECA00001207047C94389B201827047038A828973
:10ECB00011EA030092B203D011420CBF00200120E0
:10ECC000704700BFC94389B201827047B0F820C0C5
:10ECD00010B52CF0010C4FEA0C4C4FEA1C4CA0F87C
:10ECE00020C0048BB0F820C0A4B21FFA8CFC24F022
:10ECF000F30442EA04042CF0020C44EA03144CF03E
:10ED0000010C4CEA010CA4B20483A0F820C010BD91
:10ED1000B0F820C010B52CF0100C4FEA0C4C4FEAA4
:10ED20001C4CA0F820C0B0F818C0048C2CF4407C17
:10ED3000A4B24FEA0C5C4FEA1C5C24F020044CEABD
:10ED4000022C44F010044CEA033C44EA01141FFA7C
:10ED50008CFCA4B2A0F818C0048410BD38B50D46D0
:10ED6000602D1146044603D10122FFF7D1FF02E0D6
:10ED70000122FFF7ABFF29462046FFF739FD238923
:10ED80009BB243F00703238138BD00BFF8B50C46A2
:10ED9000A2884988B4F800C0054600290CBF0227A4
:10EDA0000027012A0CBF022601262389BCF1000F8F
:10EDB00010D1FFF78BFF2846E188FFF717FF2846A1
:10EDC000394632462389FFF7A3FF2846E188FFF73B
:10EDD00019FF0FE0FFF79CFF2846E188FFF712FFBD
:10EDE0002846394632462389FFF770FF2846E188D6
:10EDF000FFF7FCFEF8BD00BF38B50B880C46054692
:10EE00004BB94988A2882389FFF760FF2846E1882B
:10EE1000FFF7ECFE53E0042B09D14988A28823892F
:10EE2000FFF776FF2846E188FFF7ECFE47E0082B66
:10EE3000B1F802C0B1F804E0098920D1028C22F4B3
:10EE400080721204120C0284838B028C9BB292B2E9
:10EE500023F0F30322F4007243EA011142EA0C2C7E
:10EE600089B21FFA8CFC41EA0E0E4CF4807CA0F8AB
:10EE70001CE0A0F820C0E188FFF7D2FE1FE0028C62
:10EE800022F480521204120C0284838B028C23F42D
:10EE9000407392B21B051B0D22F4005243EA0E236D
:10EEA00042EA0C3C43EA01331FFA8CFC9BB24CF45F
:10EEB000805C8383A0F820C0E188FFF7BDFE38BDE9
:10EEC00008B52D4B984237D00BD8A3F50063984274
:10EED00026D003F58063984228D0B0F1804F4AD104
:10EEE00018E0264B984233D004D8A3F580639842AB
:10EEF00041D127E0224B984204D003F500639842A9
:10EF000039D12EE04FF400600121FFF715F84FF4DE
:10EF100000602DE001200146FFF71CF801201CE0F5
:10EF200002200121FFF716F8022016E0042001213B
:10EF3000FFF710F8042010E008200121FFF70AF87D
:10EF400008200AE010200121FFF704F8102004E057
:10EF500020200121FEF7FEFF20200021FEF7FAFF0E
:10EF600009E04FF400500121FEF7E6FF4FF4005096
:10EF70000021FEF7E1FF08BD000C00400014004036
:10EF8000002C0140002383814FF416528380C380FC
:10EF900003814FF00C030260438170470A8810B56B
:10EFA0004C88B1F804C0038AC98844EA020242EAE4
:10EFB0000C0223F470630A431B041B0C92B242EA56
:10EFC0000303038210BD00BF0023C380038043807E
:10EFD0008380704721B183899BB243F4005304E0DE
:10EFE000838923F400531B041B0C8381704700BFEB
:10EFF00001F01F034FF0010CC1F3421161450CFAFF
:10F0000003F301D10C3004E0022901D1103000E0FB
:10F0100014301AB1026842EA030302E0026822EAED
:10F0200003030360704700BF1AB1838A9BB2194380
:10F0300003E0838A9BB223EA01018182704700BF0B
:10F04000038A23F00F031B041B0C0382038A9BB269
:10F0500041EA030303827047838923F400631B049E
:10F060001B0C838183899BB241EA03038381704730
:10F0700021B183899BB243F0020304E0838923F02A
:10F0800002031B041B0C8381704700BF038A23F01B
:10F0900020031B041B0C0382038A9BB241EA030377
:10F0A0000382704721B1038A9BB243F4804304E09A
:10F0B000038A23F480431B041B0C0382704700BFA8
:10F0C000C905C90D818070478088C005C00D704793
:10F0D00083899BB243F0010383817047038BDBB2CA
:10F0E0000383038B9BB243EA01230383704700BF72
:10F0F000038B03F47F430383038B9BB241EA030337
:10F100000383704721B1838A9BB243F0200304E05C
:10F11000838A23F020031B041B0C8382704700BFEB
:10F1200021B1838A9BB243F0100304E0838A23F069
:10F1300010031B041B0C8382704700BF21B1838A1C
:10F140009BB243F0080304E0838A23F008031B0406
:10F150001B0C8382704700BF838A23F004031B04C7
:10F160001B0C8382838A9BB241EA0303838270472C
:10F1700021B1838A9BB243F0020304E0838A23F027
:10F1800002031B041B0C8382704700BF03881942D3
:10F190000CBF002001207047C94389B2018070472D
:10F1A0004FF0010CC1F3421201F01F0362450CFA4B
:10F1B00003F301D1828903E0022A0CBF028A828A0A
:10F1C00092B21340028892B20BB9184607E0090ABE
:10F1D000012313FA01F111420CBF002001207047F6
:10F1E000090A01238B40DB439BB20380704700BFB9
:10F1F000038ACA8823F440531B041B0C1343038265
:10F2000083898A8830B5044608890D4623F4B053B3
:10F21000498940EA020223F00C030A431B041B0C39
:10F2200092B242EA0303A381A38AAA8923F440731A
:10F230001B041B0C134387B0A38201A8FEF70AFE30
:10F240000E4B2A689C420CBF049B039B1921594317
:10F2500092006423B1FBF2F1B1FBF3F21201100949
:10F2600003FB101109013231B1FBF3F303F00F037B
:10F2700043EA020292B2228107B030BD0038014059
:10F2800008B5214B98422BD008D8A3F500639842CB
:10F2900016D003F58063984234D119E01B4B984295
:10F2A00026D003F5684398422CD101214FF48040C9
:10F2B000FEF742FE4FF480400021FEF73DFE21E0C4
:10F2C0004FF400300121FEF745FE4FF4003016E008
:10F2D0004FF480200121FEF73DFE4FF480200EE028
:10F2E0004FF400200121FEF735FE4FF4002006E028
:10F2F0004FF480100121FEF72DFE4FF48010002105
:10F30000FEF728FE08BD00BF004C00400050004042
:10F31000684620F007018D4601B5002303E00B4944
:10F320005958995004330A4A0A4998188842F6D322
:10F33000094B02E0002243F8042B084A9342F9D318
:10F34000F4F74AFFBDE80140854670478829010867
:10F35000000000203002002030020020580E002063
:10F3600010B5074C20B922684FF00103138205E065
:10F37000044B1B681B68984720680A3010BD00BF0B
:10F38000F00D0020AC0D002010B50A4B0A4A1B6896
:10F390005178DA7891420AD3997841B99C8834B986
:10F3A0009A72064B1B685B689847204600E0022073
:10F3B00010BD00BFF00D002004010020AC0D0020A6
:10F3C00010B5074C20B922684FF00103138205E005
:10F3D000044B1B689B68984720680C3010BD00BF29
:10F3E000F00D0020AC0D002038B50E4C0E4B2268FD
:10F3F0001B68D1789B695079984723689A7A7AB1CB
:10F4000070B91A7962B99D7855B9084B1B68DB68E9
:10F410009847236828465979DA78D9721A7300E038
:10F42000022038BDF00D0020880D0020AC0D00201A
:10F4300008B50246244B20B91B684FF0020119821F
:10F4400040E0224A4FF000011B681180197811F04A
:10F450007F0113D15B7A13F0200F03D0117841F0B4
:10F460000201117013F0400F184B15BF1A781A786B
:10F4700022F0010242F001021A701EE0012921D09F
:10F48000022901D000221DE0597911F0800F01F00E
:10F490000F0306D00E4951F8233003F03003102B30
:10F4A00006E00B4951F8233003F44053B3F5805F75
:10F4B00003D1137843F001031370064B1B681B69DB
:10F4C0009847024A104608BDF00D0020500E00205B
:10F4D000005C0040AC0D002010B51E4B19684A7945
:10F4E00012F0800F22F0800305D01B4850F8230053
:10F4F00000F0300004E0184850F8230000F44050B9
:10F50000164C94F800C0634522D24C8804BBF8B175
:10F51000897AE9B112F0800F09D00F4948F6BF721D
:10F5200051F8230000EA020282F0100208E00A49C2
:10F530004BF68F7251F8230000EA020282F48052E7
:10F5400041F82320064B1B689B699847002000E088
:10F55000022010BDF00D0020005C004004010020DE
:10F56000AC0D002008B5064B1B685A7A42F0200209
:10F570005A72044B1B68DB699847002008BD00BF26
:10F58000F00D0020AC0D0020054B1A68538A18B905
:10F590008988CB1A138201E008681818704700BFE9
:10F5A000F00D002030B50E4B1C78002310E05FFA00
:10F5B00083FC4FEA8C0202F1804202F5B8421568E2
:10F5C00048F68F7105EA010141EA0C01116001332F
:10F5D000A342ECD3034B40F08000186030BD00BF65
:10F5E000040100204C5C0040704700BF08B50C4B84
:10F5F000002093F82C1000F04FFE0A4B1B68187A7D
:10F60000082807D1084B4FF480521A80074B4FF05F
:10F6100010021A80092814BF0020012008BD00BF75
:10F6200080000020F00D0020520E0020540E00201B
:10F6300070B52D4B1C68237A032B01D0052B46D1C6
:10F64000A369228AABB1A2B1A58A954228BF15460B
:10F6500028469847228A638A521BEB180646228264
:10F660006382002000F0E8FD2A460146304600F0A3
:10F67000FBFB238A5BB11D4B4FF4405200201A80E4
:10F68000014600F0E7FD1A4B4FF030021A80A28AC3
:10F69000238A9A4203D8144B03221B6803E0124AC0
:10F6A0001BB1136805221A720DE01268062111724F
:10F6B000104A1168104A89B28A18520013600C4B24
:10F6C0004FF030021A80084B1B681B7A06E0072BAC
:10F6D00003D10A4B1B68DB6898470823024A12686B
:10F6E0001372FFF783FF70BDF00D0020520E002053
:10F6F000540E0020505C004002300020880D002095
:10F70000F8B5244B1C68238A267ABBB9042E15D180
:10F71000214822490278012A0BD1214C214A246830
:10F720000370A0B28218520013604FF030020A80BA
:10F730002BE04FF010030B80072626E0A68AA26973
:10F740009E4234BF35461D462846B34294BF042628
:10F75000022690470746002000F060FD2A46014639
:10F76000384600F069FB2946002000F073FD638AEB
:10F77000228AEB186382094B551B4FF03002258219
:10F780001A80094B4FF440521A80024B1B681E72BC
:10F79000F8BD00BFF00D002088060020540E0020A8
:10F7A000505C004002300020520E002008B5144B7F
:10F7B0001B681A7A022A01D0042A05D1FFF7A0FF9C
:10F7C0000F4B1B681B7A14E0062A11D15A78052AC0
:10F7D0000AD11A7812F07F0F06D1D878FFF7E2FE2F
:10F7E000084B1B681B6A9847074B1B689B68984728
:10F7F0000823034A12681372FFF7F8FE08BD00BF22
:10F80000F00D0020AC0D0020880D002038B5324BE3
:10F810001B68187810F07F0004D15A7A22F0200279
:10F820005A7258E0022855D15A88002A52D11A79C2
:10F83000002A4FD15A7912F0800F22F0800405D0AF
:10F84000264951F8241001F0300104E0234951F811
:10F85000241001F440512248007884423AD2002911
:10F8600038D09B7A002B35D012F0800F0FD01B4B75
:10F8700053F8243003F03003102B25D1E4B2204696
:10F8800000F082FC2046302100F05EFB1CE0134DAE
:10F8900055F8243003F44053B3F5805F14D134B9E4
:10F8A000104B204693F82C1000F0F6FC02E02046A6
:10F8B00000F056FC55F824204BF68F7302EA030340
:10F8C00083F4405345F82430074B1B685B69984725
:10F8D000002000E0022038BDF00D0020005C004058
:10F8E0000401002080000020AC0D0020F7B58D4BF6
:10F8F0008D4E1A6835688D4B92B2D3182A7A5B0008
:10F90000092A1B681BD09BB203F1005303F5405337
:10F910005B001C4614F8012B03F10A072A705B7880
:10F920006B70B4F8030000F063FE6880B4F8070061
:10F93000346800F05DFEA08033687F88DF807A4CF9
:10F9400001212368DA8819725D78002A62D11A7859
:10F9500012F07F022ED1092D02D1FFF715FD3BE0F9
:10F96000052D0DD193F90320002A4EDB9A78002A49
:10F970004BD19A88002A48D19B7A002B37D044E09B
:10F98000032D0BD1DA78012A27D19A882ABB5B7A1A
:10F9900013F0200F21D0FFF7E5FD1DE0012D1CD154
:10F9A000DA78012A19D19A88BAB95B7A13F0200F54
:10F9B00013D00AE0012A04D10B2D0ED1FFF714FD5C
:10F9C0000AE0022A09D1012D02D1FFF71FFF03E04F
:10F9D000032D02D1FFF780FD48B1554B28461B6827
:10F9E0005B699847032801D109230FE068B94D4AA4
:10F9F000504B12684FF0300192B2D3185B000022D6
:10FA00001A604D4B1980062300E00823464A12680D
:10FA10001372E3E0062D18D11A7812F07F0F40F030
:10FA200097809B78012B03D1414B1B68DB696EE00B
:10FA3000022B03D13E4B1B681B6A68E0032B40F08E
:10FA400087803B4B1B685B6A61E0002D3CD1598885
:10FA500000297DD15A6822F47F42B2F5003F77D168
:10FA60001A7812F07F0203D19B88002B70D129E015
:10FA7000012A0BD158792E4B1B689B6998470028A7
:10FA800066D123689B7A002B62D01BE0022A5FD1EB
:10FA90005B7913F0800F03F00F0205D0274951F86E
:10FAA000221001F0300104E0244951F8221001F441
:10FAB00040512348007882424AD213F0700F47D158
:10FAC000002945D01F4B23E0082D05D11B7813F0EA
:10FAD0007F0F3DD11C4B1BE00A2D39D11A7802F063
:10FAE0007F02012A34D19A7A002A31D0598800291C
:10FAF0002ED15A6822F47F42B2F5803F28D158793E
:10FB00000B4B1B689B69984710BB104B00E0FBB187
:10FB1000054A4FF000011268002093615182984716
:10FB2000002020E0505C0040F00D00200430002058
:10FB3000880D002002300020540E0020005C0040A0
:10FB40000401002031F4000861F30008C1F300084B
:10FB5000244C254B22681B6850781B699847032862
:10FB600001D1236806E01F4B4FF6FF711B681A8A0C
:10FB70008A4201D1092203E0022800D012B90822EA
:10FB80001A722BE093F90010002921DAD98801912B
:10FB90000198824202D9019A1A8211E08A420FD258
:10FBA0001149096891F82C108A4201D2002105E020
:10FBB00092FBF1F001FB102212B901210B4A1170E6
:10FBC000094A126892F82C209A82FFF799FD05E005
:10FBD00003221A72064B4FF440521A80FFF706FDBB
:10FBE000FEBD00BFF00D0020880D0020880600201B
:10FBF000520E0020074A022108B507481172074932
:10FC0000074B086007490A60074A13601B6898475A
:10FC100008BD00BF900D002008010020AC0D0020A1
:10FC200080000020F00D0020880D002008B529E09C
:10FC300047F6FF700860198801F00F018B0003F18F
:10FC40008043117003F5B843196889B211F4004F6D
:10FC500009D0186840F68F7100EA01011960127826
:10FC60000E4B013A0BE011F0800F0BD0186848F6EC
:10FC70000F7100EA010119601278094B013A53F83B
:10FC8000223098470749084B0868084A80B2188014
:10FC9000188800B20028CBDB08BD00BFE8000020B8
:10FCA000CC000020445C0040860D00208C0D00201C
:10FCB000F8B59AE047F6FF761E601688564F06F0B4
:10FCC0000F06B30003F1804303F5B8433E70002EE6
:10FCD00064D127682668236807F4405C03EA0000C3
:10FCE00080F400502060236806F0300003EA010130
:10FCF00081F0200121601388484A13F0100F108012
:10FD0000A5F800C004D023689BB213F0800F08D080
:10FD1000226848F60F7302EA03032360FFF746FDEB
:10FD200016E013F4006F08D0226840F68F7302EAE1
:10FD300003032360FFF7DAFD0AE013F4004F54D009
:10FD4000226840F68F7302EA03032360FFF770FC1A
:10FD500021682A884BF68F7301EA030312F4805F4F
:10FD600018BF83F4805312F4005F2D4A18BF83F448
:10FD700000531360294B11681A8848F6BF7301EAD3
:10FD8000030312F0100F18BF83F0100312F0200FBE
:10FD9000234A18BF83F0200313603BE01C68A4B221
:10FDA00014F4004F0BD0196840F68F7201EA02027A
:10FDB0001A603A781B4B013A53F82230984714F0F6
:10FDC000800F12D0144948F60F720B789B0003F194
:10FDD000804303F5B843186800EA02021A600A7803
:10FDE000114B013A53F822309847104B104A1D68C6
:10FDF0000B4C1FFA85FCA2F800C0B2F800C04BF60D
:10FE00008F700FFA8CFCBCF1000F48F6BF71094DE2
:10FE1000FFF650AFF8BD00BF8C0D0020540E00203F
:10FE2000005C0040E8000020CC000020445C004062
:10FE3000860D0020520E002001F10051013201F523
:10FE4000405110B549005208002308E010F803C0E3
:10FE50006478013A4CEA042C21F813C00233C41828
:10FE6000002AF3D110BD00BF01F10051013201F5AC
:10FE7000405110B549005208002304E031F8134006
:10FE8000013AC4520233002AF8D110BD014B186068
:10FE9000704700BF405C0040014B186880B270475B
:10FEA000405C0040014B1860704700BF445C00405C
:10FEB000014B186880B27047445C0040014B1868E1
:10FEC00080B27047485C0040014B1860704700BF2B
:10FED0004C5C0040014B186880B270474C5C00409D
:10FEE0004FF6F873024A00EA03031360704700BF3D
:10FEF000505C0040014B186880B27047505C004075
:10FF0000014B43F820107047005C0040024B53F84F
:10FF1000200080B2704700BF005C0040054B10B568
:10FF200053F8204048F68F1204EA02020A4343F8CD
:10FF3000202010BD005C0040024B53F8200000F46C
:10FF4000C0607047005C00400A4B10B553F8202099
:10FF500048F6BF7402EA040411F0100F18BF84F0D1
:10FF6000100411F0200F18BF84F0200443F8204043
:10FF700010BD00BF005C00400A4B10B553F82020B4
:10FF80004BF68F7402EA040411F4805F18BF84F406
:10FF9000805411F4005F18BF84F4005443F82040EB
:10FFA00010BD00BF005C004038B50D460446FFF7A9
:10FFB000ADFF012D02D120F4805003E0022D04D1C9
:10FFC00020F01000014B43F8240038BD005C0040D5
:10FFD000024B53F8200000F030007047005C0040F6
:10FFE000024B53F8200000F440507047005C004082
:10FFF000054B48F6BF7253F8201001EA020282F066
:020000040801F1
:10000000300243F820207047005C0040054B4BF65F
:100010008F7253F8201001EA020282F4405243F832
:1000200020207047005C0040054B48F68F6253F873
:10003000201001EA020242F4807243F82020704747
:10004000005C0040044B48F68F6253F8201001EA30
:10005000020243F820207047005C0040044B48F641
:100060008F6253F8201001EA020243F82020704703
:10007000005C0040054B48F68F6253F8201001EAFF
:10008000020242F4807243F820207047005C004076
:10009000054B48F68F6253F8201001EA020242F441
:1000A000807243F820207047005C0040044B48F603
:1000B0008F6253F8201001EA020243F820207047B3
:1000C000005C0040044B53F8200000F03000102882
:1000D00014BF002001207047005C0040054B53F81E
:1000E000200000F44050B0F5805F14BF00200120D4
:1000F000704700BF005C0040044B40F68F7253F81D
:10010000201001EA020243F820207047005C004002
:10011000044B48F60F7253F8201001EA020243F82C
:1001200020207047005C0040054B48F68F7253F862
:10013000201001EA020242F4804243F82020704776
:10014000005C0040054B48F68F7253F8201001EA1E
:10015000020242F0400243F820207047005C004059
:10016000084B53F8202012F4804F09D053F8201088
:1001700048F68F7201EA020242F4804243F82020DE
:10018000704700BF005C0040084B53F8202012F07D
:10019000400F09D053F8201048F68F7201EA02028E
:1001A00042F0400243F82020704700BF005C00404E
:1001B000054B10B553F8204048F68F7204EA02024E
:1001C0000A4343F8202010BD005C0040024B53F866
:1001D000200000F00F007047005C0040064B49080B
:1001E0001B6849009BB203EBC00303F1005303F506
:1001F00040535B0019607047505C0040054A064B55
:100200001268490892B202EBC002D3185B004900A1
:1002100019607047505C004004300020054B1B689B
:100220009BB203EBC00303F1005303F540535B00A3
:1002300018887047505C0040044A054B126892B21F
:1002400002EBC002D3185B0018887047505C004076
:1002500004300020044A054B126892B202EBC0023F
:10026000D3185B0019607047505C004002300020DA
:100270003E2909D94B0911F01F0F01D1013B9BB257
:100280009B0243F4004305E04B0811F0010F18BF37
:1002900001339B02036070470D4A0E4B126892B205
:1002A000D31803EBC0035B003E2909D94A0911F0BA
:1002B0001F0F01D1013A92B2920242F4004205E0CE
:1002C0004A0811F0010F18BF013292021A607047FC
:1002D000505C004006300020054A064B126892B27E
:1002E00002EBC002D3185B0018688005800D7047D0
:1002F000505C004002300020054A064B126892B262
:1003000002EBC002D3185B0018688005800D7047AF
:10031000505C0040063000200C4B30B51D681C6856
:10032000C0001FFA85FC8444A4B2094B00190CF1EB
:10033000005CC3180CF5405C490852084FEA4C00B9
:1003400049005B00520001601A6030BD505C004003
:1003500004300020064B49081B6849009BB203EBA0
:10036000C00303F1005303F540535B00196070476D
:10037000505C0040054A064B1268490892B202EBF5
:10038000C002D3185B00490019607047505C004000
:1003900004300020054B1B689BB203EBC00303F144
:1003A000005303F540535B0018887047505C0040D1
:1003B000044A054B126892B202EBC002D3185B00EC
:1003C00018887047505C004004300020012910B5A7
:1003D00024D1254B25491B68C0009BB25918091828
:1003E0004B003E2A09D9510912F01F0F01D10139E2
:1003F00089B2890241F4004105E0510812F0010F71
:1004000018BF0131890219601749194B096889B26F
:10041000CB18181840003E2A1ED913E0022922D119
:10042000114BC0001C681B68A4B21FFA83FC0F4963
:100430000F4B844400194118634449005B000A6073
:100440001A6010E0530912F01F0F01D1013B9BB25B
:100450009B0243F4004305E0530812F0010F18BF5C
:1004600001339B02036010BD505C0040023000204D
:100470000630002001291BD11349144B096889B2A9
:10048000CB1803EBC00040003E2A09D9530912F0F3
:100490001F0F01D1013B9BB29B0243F4004305E0D7
:1004A000530812F0010F18BF01339B0203600AE0EA
:1004B000022908D10449054B096889B201EBC00043
:1004C000C3185B001A607047505C00400230002087
:1004D00001291BD11349144B096889B2CB1803EBCE
:1004E000C00040003E2A09D9530912F01F0F01D164
:1004F000013B9BB29B0243F4004305E0530812F01A
:10050000010F18BF01339B0203600AE0022908D1E2
:100510000449054B096889B201EBC000C3185B00B0
:100520001A607047505C004006300020054A064BB8
:10053000126892B202EBC002D3185B001868800503
:10054000800D7047505C004002300020054A064B89
:10055000126892B202EBC002D3185B0018688005E3
:10056000800D7047505C0040063000200D4BC000ED
:1005700019680D4A89B241188A185200128812F47B
:100580007C4F01D001200CE01A68084B92B2801811
:10059000C3185B0018888005800D002814BF022056
:1005A00000207047505C00400630002002300020E0
:1005B000012909D10B4A48F68F7352F8201001EA3D
:1005C000030343F040030AE002290AD1054A48F632
:1005D0008F7352F8201001EA030343F4804342F87A
:1005E00020307047005C004041EA0020704700BFA7
:1005F000030AC0B243EA0020704700BF08B50022DA
:100600000A2300F045F808BD08B500210A2200F0D1
:10061000DFF808BDF0B40378002B2DD040F234127F
:10062000C2F20002156802E010F8013FEBB15A195E
:1006300003F12004527812F001070A7808BF1C4623
:1006400001F10101561C9446AE5D16F0010F18BF72
:1006500002F1200C6445E7D007B1203316F0010FFA
:1006600018BF2032981AF0BC70470A786F78561C71
:1006700007F00107AE5DEFE740F234100A78C2F2EE
:100680000000561C05686F78AE5D07F00107E3E7D0
:100690002DE9F04F40F23415C2F2000583B00C464C
:1006A0001F46D5F800800E460190009216F8015BB7
:1006B00008EB050393F801B01BF0080BF6D12D2DC4
:1006C00065D02B2D08BF16F8015BD7F1010338BFA9
:1006D0000023102F14BF1A4643F0010232B1302D0F
:1006E00066D01BB1302D0CBF08270A27BBF1000FC5
:1006F000394614BF4FF000496FF00049484600F0FA
:1007000059FC48468A46394600F026FB00218C46B3
:1007100008EB0502A5F13003527812F0040F08D15E
:1007200012F0030F20D012F0010F14BF372357230C
:10073000EB1A9F4218DD844594BF0022012252EA41
:10074000D1714FF0FF310CD1844514BF002201223A
:100750005345D4BF002202F0010212B907FB0C3C42
:10076000012116F8015BD3E7B1F1FF3F14D0BBF1D3
:10077000000F09D16046009B1BB101B1741E009AA5
:10078000146003B0BDE8F08FCCF10000F3E716F879
:10079000015B4FF0010B98E7019ABBF1000F4FF09E
:1007A000220314BF4FF000406FF000401360E2E7F7
:1007B0003278782A14BF00210121582A14BF0A4632
:1007C00041F00102002A8CD07578102702368DE79F
:1007D00010B540F23814C2F200048C4613460146AC
:1007E00062462068FFF754FF10BD00BF2DE9F043BB
:1007F0008BB006460F4600F07BF840F22C24C2F284
:10080000000494F90030B3F1FF3F8046894638D0A8
:100810003046394600F084FA0546002831D130468A
:1008200039460022002301F01DF8002829D1247840
:1008300042F67813C0F6010308950193CDE90267EB
:10084000CDE90467002C21D040F200030022CFF64E
:10085000F0733046CDE9062339460022002300F02C
:10086000D9FF002822D0022300939C4234D068464E
:1008700000F064FA00282FD0089B002B27D1DDE977
:100880000689404649460BB0BDE8F0834FF6FF733A
:100890004FF06042CCF2EF733046CDE90623394683
:1008A0000022002300F0B6FF0028DCD10123022C37
:1008B000009316D0684600F041FA90B142F67C10E1
:1008C000C0F6010000F03CFACDE90601D4E700F0E3
:1008D0003DFA089B0360D2E700F038FA2223036058
:1008E000CAE700F033FA21230360E7E700000000C5
:1008F000B1F5801F0B462DE9F04F804687B0894641
:1009000004460D463EDB4FF6FF720026C7F6EF7237
:10091000934251DC23F07F4445F6647C24F4700458
:10092000C0F2090CA44440F20002A6F57E760CF455
:10093000801C073EC3F6F0728CEA020206EB2356D7
:1009400040F20003404642EA0401C3F6F07300227D
:1009500006EB1C5600F042FBA31C23F07F4323F45C
:100960007003022B804689462FDC0022002300F012
:1009700051FF002800F0CA80002E40F07C8100204A
:1009800000211FE021F00043034300F0B58000295F
:10099000C0F2468140F200030022C4F250336FF0EF
:1009A000350600F0CFFC4FF6FF72C7F6EF720B462C
:1009B000804693428946ADDD4046494642464B4615
:1009C00000F00EFB07B0BDE8F08F00224FF080432F
:1009D00000F006FB4EF68635CFF6F975651902462E
:1009E0000B464046494600F0D7FDCDE902013046AE
:1009F00000F042FCCDE90401DDE9020102460B46AC
:100A000000F0A0FC02460B46CDE9000100F09AFC84
:100A1000A7A3D3E9002382468B4600F093FCA6A34C
:100A2000D3E9002300F0DCFA52465B4600F08AFC72
:100A3000A3A3D3E9002300F0D3FA52465B4600F0AB
:100A400081FCA1A3D3E9002300F0CAFADDE9002369
:100A500000F078FC9EA3D3E90023CDE900015046C5
:100A6000594600F06FFC9CA3D3E9002300F0B8FACC
:100A700052465B4600F066FC99A3D3E9002300F0E0
:100A8000AFFA52465B4600F05DFC0B460246DDE9DC
:100A9000000100F0A5FA4BF65103C0F206031B1B40
:100AA00043EA0505002D82468B4656DD40F20003E1
:100AB0000022C3F6E0734046494600F043FC42463C
:100AC0004B4600F03FFC04460D46002E75D15246C1
:100AD0005B4600F085FADDE9022300F033FC0246B4
:100AE0000B462046294600F079FA02460B4640465E
:100AF000494600F073FA65E740F200010020002249
:100B00000023CCF2503100F047FD5BE742464B46F4
:100B10004046494600F016FC73A3D3E9002304467F
:100B20000D464046494600F00DFC40F2000300220D
:100B3000C3F6E07300F054FA02460B4620462946FD
:100B400000F000FC04460D46002E72D14046494696
:100B500022462B4600F042FA34E7002E00F0D48003
:100B600063A3D3E90023DDE9040100F0EBFB524667
:100B70005B4606460F464046494600F02FFADDE93F
:100B8000022300F0DFFB5CA3D3E9002304460D46FB
:100B9000DDE9040100F0D6FB02460B46204629465B
:100BA00000F01EFA42464B4600F018FA02460B4689
:100BB0003046394600F012FA04E74DA3D3E900238A
:100BC000DDE9040100F0BEFB52465B46CDE90001C1
:100BD0002046294600F004FADDE9022300F0B2FBCA
:100BE00047A3D3E9002306460F46DDE9040100F0E0
:100BF000A9FB02460B463046394600F0F1F90246A1
:100C00000B462046294600F0E9F942464B4600F0E3
:100C1000E5F902460B46DDE9000100F0DFF9D1E617
:100C200002460B4600F0DAF90022002300F0B4FC83
:100C3000C8E6304600F020FB2DA3D3E9002306468A
:100C40000F4600F07FFB2CA3D3E9002382468B469E
:100C50003046394600F076FB22462B4600F0C0F9BC
:100C600042464B4600F0BAF902460B4650465946FA
:100C700000F0B4F9A6E6304600F0FEFA1CA3D3E972
:100C8000002306460F4600F05DFB1DA3D3E90023B9
:100C900004460D463046394600F054FB02460B46EA
:100CA0002046294600F09CF98CE600BFAFF3008097
:100CB00044523EDF12F1C23FDE03CB966446C73F8B
:100CC000599322942449D23F935555555555E53FA4
:100CD0009FC678D0099AC33FAF788E1DC571CC3FAF
:100CE00004FA97999999D93F555555555555D5BFFA
:100CF0000000E0FE422EE63F763C7935EF39EABD52
:100D0000763C7935EF39EA3D02460B464046494686
:100D100000F064F9DDE9022300F014FBE5E600BF12
:100D200002464042104321F0004141EAD070C0F138
:100D3000FE4000F57000C00F704700BF00207047F4
:100D400040F200010020C7F6F871704740F23813F6
:100D5000C2F20003186870474A1E08BF7047C0F00F
:100D60002481884240F21681114200F01781B0FAC6
:100D700080F3B1FA81F2A2EB0303C3F11F0304A2D3
:100D800002EB03134FF000029F4600BFAFF3008059
:100D9000B0EBC17F00BF42EB020228BFA0EBC170E5
:100DA000B0EB817F00BF42EB020228BFA0EB817055
:100DB000B0EB417F00BF42EB020228BFA0EB4170C5
:100DC000B0EB017F00BF42EB020228BFA0EB017035
:100DD000B0EBC16F00BF42EB020228BFA0EBC160C5
:100DE000B0EB816F00BF42EB020228BFA0EB816035
:100DF000B0EB416F00BF42EB020228BFA0EB4160A5
:100E0000B0EB016F00BF42EB020228BFA0EB016014
:100E1000B0EBC15F00BF42EB020228BFA0EBC150A4
:100E2000B0EB815F00BF42EB020228BFA0EB815014
:100E3000B0EB415F00BF42EB020228BFA0EB415084
:100E4000B0EB015F00BF42EB020228BFA0EB0150F4
:100E5000B0EBC14F00BF42EB020228BFA0EBC14084
:100E6000B0EB814F00BF42EB020228BFA0EB8140F4
:100E7000B0EB414F00BF42EB020228BFA0EB414064
:100E8000B0EB014F00BF42EB020228BFA0EB0140D4
:100E9000B0EBC13F00BF42EB020228BFA0EBC13064
:100EA000B0EB813F00BF42EB020228BFA0EB8130D4
:100EB000B0EB413F00BF42EB020228BFA0EB413044
:100EC000B0EB013F00BF42EB020228BFA0EB0130B4
:100ED000B0EBC12F00BF42EB020228BFA0EBC12044
:100EE000B0EB812F00BF42EB020228BFA0EB8120B4
:100EF000B0EB412F00BF42EB020228BFA0EB412024
:100F0000B0EB012F00BF42EB020228BFA0EB012093
:100F1000B0EBC11F00BF42EB020228BFA0EBC11023
:100F2000B0EB811F00BF42EB020228BFA0EB811093
:100F3000B0EB411F00BF42EB020228BFA0EB411003
:100F4000B0EB011F00BF42EB020228BFA0EB011073
:100F5000B0EBC10F00BF42EB020228BFA0EBC10003
:100F6000B0EB810F00BF42EB020228BFA0EB810073
:100F7000B0EB410F00BF42EB020228BFA0EB4100E3
:100F8000B0EB010F00BF42EB020228BFA0EB010053
:100F9000104670470CBF012000207047B1FA81F263
:100FA000C2F11F0220FA02F0704708B14FF0FF3083
:100FB00000F00EB80029F8D02DE90340FFF7CCFE71
:100FC000BDE8064002FB00F3A1EB0301704700BF40
:100FD000704700BF81F0004102E000BF83F0004392
:100FE00030B54FEA41044FEA430594EA050F08BFC4
:100FF00090EA020F1FBF54EA000C55EA020C7FEA88
:10100000645C7FEA655C00F0E2804FEA5454D4EB04
:101010005555B8BF6D420CDD2C4480EA020281EACE
:10102000030382EA000083EA010180EA020281EA06
:101030000303362D88BF30BD11F0004F4FEA013158
:101040004FF4801C4CEA113102D0404261EB410167
:1010500013F0004F4FEA03334CEA133302D05242ED
:1010600063EB430394EA050F00F0A780A4F10104A9
:10107000D5F1200E0DDB02FA0EFC22FA05F28018E3
:1010800041F1000103FA0EF2801843FA05F35941C9
:101090000EE0A5F120050EF1200E012A03FA0EFC48
:1010A00028BF4CF0020C43FA05F3C01851EBE37172
:1010B00001F0004507D54FF0000EDCF1000C7EEB8F
:1010C00000006EEB0101B1F5801F1BD3B1F5001FCD
:1010D0000CD349085FEA30004FEA3C0C04F10104EC
:1010E0004FEA445212F5800F80F09A80BCF1004F15
:1010F00008BF5FEA500C50F1000041EB045141EA97
:10110000050130BD5FEA4C0C404141EB010111F497
:10111000801FA4F10104E9D191F0000F04BF014642
:101120000020B1FA81F308BF2033A3F10B03B3F120
:1011300020020CDA0C3208DD02F1140CC2F10C02B0
:1011400001FA0CF021FA02F10CE002F11402D8BF0E
:10115000C2F1200C01FA02F120FA0CFCDCBF41EADA
:101160000C019040E41AA2BF01EB0451294330BDA9
:101170006FEA04041F3C1CDA0C340EDC04F1140486
:10118000C4F1200220FA04F001FA02F340EA03005D
:1011900021FA04F345EA030130BDC4F10C04C4F1A3
:1011A000200220FA02F001FA04F340EA0300294683
:1011B00030BD21FA04F0294630BD94F0000F83F4CD
:1011C000801306BF81F480110134013D4EE77FEAB0
:1011D000645C18BF7FEA655C29D094EA050F08BFFC
:1011E00090EA020F05D054EA000C04BF19461046DD
:1011F00030BD91EA030F1EBF0021002030BD5FEA21
:10120000545C05D14000494128BF41F0004130BD48
:1012100014F580043CBF01F5801130BD01F000459C
:1012200045F0FE4141F470014FF0000030BD7FEA0F
:10123000645C1ABF194610467FEA655C1CBF0B460A
:10124000024650EA013406BF52EA033591EA030F21
:1012500041F4002130BD00BF90F0000F04BF002119
:10126000704730B54FF4806404F132044FF000054C
:101270004FF0000150E700BF90F0000F04BF0021C5
:10128000704730B54FF4806404F1320410F000452B
:1012900048BF40424FF000013EE700BF42004FEA26
:1012A000E2014FEA31014FEA02701FBF12F07F43A3
:1012B00093F07F4F81F06051704792F0000F14BFA0
:1012C00093F07F4F704730B54FF4607401F00045E4
:1012D00021F0004120E700BF50EA010208BF70473B
:1012E00030B54FF000050AE050EA010208BF704730
:1012F00030B511F0004502D5404261EB41014FF499
:10130000806404F132045FEA915C3FF4DCAE4FF09C
:1013100003025FEADC0C18BF03325FEADC0C18BF83
:10132000033202EBDC02C2F1200300FA03FC20FAD4
:1013300002F001FA03FE40EA0E0021FA02F1144421
:10134000C1E600BF70B54FF0FF0C4CF4E06C1CEA36
:1013500011541DBF1CEA135594EA0C0F95EA0C0FAB
:1013600000F0DEF82C4481EA030621EA4C5123EA1E
:101370004C5350EA013518BF52EA033541F480114D
:1013800043F4801338D0A0FB02CE4FF00005E1FB00
:1013900002E506F00042E0FB03E54FF00006E1FB4A
:1013A00003569CF0000F18BF4EF0010EA4F1FF048D
:1013B000B6F5007F64F5407404D25FEA4E0E6D41CD
:1013C00046EB060642EAC62141EA55514FEAC520DE
:1013D00040EA5E504FEACE2EB4F1FD0C88BFBCF55A
:1013E000E06F1ED8BEF1004F08BF5FEA500E50F10B
:1013F000000041EB045170BD06F0004646EA0101D1
:1014000040EA020081EA0301B4EB5C04C2BFD4EB02
:101410000C0541EA045170BD41F480114FF0000EFB
:10142000013C00F3AB8014F1360FDEBF002001F069
:10143000004170BDC4F10004203C35DA0C341BDCE3
:1014400004F11404C4F1200500FA05F320FA04F0B5
:1014500001FA05F240EA020001F0004221F00041E9
:1014600010EBD37021FA04F642EB06015EEA430E5C
:1014700008BF20EAD37070BDC4F10C04C4F120058C
:1014800000FA04F320FA05F001FA04F240EA02003F
:1014900001F0004110EBD37041F100015EEA430E10
:1014A00008BF20EAD37070BDC4F1200500FA05F230
:1014B0004EEA020E20FA04F301FA05F243EA0203AF
:1014C00021FA04F001F0004121FA04F220EA0200BE
:1014D00000EBD3705EEA430E08BF20EAD37070BD04
:1014E00094F0000F0FD101F00046400041EB0101E4
:1014F00011F4801F08BF013CF7D041EA060195F0C6
:10150000000F18BF704703F00046520043EB03037F
:1015100013F4801F08BF013DF7D043EA060370476C
:1015200094EA0C0F0CEA135518BF95EA0C0F0CD077
:1015300050EA410618BF52EA4306D1D181EA0301BD
:1015400001F000414FF0000070BD50EA410606BFB7
:101550001046194652EA430619D094EA0C0F02D1FC
:1015600050EA013613D195EA0C0F05D152EA033641
:101570001CBF104619460AD181EA030101F000415F
:1015800041F0FE4141F470014FF0000070BD41F0A8
:10159000FE4141F4780170BD70B54FF0FF0C4CF482
:1015A000E06C1CEA11541DBF1CEA135594EA0C0FA1
:1015B00095EA0C0F00F0A7F8A4EB050481EA030EEE
:1015C00052EA03354FEA013100F088804FEA0333D5
:1015D0004FF0805545EA131343EA12634FEA0222A3
:1015E00045EA111545EA10654FEA00260EF0004164
:1015F0009D4208BF964244F1FD0404F5407402D2B6
:101600005B084FEA3202B61A65EB03055B084FEA46
:1016100032024FF480104FF4002CB6EB020E75EB43
:10162000030E22BFB61A754640EA0C005B084FEA6B
:101630003202B6EB020E75EB030E22BFB61A7546E8
:1016400040EA5C005B084FEA3202B6EB020E75EB33
:10165000030E22BFB61A754640EA9C005B084FEAAB
:101660003202B6EB020E75EB030E22BFB61A7546B8
:1016700040EADC0055EA060E18D04FEA051545EAA7
:1016800016754FEA06164FEAC30343EA52734FEA50
:10169000C2025FEA1C1CC0D111F4801F0BD141EAC9
:1016A00000014FF000004FF0004CB6E711F4801F2E
:1016B00004BF01430020B4F1FD0C88BFBCF5E06F0E
:1016C0003FF6AFAEB5EB030C04BFB6EB020C5FEA1E
:1016D000500C50F1000041EB045170BD0EF0004E73
:1016E0004EEA113114EB5C04C2BFD4EB0C0541EAA5
:1016F000045170BD41F480114FF0000E013C90E6A2
:1017000045EA060E8DE60CEA135594EA0C0F08BF65
:1017100095EA0C0F3FF43BAF94EA0C0F0AD150EA64
:1017200001347FF434AF95EA0C0F7FF425AF1046F7
:1017300019462CE795EA0C0F06D152EA03353FF41F
:10174000FDAE1046194622E750EA410618BF52EA9C
:1017500043067FF4C5AE50EA41047FF40DAF52EA70
:1017600043057FF4EBAE12E74FF0FF3C06E000BF0D
:101770004FF0010C02E000BF4FF0010C4DF804CD1A
:101780004FEA410C7FEA6C5C4FEA430C18BF7FEADA
:101790006C5C1BD001B050EA410C0CBF52EA430C08
:1017A00091EA030F02BF90EA020F0020704710F188
:1017B000000F91EA030F58BF994208BF90422CBF17
:1017C000D8176FEAE37040F0010070474FEA410C10
:1017D0007FEA6C5C02D150EA013C07D14FEA430C2E
:1017E0007FEA6C5CD6D152EA033CD3D05DF8040B9F
:1017F000704700BF8446104662468C4619466346D1
:1018000000E000BF01B5FFF7B7FF002848BF10F1A7
:10181000000F01BD4DF808EDFFF7F4FF0CBF0120EC
:1018200000205DF808FB00BF4DF808EDFFF7EAFF68
:1018300034BF012000205DF808FB00BF4DF808ED23
:10184000FFF7E0FF94BF012000205DF808FB00BF18
:101850004DF808EDFFF7CEFF94BF012000205DF8A2
:1018600008FB00BF4DF808EDFFF7C4FF34BF0120AF
:1018700000205DF808FB00BF4FEA410212F500129C
:1018800015D211D56FF47873B3EB625212D94FEAC7
:10189000C12343F0004343EA505311F0004F23FAB1
:1018A00002F018BF404270474FF00000704750EA06
:1018B000013005D111F0004008BF6FF000407047C3
:1018C0004FF00000704700BF4FEA4102B2F1E04321
:1018D00024BFB3F5001CDCF1FE5C0DD901F0004C17
:1018E0004FEAC0024CEA5070B2F1004F40EB830067
:1018F00008BF20F00100704711F0804F21D113F193
:101900003872BCBF01F00040704741F480114FEACB
:101910005252C2F11802C2F1200C10FA0CF320FA54
:1019200002F018BF40F001004FEAC1234FEAD32371
:1019300003FA0CFC40EA0C0023FA02F34FEA4303DB
:10194000CCE77FEA625307D150EA01331EBF4FF064
:10195000FE4040F44000704701F0004040F0FE407F
:1019600040F40000704700BF80F0004002E000BF7C
:1019700081F0004142001FBF5FEA410392EA030F7A
:101980007FEA226C7FEA236C6AD04FEA1262D2EBC4
:101990001363C1BFD218414048404140B8BF5B42C9
:1019A000192B88BF704710F0004F40F4000020F062
:1019B0007F4018BF404211F0004F41F4000121F078
:1019C0007F4118BF494292EA030F3FD0A2F10102C2
:1019D00041FA03FC10EB0C00C3F1200301FA03F100
:1019E00000F0004302D5494260EB4000B0F5000F23
:1019F00013D3B0F1807F06D340084FEA310102F1E2
:101A00000102FE2A51D2B1F1004F40EBC25008BF93
:101A100020F0010040EA03007047490040EB00005D
:101A200010F4000FA2F10102EDD1B0FA80FCACF18C
:101A3000080CB2EB0C0200FA0CF0AABF00EBC2508B
:101A400052421843BCBFD0401843704792F0000F79
:101A500081F4000106BF80F400000132013BB5E7CC
:101A60004FEA41037FEA226C18BF7FEA236C21D042
:101A700092EA030F04D092F0000F08BF08467047A7
:101A800090EA010F1CBF0020704712F07F4F04D175
:101A9000400028BF40F00040704712F100723CBF88
:101AA00000F50000704700F0004343F0FE4040F4B2
:101AB000000070477FEA226216BF08467FEA236370
:101AC0000146420206BF5FEA412390EA010F40F45B
:101AD000800070474FF0000304E000BF10F00043A7
:101AE00048BF40425FEA000C08BF704743F096438E
:101AF00001464FF000001CE050EA010208BF7047A9
:101B00004FF000030AE000BF50EA010208BF70472F
:101B100011F0004302D5404261EB41015FEA010C44
:101B200002BF84460146002043F0B64308BFA3F13C
:101B30008053A3F50003BCFA8CF2083AA3EBC2531E
:101B400010DB01FA02FC634400FA02FCC2F120023D
:101B5000BCF1004F20FA02F243EB020008BF20F074
:101B60000100704702F1200201FA02FCC2F12002DA
:101B700050EA4C0021FA02F243EB020008BF20EACF
:101B8000DC7070474FF0FF0C1CEAD0521EBF1CEAFD
:101B9000D15392EA0C0F93EA0C0F6FD01A4480EAEB
:101BA000010C400218BF5FEA41211ED04FF00063D4
:101BB00043EA501043EA5111A0FB01310CF0004000
:101BC000B1F5000F3EBF490041EAD3715B0040EA26
:101BD000010062F17F02FD2A1DD8B3F1004F40EBF6
:101BE000C25008BF20F00100704790F0000F0CF0C9
:101BF000004C08BF49024CEA502040EA51207F3A8D
:101C0000C2BFD2F1FF0340EAC250704740F4000067
:101C10004FF00003013A5DDC12F1190FDCBF00F058
:101C200000407047C2F10002410021FA02F1C2F106
:101C3000200200FA02FC5FEA310040F1000053EAA2
:101C40004C0308BF20EADC70704792F0000F00F0F0
:101C5000004C02BF400010F4000F013AF9D040EAF6
:101C60000C0093F0000F01F0004C02BF490011F48A
:101C7000000F013BF9D041EA0C018FE70CEAD15388
:101C800092EA0C0F18BF93EA0C0F0AD030F0004C08
:101C900018BF31F0004CD8D180EA010000F00040BC
:101CA000704790F0000F17BF90F0004F084691F07A
:101CB000000F91F0004F14D092EA0C0F01D14202B4
:101CC0000FD193EA0C0F03D14B0218BF084608D17D
:101CD00080EA010000F0004040F0FE4040F40000C7
:101CE000704740F0FE4040F4400070474FF0FF0C5A
:101CF0001CEAD0521EBF1CEAD15392EA0C0F93EAA1
:101D00000C0F69D0A2EB030280EA010C49024FEAF2
:101D1000402037D04FF0805343EA111143EA1013AB
:101D20000CF000408B4238BF5B0042F17D024FF463
:101D3000000C8B4224BF5B1A40EA0C00B3EB510F3E
:101D400024BFA3EB510340EA5C00B3EB910F24BF27
:101D5000A3EB910340EA9C00B3EBD10F24BFA3EBAC
:101D6000D10340EADC001B0118BF5FEA1C1CE0D174
:101D7000FD2A3FF650AF8B4240EBC25008BF20F027
:101D8000010070470CF0004C4CEA50207F32C2BF7B
:101D9000D2F1FF0340EAC250704740F400004FF018
:101DA0000003013A37E792F0000F00F0004C02BF49
:101DB000400010F4000F013AF9D040EA0C0093F013
:101DC000000F01F0004C02BF490011F4000F013B6D
:101DD000F9D041EA0C0195E70CEAD15392EA0C0FD5
:101DE00008D142027FF47DAF93EA0C0F7FF470AF0D
:101DF000084676E793EA0C0F04D14B023FF44CAF50
:101E000008466EE730F0004C18BF31F0004CCAD1E4
:101E100030F000427FF45CAF31F000437FF43CAF20
:101E20005FE700BF4FF0FF3C06E000BF4FF0010C42
:101E300002E000BF4FF0010C4DF804CD4FEA400224
:101E40004FEA41037FEA226C18BF7FEA236C11D06E
:101E500001B052EA530C18BF90EA010F58BFB2EB21
:101E6000030088BFC81738BF6FEAE17018BF40F0A1
:101E7000010070477FEA226C02D15FEA402C05D155
:101E80007FEA236CE4D15FEA412CE1D05DF8040BDA
:101E9000704700BF844608466146FFE70FB5FFF76D
:101EA000C9FF002848BF10F1000F0FBD4DF808ED25
:101EB000FFF7F4FF0CBF012000205DF808FB00BF16
:101EC0004DF808EDFFF7EAFF34BF012000205DF870
:101ED00008FB00BF4DF808EDFFF7E0FF94BF0120BD
:101EE00000205DF808FB00BF4DF808EDFFF7D2FFBA
:101EF00094BF012000205DF808FB00BF4DF808EDFD
:101F0000FFF7C8FF34BF012000205DF808FB00BFC9
:101F100042000ED2B2F1FE4F0BD34FF09E03B3EB53
:101F2000126209D44FEA002343F0004323FA02F07F
:101F300070474FF00000704712F1610F01D142026B
:101F400002D14FF0FF3070474FF00000704700BFE4
:101F500073B96AB9002908BF0028BCBF00204FF040
:101F60000041C4BF6FF000414FF0FF30FFF730B8C1
:101F700082B0EC462DE9005000F01CF8DDF804E0DA
:101F800002B00CBC704700BFF8B514461D460646AB
:101F90000F4600F0D3F900FB05F5A0FB042304FB7A
:101FA0000154E318B61A67EB0307069BC3E9006701
:101FB000F8BD00BFF8B514461D4606460F4600F0B2
:101FC0000FF800FB05F5A0FB042304FB0154E31804
:101FD000B61A67EB0307069BC3E90067F8BD00BFAD
:101FE00000292DE9F04F85B0C0F2C9800026002BF2
:101FF000C0F2C0808946144605469B46002B4BD153
:102000008A4258D9B2FA82F353B1C3F1200001FADF
:1020100003F925FA00F812FA03F49D4048EA090989
:10202000270C484639461FFA84FBFEF795FE3946D1
:1020300082464846FEF7BEFF4FEA15420BFB0AF305
:1020400042EA01494B4509D919EB04090AF1FF3A63
:1020500004D24B4584BF0AF1FF3AA144C3EB0909FE
:1020600039464846ADB2FEF777FE394680464846C7
:10207000FEF7A0FF0BFB08FB45EA0145AB4507D97E
:102080002D1908F1FF3803D2AB4588BF08F1FF389E
:1020900048EA0A48002703E08B4257D90027B84690
:1020A00042463B4616B1524263EB43031946104683
:1020B00005B0BDE8F08F22B911460120FEF74CFEB5
:1020C0000446B4FA84F8B8F1000F5ED1C4EB0908F5
:1020D000270C1FFA84F90121029139464046FEF788
:1020E0003BFE394682464046FEF764FF4FEA1548FC
:1020F00009FB0AF348EA014B5B4509D91BEB040BCA
:102100000AF1FF3A04D25B4584BF0AF1FF3AA344C7
:10211000C3EB0B0B39465846ADB2FEF71DFE3946F0
:1021200080465846FEF746FF09FB08F945EA014597
:10213000A94507D92D1908F1FF3803D2A94588BF51
:1021400008F1FF3848EA0A48029FA9E7B3FA83F783
:10215000002F67D18B422CBF4FF000094FF00109CF
:1021600082428CBF4C4649F00104002C96D04FF0BF
:10217000010895E7524263EB4303F6433AE74042D6
:1021800061EB41014FF0FF3631E704FA08F4C8F182
:10219000200735FA07F329FA07FA270C09FA08FB92
:1021A0003946504643EA0B020292FEF7D5FD394606
:1021B0001FFA84F983465046FEF7FCFE029809FB9D
:1021C0000BF2030C43EA01439A4204D91B190BF1A9
:1021D000FF3BC0F0AD809B1A394618460193FEF7CD
:1021E000BBFD0199824608463946FEF7E3FE029898
:1021F00009FB0AF31FFA80FC4CEA0142934208D91A
:1022000012190AF1FF3A04D2934284BF0AF1FF3A4D
:10221000121905FA08F54AEA0B4EC3EB0208CDF88D
:1022200008E05AE7C7F1200003FA07FAC24035FA7E
:1022300000F342EA0A0B21FA00F801FA07F94046D6
:102240004FEA1B4A43EA0901029151461FFA8BF2F9
:102250000392FEF781FD514681464046FEF7AAFEF5
:102260000398029B00FB09F2180C14FA07F340EAEA
:102270000144A24204D914EB0B0409F1FF3951D3F4
:10228000A41A514620460193FEF766FD514680464A
:102290002046FEF78FFE039C019B04FB08F2029C84
:1022A0001FFA84FC4CEA0140824204D910EB0B0077
:1022B00008F1FF3830D348EA09481FFA83FC1B0CA9
:1022C000801A1FFA88FE4FEA184A0CFB0EF90CFB25
:1022D0000AF203FB0E2103FB0AF301EB19418A42C8
:1022E00088BF03F5803303EB114E704510D31FFAFE
:1022F00089F905FA07F709EB014014BF0022012212
:1023000087422CBF002702F00107002F3FF4C8AE20
:1023100008F1FF380027C3E6824284BF584408F121
:10232000FF38C8E7A24284BF09F1FF395C44A7E740
:102330009A4284BF0BF1FF3B1B194CE72DE9F04F8C
:102340000C4683B08046164689461F4615468A4687
:10235000002B4BD18A425CD9B2FA82F35BB1C3F154
:10236000200001FA03FA28FA00F216FA03F508FA37
:1023700003F842EA0A0A2E0C50463146AFB2FEF785
:10238000EBFC31464FEA184481465046FEF712FEF8
:1023900007FB09F344EA014A534509D91AEB050A38
:1023A00009F1FF3904D2534584BF09F1FF39AA442A
:1023B000C3EB0A0A314650461FFA88F8FEF7CCFCF8
:1023C000314604465046FEF7F5FD07FB04F748EAA0
:1023D0000148474506D9013C18EB050802D247459C
:1023E00088BF013C44EA094400265CE08B4258D88F
:1023F000B3FA83F6002E5BD18B422CBF0022012260
:1024000085428CBF154642F00105002D49D00124BC
:1024100049E022B911460120FEF79EFC0546B5FAB7
:1024200085F6002E40F0BB80641B2F0C1FFA85FA46
:10243000012639462046FEF78FFC39464FEA184BF5
:1024400081462046FEF7B6FD0AFB09F34BEA014B35
:102450005B4509D91BEB050B09F1FF3904D25B453C
:1024600084BF09F1FF39AB44C3EB0B0B3946584627
:102470001FFA88F8FEF770FC394604465846FEF706
:1024800099FD0AFB04FA48EA0148C24506D9013C15
:1024900018EB050802D2C24588BF013C44EA094452
:1024A00001E0002634463146204603B0BDE8F08FF7
:1024B000C6F12000B34032FA00F721FA00FB1F43B7
:1024C00014FA06F228FA00F158464FEA174A114367
:1024D00000915146BBB20193FEF73EFC5146B54018
:1024E00081465846FEF766FD019C009804FB09F3FF
:1024F0004FEA104C4CEA014B5B4505D91BEB070B2F
:1025000009F1FF39C0F08F80C3EB0B0B51465846E1
:10251000FEF722FC514604465846FEF74BFD019853
:10252000009A00FB04F31FFA82FC4CEA014293423A
:1025300006D9013CD21903D2934201D9D219013CE8
:1025400044EA0944A8B2D21A2D0C1FFA84FC4FEABF
:10255000144300FB0CF700FB03FE05FB0CE105FB3D
:1025600003F501EB17418E4588BF05F5803505EB76
:102570001145AA4210D3BFB208FA06F607EB014292
:1025800014BF4FF0000E4FF0010E96422CBF0026F4
:102590000EF00106002E86D0013C002683E7B540F0
:1025A000C6F1200124FA01F928FA01F22F0CB440F7
:1025B0003946484622430092FEF7CEFB39461FFAC1
:1025C00085FA83464846FEF7F5FC009B1A0C0AFB89
:1025D0000BF342EA0144A34203D964190BF1FF3B18
:1025E00027D3E41A39462046FEF7B6FB3946814622
:1025F0002046FEF7DFFC00980AFB09F31FFA80FC77
:102600004CEA0144A34208D9641909F1FF3904D204
:10261000A34284BF09F1FF39641908FA06F8E41AE5
:1026200049EA0B4605E75B4584BF09F1FF39BB4426
:102630006AE7A34284BF0BF1FF3B6419D1E700BFF7
:102640000000000000000000010003E8000000009E
:1026500000000003E800000000000200FA0600038A
:10266000000000000037060000000000000000002D
:10267000F401000064000000018008080000000070
:10268000006400000000000000000000C80000001E
:102690001201100102000040D0169E05011801022F
:1026A0000301000009024300020100C032090400D6
:1026B00000010202010005240010010524010001AF
:1026C000042402020524060001070582030800FF16
:1026D00009040100020A000000070503024000008F
:1026E000070581024000000004030904260354008A
:1026F000720069006E0061006D00690063004D00AA
:102700006F00740069006F006E00200043007400C9
:102710006C000000320354004D0043004D002D00BA
:1027200031003100340030002000280076006900BC
:1027300072007400750061006C00200043004F00BF
:102740004D00290020000000524F520000010652A7
:102750004F4C000002064D5354000003024D5650EA
:102760000000040753415000000507474150000096
:1027700006035354415000070352534150000803CD
:102780005347500000090747475000000A035354BD
:102790004750000B0352534750000C03524653005E
:1027A000000D0353494F00000E0747494F00000F2B
:1027B0000353414300001D0753434F00001E0747CA
:1027C000434F00001F0343434F0000200341434F8A
:1027D00000002703554630000040075546310000F1
:1027E0004107554632000042075546330000430773
:1027F0005546340000440755463500004507554608
:1028000036000046075546370000470752554E0030
:1028100000810553544F5000800042494E00008B08
:1028200000000000000000000200000000000001A5
:102830000000000001020304010203040607080966
:102840000204060800202020202020202020282804
:102850002828282020202020202020202020202060
:1028600020202020208810101010101010101010A0
:1028700010101010100404040404040404040410D0
:10288000101010101010414141414141010101015E
:102890000101010101010101010101010101010128
:1028A0001010101010104242424242420202020234
:1028B00002020202020202020202020202020202F8
:1028C00010101010200000000000000000000000A8
:1028D00000000000000000000000000000000000F8
:1028E00000000000000000000000000000000000E8
:1028F00000000000000000000000000000000000D8
:1029000000000000000000000000000000000000C7
:1029100000000000000000000000000000000000B7
:1029200000000000000000000000000000000000A7
:102930000000000000000000000000000000000097
:1029400000000000000000003131343056313234D4
:10295000004142530052454C00434F4F52440053F4
:10296000544152540053544F500053544154555302
:1029700000000000430000006C6F670000000000D2
:0829800060F6FF7F010000007A
:1029880048290108000100000001020000080000B9
:10299800010000000200000000000000000000002C
:1029A800000000000000000000000000000000001F
:1029B800000000000000000000000000000000000F
:1029C800000000000000000000C201000000080034
:1029D800E826010804000000EC2601082600000093
:1029E8001427010832000000B00000201A0000007F
:1029F800A4260108430000009026010812000000E8
:102A0800699B00088599000895970008A997000810
:102A1800AD9700080D9800083198000875990008CE
:102A28006599000841990008000000004000000076
:102A38001A0354004D0043003100310034003000C7
:102A4800000000000000000000000000959600084B
:102A5800E9F50008E9F50008E9F50008E9F50008D6
:102A6800E9F50008E9F50008E9F50008E9F50008C6
:102A7800D59A0008E9F50008E9F50008E9F5000825
:102A8800E9F5000804010000E9F50008719700085D
:102A9800E9F50008E9F50008E9F50008E9F5000896
:102AA800E9F50008E9F50008899700080100000029
:102AB80045280108442801083C01002000000000C6
:102AC80000000000000000000000000000000000FE
:102AD8000000000000000000000000007429010848
:102AE80000000000000000000000000000000000DE
:102AF80000000000000000000000000000000000CE
:102B080000000000000000000000000000000000BD
:102B180000000000000000000000000000000000AD
:102B2800000000000000000000000000000000009D
:102B3800000000000000000000000000000000008D
:102B4800000000000000000000000000000000007D
:102B5800000000000000000000000000000000006D
:102B6800000000000000000000000000000000005D
:102B7800000000000000000000000000000000004D
:102B8800000000000000000000000000000000003D
:102B9800000000000000000000000000000000002D
:102BA800000000000000000000000000010000001C
:04000005080041109E
:00000001FF
